:100000000C9475060C9494060C9494060C94940627
:100010000C9494060C9494060C940E090C944D09BF
:100020000C9494060C9494060C9494060C949406E8
:100030000C9494060C9494060C9494060C94C30CA3
:100040000C9494060C9494060C9494060C949406C8
:100050000C9478400C949A370C9494060C94940663
:100060000C9494060C946F380C9494060C9463389A
:100070000C9494060C9494060C9494060C94940698
:100080000C94244D0C9494060C9494060C949406B1
:100090000C94AD380C9494060C94A1380C949406EE
:1000A0000C9494060C9494060C9494060C94940668
:1000B0000C9494060C9494060C9494060C94940658
:1000C0000C9494060C9494060C9494060C94940648
:1000D0000C9494060C9494060C9494060C94940638
:1000E0000C9494060C9431400C943B400C942740A3
:1000F0000C94E13F0C946C400C945D400C94514086
:100100000C9445400C9494060C9494060C9494061C
:100110000C9494060C9494060C9494060C949406F7
:100120000A0025303278002025362E3266204F6EA8
:100130002D426F61726400202573002530327800F3
:100140002025362E3266200020257300756E6B6EDA
:100150006F776E20636D640A00256300682020209D
:10016000202020202020202020202020202020208F
:1001700020202020202020202D2068656C700A0D72
:100180000076202020202020202020202020202039
:10019000202020202020202020202020202D2076FC
:1001A000657273696F6E0A0D007520202020202073
:1001B000202020202020202020202020202020203F
:1001C00020202020202D20757074696D650A0D0097
:1001D000616573205B6F6E7C6F66665D20202020FA
:1001E0002020202020202020202020202D20696E6B
:1001F000746567726574790A0D006164632020205C
:1002000020202020202020202020202020202020EE
:100210002020202020202D2073686F7720765F69B2
:100220006E2C2061312C20613220766F6C746167F6
:1002300065730A0D0063616C69205B5B765F696EB4
:100240007C61317C61325D20766F6C746167655DC5
:10025000202D2063616C6962726174650A0D00640F
:1002600065205B6D61736B5D2020202020202020A5
:1002700020202020202020202020202D20646562A6
:1002800075670A0D0068756D202020202020202031
:10029000202020202020202020202020202020205E
:1002A000202D2068756D69646974792073656E739B
:1002B0006F720A0D0068756D70205B6F6E7C6F66E3
:1002C000665D2020202020202020202020202020AB
:1002D000202D2068756D6964697479207065726D70
:1002E0002073656E736F72207077720A0D006964F7
:1002F000205B72657365745D202020202020202003
:10030000202020202020202020202D20696420680B
:10031000616E646C696E670A0D006D637520202044
:1003200020202020202020202020202020202020CD
:100330002020202020202D206D637520696E666F9F
:100340000A0D006E65205B666C7573685D20202069
:100350002020202020202020202020202020202D90
:10036000206E65696768626F72207461626C650AED
:100370000D006C6F67205B6175746F7C6F6E7C6FB6
:1003800066665D20202020202020202020202D2097
:100390006D6F7465732064617461206F6E205553B6
:1003A000420A0D006F7720202020202020202020CE
:1003B000202020202020202020202020202020203D
:1003C0002D206F6E652D776972652073656E736F72
:1003D00072730A0D007265205B6D61736B5D202086
:1003E000202020202020202020202020202020200D
:1003F000202D206D6F7465207265706F727420738C
:10040000657474696E670A0D007269205B696E74A9
:100410005D2020202020202020202020202020209F
:1004200020202020202D207265706F727420696E4C
:1004300074657276616C0A0D007273202020202092
:1004400020202020202020202020202020202020AC
:1004500020202020202D20726164696F2073746138
:1004600074730A0D00737320202020202020202088
:10047000202020202020202020202020202020207C
:10048000202D207374617475732073756D6D6172A6
:10049000790A0D0070777231205B6F6E7C6F666633
:1004A0005D2020202020202020202020202020200F
:1004B0002D2070696E31207077720A0D007265739D
:1004C0007420656570726F6D202020202020202010
:1004D0002020202020202020202D20726573746F82
:1004E000726520656570726F6D0A0D00626F6F74C2
:1004F00020202020202020202020202020202020FC
:1005000020202020202020202D207265626F6F7413
:100510000A0D0075706772202020202020202020E6
:100520002020202020202020202020202020202DBE
:10053000207265626F6F742076696120626F6F74DC
:100540006C6F616465720A0D00557074696D652089
:10055000256420646179732C20253032643A25307B
:1005600032643A253032640A00204E657665722D79
:100570007573656420737461636B203E202564206D
:1005800062797465730A0025352E3266200025379E
:100590002E33662025372E3366002530327800252D
:1005A000730A004E65772064656275673D30782573
:1005B000580A0043757272656E74206465627567CF
:1005C0003D307825580A00445F4F5045523D307801
:1005D00025780A00445F52583D307825780A004457
:1005E0005F54583D307825780A00445F504B543DA5
:1005F000307825780A00445F4F573D307825780AD7
:1006000000445F4C45443D307825780A00445F50F3
:100610004F5745523D307825780A00445F4556458E
:100620004E543D307825780A00445F50305F4C4589
:10063000443D307825780A00445F50315F4C454492
:100640003D307825780A00445F4145533D30782598
:10065000780A00445F5057525F313D307825780A60
:10066000002563002563002563004F4B0A002563C6
:10067000007268206D6973732020202072682073D7
:1006800074616C652020207268206D6973630A00B4
:10069000252D31306C7520252D31306C7520252DA0
:1006A00031306C75200A002563004D43553D2530DF
:1006B000366C780020467573653A2065653D2530B7
:1006C00032782068663D25303278206C663D2530D2
:1006D0003278206C623D2530327800204F534343FE
:1006E000414C3D25642000256300256300256300FF
:1006F0002563004E6577207265706F72743D3078A7
:1007000025580A005573696E67207265706F7274A0
:100710003D307825580A00525F49443D0909307838
:1007200025780A00525F543D0909307825780A007F
:10073000525F545F4D43553D09307825780A005289
:100740005F565F4D43553D09307825780A00525F6A
:1007500050303D0909307825780A00525F50305FEB
:10076000543D0909307825780A00525F50313D091F
:1007700009307825780A00525F555054494D453D5F
:1007800009307825780A00525F52483D09093078CF
:1007900025780A00525F565F494E3D090930782599
:1007A000780A00525F41313D0909307825780A0006
:1007B000525F41323D0909307825780A00525F5472
:1007C000313D0909307825780A002563004E6577A8
:1007D000207265706F727420696E74657276616CD8
:1007E0003D252D64207365630A0043757272656E42
:1007F00074207265706F727420696E7465727661B0
:100800006C3D252D64207365630A00256300256314
:10081000005374617475732053756D6D6172790A3C
:1008200049443D004E65696768626F722074616279
:100830006C652073697A653D25640A0052494D450F
:1008400020616464723D252D642E252D640A0052BA
:100850006164696F205265706F727420496E7465AF
:100860007276616C3D252D640A00526164696F20C7
:100870005265706F7274204D61736B3D3078252D19
:10088000780A00565F494E3D252D352E32660A0006
:10089000565F4D43553D252D352E32660A00555382
:1008A000425F5057523D25730A00546F74616C20AB
:1008B000696E74723A2050303D252D6C64205031A1
:1008C0003D252D6C640A004C6F67206D6F646520B8
:1008D000697320006175746F0A0025730A0048551A
:1008E0004D5F5057525F414C574159533D25730A54
:1008F0000044656275673D3078252D780A00507791
:1009000072312069732025730A0025630025630076
:1009100052483D252D342E31662000545F52483D0B
:10092000252D342E316620002563005854414C5F3C
:100930005452494D3D2564004572726F722030203B
:10094000566F6C74004572726F72203020566F6C57
:1009500074004572726F72203020566F6C740025DF
:10096000352E3266200025372E33662025372E336C
:10097000660025730A0025730A0025730A00257393
:100980000A00256300256300532025642E2564207A
:10099000636C6F636B20256C7520747820256C75F3
:1009A00020727820256C752072747820256C752053
:1009B00072727820256C75207265786D69742025B7
:1009C0006C752061636B747820256C75206E6F6187
:1009D000636B747820256C752061636B72782025B9
:1009E0006C752074696D65646F757420256C752055
:1009F00062616461636B727820256C7520746F6F1F
:100A00006C6F6E6720256C7520746F6F73686F72E2
:100A10007420256C752062616473796E636820258B
:100A20006C752062616463726320256C7520636F4E
:100A30006E74656E74696F6E64726F7020256C756C
:100A40002073656E64696E6764726F7020256C75C3
:100A5000206C6C747820256C75206C6C7278202565
:100A60006C750A00452025642E256420636C6F6335
:100A70006B20256C752063707520256C75206C705B
:100A80006D20256C752069727120256C7520676C4E
:100A9000656420256C7520796C656420256C752053
:100AA000726C656420256C7520747820256C752027
:100AB0006C697374656E20256C752073656E736F39
:100AC000727320256C752073657269616C20256CCA
:100AD000750A000A2A2A2A2A2A2A2A426F6F74696A
:100AE0006E672025732A2A2A2A2A2A2A0A00526196
:100AF0006E646F6D204555493634206164647265BB
:100B000073732067656E6572617465640A004D4198
:100B1000432061646472657373200025783A000A8B
:100B20000025732025732C206368616E6E656C2030
:100B3000257520706F776572202575002C206368FD
:100B400065636B207261746520257520487A000A00
:100B5000004F6E6C696E650A00257325730A006C80
:100B60006F63616C686F73740041544D4547413148
:100B700032387266613100020000FFFE000001455C
:100B80004550524F4D20697320636F7272757074B7
:100B90002C20726577726974696E67207769746852
:100BA0002064656661756C74732E0A006E616E0058
:100BB000696E660000407A10F35A00A0724E180960
:100BC0000010A5D4E80000E87648170000E40B54B4
:100BD000020000CA9A3B000000E1F5050000809683
:100BE0009800000040420F000000A08601000000B5
:100BF000102700000000E80300000000640000006F
:100C000000000A00000000000100000000002C7637
:100C1000D888DC674F0823DFC1DFAE59E1B1B79652
:100C2000E5E3E453C63AE651997696E8E6C28426AF
:100C3000EB898C9B62ED407C6FFCEFBC9C9F40F28B
:100C4000BAA56FA5F490055A2AF75C936B6CF96707
:100C50006DC11BFCE0E40D47FEF520E6B500D0EDCC
:100C6000902E0300943577050080841E0800002034
:100C70004E0A000000C80C333333330F986E1283D2
:100C80001141EF8D2114893BE65516CFFEE6DB18A6
:100C9000D1844B381BF77C1D901DA4BBE42420326B
:100CA00084725E228100C9F124ECA1E53D27494E02
:100CB00046494E4954594E414E000020410000C85B
:100CC0004200401C4620BCBE4CCA1B0E5AAEC59DFD
:100CD00074CDCCCC3D0AD7233C17B7D13877CC2B79
:100CE000329595E6241FB14F0A0011241FBECFEFA5
:100CF000D1E4DEBFCDBF15E0A0E0B2E0ECE6FEEC53
:100D000000E00BBF02C007900D92A63EB107D9F7D5
:100D100018E2A6EEB5E001C01D92A039B107E1F7D7
:100D20000E944C5A0C9434670C940000E091B0126D
:100D3000F0E0EF71F070E350FD4E80838091B012CF
:100D40008F5F8093B0128091CA1F88608093CA1F02
:100D500044E254E0CA0161E10E946E2A80E090E022
:100D600008956F927F928F929F92AF92BF92CF928F
:100D7000DF92EF92FF920F931F93CF93DF934B017C
:100D80008091F0059091F10581FD74980E94C62F25
:100D90005C018AEF95E00E946A2B0AC0CE010296A0
:100DA000B4010E9445280097E9F4CE010E94102C5E
:100DB000EC01009799F7CCC0CE010296B4010E94D5
:100DC0003C28D5018C918150888780E091E0A0E09B
:100DD000B0E089879A87AB87BC878AEF95E0BE0130
:100DE0000E94D92B84E00E94EA309D838C8383E0AB
:100DF0000E94EA303C019F838E83F501C080888584
:100E0000C81ADD24EE24FF24A6E0CC0CDD1CEE1C69
:100E1000FF1CAA95D1F769857A858B859C8520EC86
:100E200030E040E050E00E943460DC01CB01892FCB
:100E30009A2FAB2FBB27C80ED91EEA1EFB1EC986F0
:100E4000DA86EB86FC86D5018C9188878091F00547
:100E50009091F10581FD08C080915A0480FD04C085
:100E600081FF6EC01D9B6CC0EDB7FEB772970FB6C9
:100E7000F894FEBF0FBEEDBF0DB71EB70F5F1F4F3B
:100E800080E092E092838183C5010196D801139698
:100E90009C938E931297F401808114968C931497EF
:100EA00015961C921597818116968C931697179616
:100EB0001C92D5018C91F801808711868C819D81CF
:100EC0009387828775866486BB27AF2D9E2D8D2DD7
:100ED00097878687C701B60124E630E040E050E0FE
:100EE0000E943460672F782F892F99270E947A609B
:100EF000DC01CB01F801918B808B0E940A64209168
:100F000076048DB79EB742960FB6F8949EBF0FBE7B
:100F10008DBF2223A9F000D000D0EDB7FEB73196E7
:100F200085E899E0ADB7BEB712969C938E93119762
:100F3000228313820E941C640F900F900F900F90D9
:100F40008091F0059091F10581FF0BC0749A09C062
:100F50008BE894E00E94F72AEC01009709F02CCF6F
:100F6000EFCFDF91CF911F910F91FF90EF90DF9026
:100F7000CF90BF90AF909F908F907F906F9008958B
:100F800087EE93E08115910511F00197F1F708952F
:100F90000F931F93CF93DF93CEE7DFE10CE312E0D3
:100FA00088819981009739F12DB73EB7285030409C
:100FB0000FB6F8943EBF0FBE2DBFEDB7FEB731960A
:100FC000ADB7BEB712961C930E9311974A815B8101
:100FD0006C817D8142835383648375839783868389
:100FE0000E940A642DB73EB7285F3F4F0FB6F894B2
:100FF0003EBF0FBE2DBF26963FE1CA3BD30781F609
:10100000DF91CF911F910F910895EEE7FFE11182DB
:10101000108236968FE1EA3BF807C9F70895CF931F
:10102000DF93CEE7DFE1E881F981309761F140910C
:10103000E6055091E7056091E8057091E90580911A
:10104000F4059091F505A091F605B091F705841B84
:10105000950BA60BB70B4A815B816C817D81840F58
:10106000951FA61FB71F8A839B83AC83BD83181669
:1010700019061A061B063CF00995198218821A8275
:101080001B821C821D8226968FE1CA3BD80759F627
:101090008091E6059091E705A091E805B091E905FA
:1010A0008093F4059093F505A093F605B093F705AA
:1010B000DF91CF910895CF93DF93EC0188819981DF
:1010C000009729F027E084349207A9F40BC082E04E
:1010D00096E060E870E00E94022D84E497E0998336
:1010E00088830DC082E096E00E942D2D009739F094
:1010F0000E940F08ECCF1982188283E001C081E0C2
:10110000DF91CF910895DC01EEE7FFE180E090E010
:10111000208131812115310591F4FC01EE0FFF1F73
:10112000E80FF91FEE0FFF1FE258F04E4283538382
:1011300064837583B183A08381E090E00895019674
:1011400036968A30910521F780E090E0089587EA8D
:1011500098E040EA50E060E070E00E94830887EA8F
:1011600098E040EA50E060E070E00E948308009759
:10117000B9F18091F0059091F10587FF31C0409160
:10118000E6055091E7056091E8057091E9058DB796
:101190009EB70A970FB6F8949EBF0FBE8DBFEDB7EE
:1011A000FEB731968EE592E0ADB7BEB712969C932E
:1011B0008E931197428353836483758380EA90E012
:1011C000A0E0B0E086839783A087B1870E940A647D
:1011D0008DB79EB70A960FB6F8949EBF0FBE8DBF0F
:1011E0000895882369F06D987598ED9A80916A004A
:1011F000886080936A0080916800816080936800B5
:101200006E987698EE9A80916A00806280936A0068
:101210008091680081608093680008951F920F920A
:101220000FB60F9211248F939F93AF93BF9380912A
:10123000680080FF29C080917A1F90917B1F0196E2
:1012400090937B1F80937A1F8091721B9091731BE8
:10125000A091741BB091751B0196A11DB11D8093C7
:10126000721B9093731BA093741BB093751B80919A
:10127000F0059091F10590FF07C0749882E090E02E
:101280009093840480938304BF91AF919F918F9139
:101290000F900FBE0F901F9018951F920F920FB6D0
:1012A0000F9211248F939F93AF93BF938091680007
:1012B00080FF29C080917C1F90917D1F01969093A3
:1012C0007D1F80937C1F8091761B9091771BA0914E
:1012D000781BB091791B0196A11DB11D8093761BDF
:1012E0009093771BA093781BB093791B8091F005A6
:1012F0009091F10591FF07C0739882E090E0909380
:10130000840480938304BF91AF919F918F910F903C
:101310000FBE0F901F90189580937C0080917B00EA
:10132000877F80937B0080917C00806C80937C0021
:1013300085E080937A0080917A00806880937A00BB
:1013400080917B0087FFFCCF80917B0085FFFCCFE5
:1013500080917A00806480937A0080917A0086FD83
:10136000FCCF109279001092780084E090E060E069
:1013700070E020917A00206420937A0020917A0016
:1013800026FDFCCF2091780030917900620F731F09
:10139000019779F710927C0080917A008F77809383
:1013A0007A00769567957695679580E090E00E9443
:1013B0001F5F462F572F682F792FCB01BA01089551
:1013C00080E00E948C0920917F043091800440913C
:1013D0008104509182040E94D15F21EE3AE744E9F2
:1013E0005EE30E944F5E462F572F682F792FCB0167
:1013F000BA01089580E18093510180935101909149
:10140000510195FF03C08F5F8F31B9F76BE4869F61
:10141000B0011124882777FD8095982F0E94215FC5
:1014200020E030E64FE954E40E944F5E462F572FEC
:10143000682F792FCB01BA0120E030E04AE754E46D
:101440000E94B75E462F572F682F792FCB01BA0124
:10145000089580915E0482FF4DC080917B0088607A
:1014600080937B0089EC80937C0085E080937A00F8
:1014700080917A00806880937A0080917B0087FF5A
:10148000FCCF80917B0085FFFCCF80917A00806447
:1014900080937A0080917A0086FDFCCF80917A005B
:1014A000806480937A0080917A0086FDFCCF609101
:1014B00078007091790080E090E00E941F5F27ED36
:1014C00033EA40E95FE30E94D15F26E636E648E86A
:1014D00053E40E944E5EDC01CB018093A4129093F2
:1014E000A512A093A612B093A71280917A008F77CD
:1014F00080937A000895CF92DF92EF92FF921F932C
:10150000CF93DF93CDB7DEB729970FB6F894DEBF40
:101510000FBECDBF6C011092EA058FEF898359EBA6
:10152000E52E52E1F52E10E03FC0183009F440C01E
:10153000CE010196BE016E5F7F4F0E94AD32898160
:101540008F3F11F08E3F19F48093EA0531C0CE0130
:101550000296C114D10479F40E94C6328093C71F49
:10156000DE011296EFEBFFE188E09D9191938150AF
:10157000E1F711E01DC00E94C632F7018083DE0151
:10158000129620E030E0C70108974D91FC01E20F70
:10159000F31F40832F5F3F4F28303105B1F71F5FA6
:1015A00089E090E0E80EF91E8981882309F0BDCF1B
:1015B000812F29960FB6F894DEBF0FBECDBFDF9105
:1015C000CF911F91FF90EF90DF90CF90089500D0C2
:1015D00080E291E0EDB7FEB7928381830E941C64A4
:1015E0000F900F9008952F923F924F925F926F92BB
:1015F0007F928F929F92AF92BF92CF92DF92EF92A3
:10160000FF920F931F93CF93DF9300D000D0CDB7FD
:10161000DEB78C01009741F489E290E06BE270E064
:101620004AE250E027E00AC08130910549F489E29E
:1016300090E06BE270E04AE250E026E00E948231E6
:10164000C8010E947B0A3BEE832E35E0932E800E6C
:10165000911ED4018C930115110599F019EBA12E5F
:1016600012E1B12E00E010E08BE3682E81E0782ECD
:1016700090E4492E91E0592E28E4222E21E0322ECA
:1016800010C18FEB9FE10E94E933FC01BF01882765
:1016900077FD8095982F0E94215FF82EE92E0FEBA1
:1016A0001FE1AA24BB24B2E2CB2EB1E0DB2ED8018D
:1016B0008D918D0100D000D0EDB7FEB73196ADB75A
:1016C000BEB71296DC92CE921197828313826B83FF
:1016D0007C830E941C640894A11CB11C0F900F9085
:1016E0000F900F906B817C81B8E0AB16B104F9F6D6
:1016F00000D000D000D00DB71EB70F5F1F4F87E29C
:1017000091E0EDB7FEB7928381839701862F972FE3
:10171000A32FBE2DBC01CD0120E030E048EC52E407
:101720000E94B75EDC01CB01F80182839383A4831E
:10173000B5830E941C642DB73EB72A5F3F4F0FB69A
:10174000F8943EBF0FBE2DBF8091C71F882319F0AC
:1017500081E892E002C08AE892E000D000D027E35E
:1017600031E0ADB7BEB712963C932E931197149605
:101770009C938E9313970E941C640F900F900F9070
:101780000F900E94E70A94C0C80163E0880F991F78
:101790006A95E1F7800F911F8F549D4E0E94E933A7
:1017A000FC01BF01882777FD8095982F0E94215F5B
:1017B0006C0120E030E0A8EFEA2EAFEFFA2EEA0C41
:1017C000FB1C00D000D0ADB7BEB71196EDB7FEB789
:1017D00072826182F701E20FF31F808112968C936F
:1017E000129713961C9229833A836B837C830E9401
:1017F0001C6429813A812F5F3F4F0F900F900F900B
:101800000F906B817C8128303105D9F600D000D053
:1018100000D0EDB6FEB60894E11CF11CADB7BEB722
:1018200012965C924E921197862F972FAC2DBD2D5C
:10183000BC01CD0120E030E048EC52E40E94B75EEC
:10184000DC01CB01F70182839383A483B5830E94DB
:101850001C642DB73EB72A5F3F4F0FB6F8943EBFCA
:101860000FBE2DBFD5018C91882319F081E892E03D
:1018700002C08AE892E000D000D0EDB7FEB7328215
:101880002182948383830E941C640F900F900F9099
:101890000F900E94E70A0F5F1F4F29E030E0A20E71
:1018A000B31ED4018C9190E0081719070CF46CCF8B
:1018B0000F900F900F900F90DF91CF911F910F918C
:1018C000FF90EF90DF90CF90BF90AF909F908F9060
:1018D0007F906F905F904F903F902F900895CF939F
:1018E000DF9300D0CDB7DEB78091C01F8983809190
:1018F000C61F8A83CE0101960E9457280F900F9031
:10190000DF91CF910895CF93DF93EC018091BF1FBA
:101910008F3FB1F58091C01F8F3F91F58091C11F1E
:101920008F3F71F58091C21F8F3F51F58091C31F8A
:101930008F3F31F58091C41F8F3F11F58091C51FF6
:101940008F3FF1F48091C61F8F3FD1F489E290E080
:101950006BE270E04AE250E027E00E94823180E0D2
:1019600090E00E947B0AC551DA4F88838FEB9FE19C
:1019700060E070E049E050E00E9462650E946F0CF8
:10198000DF91CF9108951F920F920FB60F920BB671
:101990000F9211242F933F934F935F936F937F93F5
:1019A0008F939F93AF93BF93EF93FF938091CA1F41
:1019B00082608093CA1F80918304909184041816DA
:1019C000190614F4749A739A8091F0059091F105B8
:1019D00085FF02C0749873988091E6059091E705A1
:1019E000A091E805B091E9050196A11DB11D809374
:1019F000E6059093E705A093E805B093E90580918B
:101A000085049091860401979093860480938504C1
:101A1000009709F064C08091F8059091F9059C0148
:101A20002F5F3F4F3093F9052093F8054091211B1C
:101A30005091221B6091231B7091241B4F5F5F4FBD
:101A40006F4F7F4F4093211B5093221B6093231BAA
:101A50007093241B20E130E03093860420938504AA
:101A600020915A0420FD02C01D9B05C01092EE0576
:101A70001092ED0506C021E030E03093EE05209392
:101A8000ED0520915C0430915D0421153105A1F034
:101A90000296B9010E945360009771F47798809183
:101AA000F0059091F10593FF07C0749884E090E0F1
:101AB00090938404809383042115310581F08091F3
:101AC000F8059091F905B9010E945360009739F427
:101AD0008CE094E062E140E050E00E946E2AFF91C9
:101AE000EF91BF91AF919F918F917F916F915F9196
:101AF0004F913F912F910F900BBE0F900FBE0F9003
:101B00001F9018958091B0129091311B891B0895F8
:101B10000E94820D882379F0E091311BF0E0EF7193
:101B2000F070E350FD4E808190E02091311B2F5FDB
:101B30002093311B08958FEF9FEF0895CF93DF938C
:101B4000EC011092F3051092F205888199810097BB
:101B500031F022E0843D920709F0B7C009C00E942D
:101B6000820D882341F484ED92E099838883B1C08B
:101B7000613109F0AEC0F89478940E94880D90E02D
:101B800090930B0680930A068D3009F47CC08F3F3A
:101B900031F38231910569F18F37910521F0883059
:101BA000910509F053C080910C0690910D0618160E
:101BB00019060CF060C060918A2870918B2888E02B
:101BC00090E00E94DE6360918A2870918B2880E209
:101BD00090E00E94DE6360918A2870918B2888E0F3
:101BE00090E00E94DE6380910C0690910D060197B3
:101BF0003EC060918A2870918B288DE090E00E9411
:101C0000DE6310920F0610920E0614C08E5C944E86
:101C1000FC01808160918A2870918B2890E00E945D
:101C2000DE6380910E0690910F06019690930F0649
:101C300080930E0680910E0690910F0620910C065F
:101C400030910D06821793070CF315C060918A2816
:101C500070918B280E94DE6380910C0690910D0696
:101C600020910A06FC01EE5CF44E208301969093CD
:101C70000D0680930C0680910C0690910D068F3313
:101C8000910509F06CCF1092311B1092B012809127
:101C90000C0690910D06FC01EE5CF44E10829093C0
:101CA000F3058093F20510920D0610920C068091B8
:101CB000C81F9091C91F009709F451CF6091000689
:101CC00040E050E00E946E2A4ACF1982188283E0D9
:101CD00001C081E0DF91CF91089578948091ED0566
:101CE0009091EE05009719F483B7817F03C083B705
:101CF000817F866083BFF89483B7816083BF7894C7
:101D0000889583B78E7F83BF78940895CF93DF93B0
:101D1000EC0188819981009721F027E081359207B5
:101D200089F40E946D0E80919E0990919F0965E84B
:101D300040E050E00E946E2A81E597E09983888315
:101D400081E003C01982188283E0DF91CF9108956A
:101D5000FF920F931F93CF93DF93729A80915A044F
:101D600083FD06C0C0E5D0E00E94C0072197E1F7DF
:101D70008EE40E946834882309F08BC0C0E5D0E06F
:101D80000E94C0072197E1F78FE40E9468340E9407
:101D9000D034C82F82958695869583708130A9F4BA
:101DA0004091291B50912A1B60912B1B70912C1B79
:101DB0004F5F5F4F6F4F7F4F4093291B50932A1BFC
:101DC00060932B1B70932C1B16C08230A0F04091A7
:101DD0002D1B50912E1B60912F1B7091301B4F5F5C
:101DE0005F4F6F4F7F4F40932D1B50932E1B60937F
:101DF0002F1B7093301B0E94D0341C2F1F7300E0E8
:101E0000080F111D0E94D034F82E0E94DA34DF2D05
:101E100090E0C92FC80FD11DD695C795D695C79507
:101E20000E94B73480915A0483FF7298B80180E011
:101E300090E00E941F5F20E134E048EC5BE30E94E9
:101E4000D15FDC01CB0180931D1390931E13A093EF
:101E50001F13B0932013BE0180E090E00E941F5F2B
:101E600024EA3CEF44E25CE30E94D15F20E030E0F2
:101E700040E252E40E944E5EDC01CB018093CB1F16
:101E80009093CC1FA093CD1FB093CE1F80E090E025
:101E900015C08091251B9091261BA091271BB09106
:101EA000281B0196A11DB11D8093251B9093261B15
:101EB000A093271BB093281B81E090E0DF91CF9186
:101EC0001F910F91FF9008950E94290A80915E044E
:101ED00090915F0490FF02C00E94A80E80915E0462
:101EE00090915F0491FF0CC00E94E009DC01CB01DE
:101EF0008093BA1F9093BB1FA093BC1FB093BD1FCC
:101F000008954F925F926F927F928F929F92AF92BD
:101F1000BF92CF92DF92EF92FF920F931F93CF93D6
:101F2000DF93CDB7DEB7C656D0400FB6F894DEBF0C
:101F30000FBECDBF2C01633851F480E196E0A79627
:101F40006FAFA7970E94A828A7966FADA797D20159
:101F50008D919C911197009731F0B6E085399B07E0
:101F600009F0C3C40EC080E196E061E870E047E884
:101F700054E00E948D2885E996E0F20191838083E8
:101F8000BAC4623109F0B7C40E94640F80915E0444
:101F900080FF60C000D000D000D0EDB7FEB7319612
:101FA000A2E0CA2ED12CCC0EDD1EADB7BEB7129664
:101FB000DC92CE92119784E690E0938382838BE843
:101FC00092E0958384830E9471648C018FEBA82E2C
:101FD0008FE1B82EEDB7FEB736960FB6F894FEBF78
:101FE0000FBEEDBFEE24FF2494E6892E912C2FE83E
:101FF000622E22E0722ED5012D915D01EDB7FEB764
:1020000038970FB6F894FEBF0FBEEDBF3196C601EC
:10201000800F911FADB7BEB712969C938E93119708
:102020009382828275826482268317820E94716401
:10203000080F191F0894E11CF11CEDB7FEB7389684
:102040000FB6F894FEBF0FBEEDBFF8E0EF16F10437
:1020500091F602C000E010E080915E0490915F0470
:10206000009781F12DB73EB7285030400FB6F89455
:102070003EBF0FBE2DBFEDB7FEB73196CE01029623
:10208000800F911FADB7BEB712969C938E93119798
:1020900084E690E09383828384E992E0958384834D
:1020A0008091ED059091EE05978386830E9471647F
:1020B000080F191FEDB7FEB738960FB6F894FEBF9C
:1020C0000FBEEDBF80915E0481FF51C089E290E0B8
:1020D0006BE270E04AE250E027E00E9482318FEB31
:1020E0009FE10E94E9332DB73EB72A5030400FB62A
:1020F000F8943EBF0FBE2DBFEDB6FEB60894E11CAE
:10210000F11C9E012E5F3F4F200F311FADB7BEB7B0
:1021100012963C932E93119724E630E0F701338317
:1021200022832BE932E0358324839C01B90188277F
:1021300077FD8095982F0E94215F20E030E048ECE9
:1021400052E40E94B75EDC01CB01F70186839783DE
:10215000A087B1870E947164080F191F2DB73EB781
:10216000265F3F4F0FB6F8943EBF0FBE2DBF809144
:102170005E0490915F0494FF54C089E290E06BE2AA
:1021800070E04AE250E026E00E94823181E090E077
:102190000E947B0A8093EC0581EB92E10E94E93377
:1021A000ADB7BEB71A970FB6F894BEBF0FBEADBF9E
:1021B000EDB6FEB60894E11CF11C9E012E5F3F4F68
:1021C000200F311F12963C932E93119724E630E096
:1021D000F7013383228325EA32E0358324839C018F
:1021E000B901882777FD8095982F0E94215F20E014
:1021F00030E048EC52E40E94B75EDC01CB01F7010D
:1022000086839783A087B1870E947164080F191F86
:102210002DB73EB7265F3F4F0FB6F8943EBF0FBEB7
:102220002DBF80915E0482FF35C08DB79EB70A979F
:102230000FB6F8949EBF0FBE8DBFEDB7FEB73196B7
:10224000CE010296800F911FADB7BEB712969C9338
:102250008E93119784E690E09383828380EB92E0E3
:10226000958384838091A4129091A512A091A612C7
:10227000B091A71286839783A087B1870E9471646B
:10228000080F191FEDB7FEB73A960FB6F894FEBFC8
:102290000FBEEDBF80915E0483FF32C00E94FA0939
:1022A000AB01BC012DB73EB72A5030400FB6F894B1
:1022B0003EBF0FBE2DBFEDB7FEB73196CE010296E1
:1022C000800F911FADB7BEB712969C938E93119756
:1022D00084E690E0938382838EEB92E095838483FF
:1022E00046835783608771870E947164080F191FA6
:1022F000EDB7FEB73A960FB6F894FEBF0FBEEDBF2E
:1023000080915E0484FF36C04091721B5091731B14
:102310006091741B7091751B2DB73EB72A503040E9
:102320000FB6F8943EBF0FBE2DBFEDB7FEB7319686
:10233000CE010296800F911FADB7BEB712969C9347
:102340008E93119784E690E0938382838CEC92E0E5
:102350009583848346835783608771870E94716465
:10236000080F191FEDB7FEB73A960FB6F894FEBFE7
:102370000FBEEDBFA0905C04B0905D0480915E0440
:1023800090915F048A219B2185FF6AC04091721B56
:102390005091731B6091741B7091751BC090A812B3
:1023A000D090A912E090AA12F090AB122DB73EB7D0
:1023B0002A5030400FB6F8943EBF0FBE2DBF8DB6E9
:1023C0009EB60894811C911CCE010296800F911F2D
:1023D000ADB7BEB712969C938E93119784E690E0AA
:1023E000F4019383828385ED92E0958384834C1975
:1023F0005D096E097F09CB01BA010E941F5F6B0165
:102400007C01B50180E090E00E941F5F9B01AC0160
:10241000C701B6010E94B75EDC01CB01F4018683DF
:102420009783A087B1870E947164080F191F80915C
:10243000721B9091731BA091741BB091751B8093BC
:10244000A8129093A912A093AA12B093AB122DB721
:102450003EB7265F3F4F0FB6F8943EBF0FBE2DBF6D
:1024600080915E0486FF35C04091761B5091771BAA
:102470006091781B7091791B8DB79EB70A970FB644
:10248000F8949EBF0FBE8DBFEDB7FEB73196CE015B
:102490000296800F911FADB7BEB712969C938E9394
:1024A000119784E690E09383828382EE92E0958395
:1024B000848346835783608771870E947164080F05
:1024C000191FEDB7FEB73A960FB6F894FEBF0FBED0
:1024D000EDBF80915E0487FF36C04091211B509173
:1024E000221B6091231B7091241B2DB73EB72A50ED
:1024F00030400FB6F8943EBF0FBE2DBFEDB7FEB70C
:102500003196CE010296800F911FADB7BEB71296DD
:102510009C938E93119784E690E0938382838BEE55
:1025200092E09583848346835783608771870E94F6
:102530007164080F191FEDB7FEB73A960FB6F894FD
:10254000FEBF0FBEEDBF80915E0490915F0490FFCF
:1025500036C02DB73EB72A5030400FB6F8943EBF74
:102560000FBE2DBFEDB7FEB73196CE010296800F9C
:10257000911FADB7BEB712969C938E93119784E6C8
:1025800090E09383828384EF92E0958384838091AB
:102590001D1390911E13A0911F13B09120138683D9
:1025A0009783A087B1870E947164080F191FEDB748
:1025B000FEB73A960FB6F894FEBF0FBEEDBF8091FE
:1025C0005E0490915F0491FF36C02DB73EB72A504C
:1025D00030400FB6F8943EBF0FBE2DBFEDB7FEB72B
:1025E0003196CE010296800F911FADB7BEB71296FD
:1025F0009C938E93119784E690E0938382838FEF70
:1026000092E0958384838091BA1F9091BB1FA09123
:10261000BC1FB091BD1F86839783A087B1870E949E
:102620007164080F191FEDB7FEB73A960FB6F8940C
:10263000FEBF0FBEEDBF80915E0490915F0492FFDC
:1026400046C081E00E948C09AB01BC012DB73EB7AA
:102650002A5030400FB6F8943EBF0FBE2DBFEDB6E6
:10266000FEB60894E11CF11CCE010296800F911F6A
:10267000ADB7BEB712969C938E93119784E690E007
:10268000F701938382838CE093E095838483CB016D
:10269000BA0120917B0430917C0440917D045091DB
:1026A0007E040E94D15FDC01CB01F7018683978312
:1026B000A087B1870E947164080F191F2DB73EB71C
:1026C000265F3F4F0FB6F8943EBF0FBE2DBF8091DF
:1026D0005E0490915F0493FF45C082E00E948C09E4
:1026E000AB01BC018DB79EB70A970FB6F8949EBF99
:1026F0000FBE8DBFEDB6FEB60894E11CF11CCE01F5
:102700000296800F911FADB7BEB712969C938E9321
:10271000119784E690E0F7019383828389E193E047
:1027200095838483CB01BA0120917704309178049A
:102730004091790450917A040E94D15FDC01CB0171
:10274000F70186839783A087B1870E947164080F81
:10275000191F2DB73EB7265F3F4F0FB6F8943EBF07
:102760000FBE2DBF779A8091F0059091F10593FDF2
:10277000749A8091F0059091F10582FD08C08091D6
:102780005A0480FD04C081FF31C01D9B2FC000D0C2
:1027900000D086E293E0ADB7BEB712969C938E93BD
:1027A0001197CE01029614969C938E9313970E94D4
:1027B0000A64209176040F900F900F900F902223BF
:1027C000A9F000D000D0EDB7FEB7319682E899E0CD
:1027D000ADB7BEB712969C938E9311972283138246
:1027E0000E941C640F900F900F900F9080911B0619
:1027F0008983FE01E00FF11F128272E0C72ED12CF7
:10280000C00ED11ECE010196B6010E948E3080917D
:102810005A0482FF49C080E694E0BE016F5F7F4F9B
:10282000A6012AE73BE10E94E4348091F0059091F3
:10283000F10592FF39C05AE7E52E5BE1F52E00E085
:1028400010E06DE2A62E63E0B62EF70181917F01C4
:1028500000D000D0EDB7FEB73196ADB7BEB7129637
:10286000BC92AE921197828313820E940A640F5F1A
:102870001F4F0F900F900F900F900031110529F707
:102880008AE090E00E943C6400D000D082E393E0B4
:10289000EDB7FEB792838183D482C3820E940A641B
:1028A0000F900F900F900F908091F0059091F1058F
:1028B00082FD73980E94AA3A80E196E00E94AB28BC
:1028C0008091ED059091EE05009711F00E949B3BE1
:1028D00080911B068F5F80931B068091F00590917D
:1028E000F10582FF48CB739A46CBD20111961C9218
:1028F0001E9283E001C081E0CA59DF4F0FB6F89401
:10290000DEBF0FBECDBFDF91CF911F910F91FF9022
:10291000EF90DF90CF90BF90AF909F908F907F907F
:102920006F905F904F9008957298729A8EE40E9413
:10293000683480EA0E94BF3480E00E94BF3480E0A7
:102940000E94BF348FE40E9468340E94D034829584
:102950008695869583708130A9F44091291B50910A
:102960002A1B60912B1B70912C1B4F5F5F4F6F4F89
:102970007F4F4093291B50932A1B60932B1B70930E
:102980002C1B16C08230A0F040912D1B50912E1BA5
:1029900060912F1B7091301B4F5F5F4F6F4F7F4FC8
:1029A00040932D1B50932E1B60932F1B7093301B55
:1029B00000D000D0EDB7FEB731962AE333E0ADB7D3
:1029C000BEB712963C932E931197828313820E9476
:1029D0000A640F900F900F900F908EE40E9468345D
:1029E00080E80E94BF3480E00E94BF3480E00E94F3
:1029F000BF340E94B73480E090E0089500D08CE4AA
:102A000091E0ADB7BEB712969C938E9311970E943A
:102A10001C64209176040F900F902223A9F000D01F
:102A200000D0EDB7FEB7319689E591E0ADB7BEB7FE
:102A300012969C938E931197228313820E941C649A
:102A40000F900F900F900F90089500D08CE591E0BB
:102A5000EDB7FEB7928381830E941C6481E891E008
:102A6000EDB7FEB7928381830E941C6489EA91E0EE
:102A7000EDB7FEB7928381830E941C6480ED91E0E4
:102A8000EDB7FEB7928381830E941C648AEF91E0C8
:102A9000EDB7FEB7928381830E941C6485E392E0C8
:102AA000EDB7FEB7928381830E941C648FE592E0AC
:102AB000EDB7FEB7928381830E941C6485E892E0A3
:102AC000EDB7FEB7928381830E941C6485EB92E090
:102AD000EDB7FEB7928381830E941C648EEE92E074
:102AE000EDB7FEB7928381830E941C648AE193E074
:102AF000EDB7FEB7928381830E941C6483E493E068
:102B0000EDB7FEB7928381830E941C6482E793E055
:102B1000EDB7FEB7928381830E941C6484EA93E040
:102B2000EDB7FEB7928381830E941C6485ED93E02C
:102B3000EDB7FEB7928381830E941C6489E094E024
:102B4000EDB7FEB7928381830E941C6489E394E011
:102B5000EDB7FEB7928381830E941C6485E694E002
:102B6000EDB7FEB7928381830E941C6484E994E0F0
:102B7000EDB7FEB7928381830E941C648DEB94E0D5
:102B8000EDB7FEB7928381830E941C648CEE94E0C3
:102B9000EDB7FEB7928381830E941C6483E195E0C8
:102BA000EDB7FEB7928381830E941C640F900F9053
:102BB00008958AE493E00E94436408954F925F92DF
:102BC0006F927F928F929F92AF92BF92CF92DF923D
:102BD000EF92FF920F931F93CF93DF9300D000D01B
:102BE000CDB7DEB76091211B7091221B8091231B12
:102BF0009091241B8090211B9090221BA090231B5E
:102C0000B090241B4090211B5090221B6090231BEE
:102C10007090241B2091211B3091221B4091231B7B
:102C20005091241B29833A834B835C834DB75EB755
:102C30004A5050400FB6F8945EBF0FBE4DBF0DB75F
:102C40001EB70F5F1F4F29E435E0EDB7FEB73283A3
:102C50002183A0E8CA2EA1E5DA2EA1E0EA2EF12C0C
:102C6000A70196010E947A60F80133832283C5018F
:102C7000B401A70196010E947A60B0E1CB2EBEE0BC
:102C8000DB2EE12CF12CA70196010E947A603327FC
:102C900027FD3095F80135832483C301B201A701D4
:102CA00096010E947A602CE3C22ED12CE12CF12CEB
:102CB000A70196010E947A60332727FD3095F8011D
:102CC0003783268369817A818B819C81A701960154
:102CD0000E947A60772767FD7095F8017187608799
:102CE0000E941C642DB73EB7265F3F4F0FB6F89485
:102CF0003EBF0FBE2DBF0F900F900F900F90DF9132
:102D0000CF911F910F91FF90EF90DF90CF90BF90E8
:102D1000AF909F908F907F906F905F904F900895AD
:102D2000E0E9F8E28081918122E482349207B9F0EF
:102D300000D000D089E695E0ADB7BEB712969C935F
:102D40008E931197E059F8421496FC93EE931397E3
:102D50000E941C640F900F900F900F9008953A9668
:102D6000B1E4E53FFB07F0F20895EF92FF920F9375
:102D70001F93CF93DF930E94E009DC01CB0100D0C9
:102D800000D000D027E835E0EDB7FEB732832183CD
:102D900083839483A583B6830E941C648DB79EB7FA
:102DA00006960FB6F8949EBF0FBE8DBF81E00E94BD
:102DB0008C0920917B0430917C0440917D045091DA
:102DC0007E040E94D15F8B01D82FC92F82E00E9420
:102DD0008C09AB01BC01EDB7FEB73A970FB6F8947A
:102DE000FEBF0FBEEDBFEDB6FEB60894E11CF11CB0
:102DF0002EE835E0328321839E01802F912FA32F6F
:102E0000B22FF70182839383A483B583CB01BA01E8
:102E100020917704309178044091790450917A049C
:102E20000E94D15FDC01CB01F70186839783A087E5
:102E3000B1870E941C648DB79EB70A960FB6F894AE
:102E40009EBF0FBE8DBF0E94E70ADF91CF911F91F9
:102E50000F91FF90EF900895EF92FF920F931F93C1
:102E6000CF93DF93882389F08FEB9FE16FEF70E0C2
:102E700049E050E00E9494638FEB9FE160E070E0D6
:102E800049E050E00E94626522C00FEB1FE1C0E004
:102E9000D0E03AE9E32E35E0F32ED8018D918D0193
:102EA00000D000D0EDB7FEB73196ADB7BEB71296E1
:102EB000FC92EE921197828313820E941C642196E9
:102EC0000F900F900F900F90C830D10531F70E94EE
:102ED000E70ADF91CF911F910F91FF90EF90089536
:102EE000CF92DF92EF92FF9260917404709175041B
:102EF00080E090E00E9486636BE673E00E949B6333
:102F0000009709F077C08FE892E090935F04809378
:102F10005E048EE594E06DE070E042E050E00E94D7
:102F200062658CE390E090935D0480935C048CE593
:102F300094E06BE070E042E050E00E94626582E065
:102F400090E090935B0480935A048AE594E069E0F2
:102F500070E042E050E00E9462651092F10510922C
:102F6000F00580EF95E06BE170E042E050E00E94F8
:102F700062650F2EF2E2CF2EFFEFDF2EFCECEF2E7C
:102F8000FBE3FF2EF02DC0927B04D0927C04E092F4
:102F90007D04F0927E048BE794E063E170E044E00E
:102FA00050E00E946265C0927704D0927804E0926B
:102FB0007904F0927A0487E794E06FE070E044E0EF
:102FC00050E00E9462658DEE97E4AAE8BCE380932E
:102FD0007F0490938004A0938104B09382048FE7D0
:102FE00094E067E170E044E050E00E94626581E0B7
:102FF0000E942C17FF90EF90DF90CF9008952F92B2
:103000003F924F925F926F927F928F929F92AF9278
:10301000BF92CF92DF92EF92FF920F931F93CF93C5
:10302000DF9300D0CDB7DEB79A838983DC018D9121
:103030009C911197009711F00C94422660917404B2
:103040007091750482E39BE10E94866382E39BE1B9
:1030500060E470E00E94A463009759F460918A28AC
:1030600070918B288AE090E00E94DE6381E00C94EE
:1030700048268130910549F42090321B33244424A2
:103080005524662477244301BEC18230910599F40A
:103090003091321B2091331B932F80E0820F911DC2
:1030A0001C01892F880F880B482E582E682E782EE9
:1030B000882E982EA8C18330910509F09CC02091DC
:1030C000321B8090331BB090341B30E040E050E066
:1030D00060E070E080E090E000E10E948F59922E65
:1030E000A32E142FF52EE62EC72E282ED92E282DEE
:1030F00030E040E050E060E070E080E090E008E028
:103100000E948F59290DB1E0291508F0B0E03A0D61
:10311000E1E03A1508F0E0E0B30FF1E0B31708F092
:10312000F0E0EF2B410F31E0411708F030E0E40F01
:10313000F1E0E41708F0F0E03F2B5F0D41E05F1590
:1031400008F040E0A32FA50F31E0A51708F030E00C
:10315000432B6E0D31E06E1508F030E0F42FF60FC2
:1031600041E0F61708F040E0342B7C0D41E07C157F
:1031700008F040E0532F570F31E0571708F030E0C8
:10318000432B820D31E0821508F030E0480F61E0FA
:10319000481708F060E0362BD90ED30EB20E81E04E
:1031A000B21608F080E0182F1B0F71E01B1708F013
:1031B00070E07E0F61E07E1708F060E06A0F31E09A
:1031C0006A1708F030E03F0F21E03F1708F020E0D9
:1031D000250F91E0251708F090E0940F81E09417F7
:1031E00008F080E02B2C312E472E562E632E722EA7
:1031F000892E982EFDC08430910509F0FBC02091E6
:10320000321B8090331BA090341BB090351B30E0F4
:1032100040E050E060E070E080E090E008E10E9473
:103220008F59722E932E142FF52EE62EC72E282E90
:10323000D92E282D30E040E050E060E070E080E0E2
:1032400090E000E10E948F59270DF1E0271508F06A
:10325000F0E0390DE1E0391508F0E0E0F30FA1E00E
:10326000F31708F0A0E0EA2B410F31E0411708F016
:1032700030E0E40FA1E0E41708F0A0E03A2B5F0D86
:1032800041E05F1508F040E0B32FB50F31E0B5170E
:1032900008F030E0432B6E0D31E06E1508F030E0A1
:1032A000A42FA60F41E0A61708F040E0342B7C0DB8
:1032B00041E07C1508F040E0532F570F31E05717DD
:1032C00008F030E0432B820D31E0821508F030E049
:1032D000480F61E0481708F060E0362BD90ED30E96
:1032E000222E2B0C81E0221608F080E0B82EBF0EB3
:1032F00081E0BF1608F080E0982E9E0E81E09E16B9
:1033000008F080E0C82ECB0E11E0CB1608F010E0DC
:103310001A0F81E01A1708F080E0F82EF50E81E010
:10332000F51608F080E0E82EE40E81E0E41608F0DF
:1033300080E0D80E2A2D30E040E050E060E070E000
:1033400080E090E008E00E948F59220DE1E0221514
:1033500008F0E0E03B0DF1E03B1508F0F0E0E30F92
:10336000A1E0E31708F0A0E0FA2B490D31E0491580
:1033700008F030E0F40FA1E0F41708F0A0E03A2BD9
:103380005C0D41E05C1508F040E0A32FA50F31E093
:10339000A51708F030E0432B610F31E0611708F00A
:1033A00030E0542F560F41E0561708F040E0342B20
:1033B0007F0D41E07F1508F040E0632F670F31E09B
:1033C000671708F030E0432B8E0D31E08E1508F0C2
:1033D00030E0480F71E0481708F070E0372BD90E45
:1033E000222E3E2E4F2E5A2E652E762E842E932E72
:1033F0009D0C09C08AE0282E3324442455246624D9
:103400007724882499240E94E70AB2E62B1689F4CF
:10341000E5E63E1671F4F4E64F1659F4552049F4EA
:10342000662039F4772029F4882019F4992009F4CA
:103430000CC59101A201B301C401B2E6AB2E15E6A1
:10344000B12E04E6C02EDD24EE24FF2400E010E0BF
:103450000E94095A823008F099C187E7281681F442
:103460009FE6391669F4442059F4552049F4662042
:1034700039F4772029F4882019F4992009F4C6C773
:103480009101A201B301C401F7E7AF2EAFE6BA2E56
:10349000CC24DD24EE24FF2400E010E00E94095A31
:1034A000823008F0B6C0A4E62A1689F4B1E63B16CD
:1034B00071F4442061F4552051F4662041F47720E2
:1034C00031F4882021F4992011F40C94A72591015E
:1034D000A201B301C40104E6A02EE1E6BE2ECC2475
:1034E000DD24EE24FF2400E010E00E94095A82301F
:1034F00008F046C0E5E72E1679F4332069F444203D
:1035000059F4552049F4662039F4772029F48820AD
:1035100019F4992009F4B9C5F6E72F1679F4332088
:1035200069F4442059F4552049F4662039F4772091
:1035300029F4882019F4992009F4B6C588E62816DC
:1035400011F00C944026332011F00C9440264420B6
:1035500011F00C944026552011F00C944026662062
:1035600011F00C944026772011F00C94402688200E
:1035700011F00C944026992011F00C94402662C55D
:1035800094E6291681F4A9E63A1669F4442059F420
:10359000552049F4662039F4772029F4882019F45D
:1035A000992009F452C5B5E62B1681F4EEE63E16D5
:1035B00069F4442059F4552049F4662039F4772001
:1035C00029F4882019F4992009F47AC7F5E62F1612
:1035D00011F00C94402684E6381611F00C94402625
:1035E000442011F00C944026552011F00C944026F4
:1035F000662011F00C944026772011F00C944026A0
:10360000882011F00C944026992011F00C9440264B
:103610001CC493E7291689F4A2E73A1671F44420F2
:1036200061F4552051F4662041F4772031F488206C
:1036300021F4992011F40C9433249101A201B301D7
:10364000C401B3E7AB2E12E7B12ECC24DD24EE2467
:10365000FF2400E010E00E94095A823008F04AC0BE
:10366000B5E62B1679F43B1469F4442059F455203F
:1036700049F4662039F4772029F4882019F4992038
:1036800009F487C7E9E62E1689F4F2E73F1671F4CC
:10369000442061F4552051F4662041F4772031F440
:1036A000882021F4992011F40C94DA2383E328165E
:1036B00011F00C94402691E7391611F00C94402635
:1036C000442011F00C944026552011F00C94402613
:1036D000662011F00C944026772011F00C944026BF
:1036E000882011F00C944026992011F00C9440266B
:1036F0000C94A725A3E62A1691F4B4E63B1679F4B8
:10370000E1E64E1661F4552051F4662041F477202D
:1037100031F4882021F4992011F40C94A725F3E7C3
:103720002F1689F485E6381671F491E6491659F496
:10373000552049F4662039F4772029F4882019F4BB
:10374000992009F4C0C4A3E72A1611F00C9440266E
:103750003A1611F00C944026442011F00C944026A7
:10376000552011F00C944026662011F00C94402650
:10377000772011F00C944026882011F00C944026FC
:10378000992011F00C9440260C944224B4E72B1697
:1037900089F4EFE63E1671F44E1661F4F2E65F1618
:1037A00049F4662039F4772029F4882019F4992007
:1037B00009F4C5C49101A201B301C40104E7A02E1C
:1037C000EFE6BE2EFFE6CF2EA2E6DA2EEE24FF2491
:1037D00000E010E00E94095A823008F0A8C085E796
:1037E000281689F493E6391671F4ADE64A1659F4B1
:1037F000552049F4662039F4772029F4882019F4FB
:10380000992009F484C59101A201B301C401A5E77F
:10381000AA2EB3E6BB2E1DE6C12EDD24EE24FF2426
:1038200000E010E00E94095A8230B0F52C1489F4AF
:103830003A1479F4B8E64B1661F4552051F4662039
:1038400041F4772031F4882021F4992011F40C946C
:10385000B625E7E62E1689F4FFE63F1671F48CE6EE
:10386000481659F4552049F4662039F4772029F494
:10387000882019F4992009F496C492E7291611F0CA
:103880000C944026391611F00C944026A5E64A16F1
:1038900011F00C94402636C0B1E32B1681F43B1690
:1038A00071F4E1E74E1659F4552049F4662039F4D5
:1038B000772029F4882019F4992009F428C5F0E725
:1038C0002F1689F485E6381671F492E7491659F4F3
:1038D000552049F4662039F4772029F4882019F41A
:1038E000992009F456C6A0E32A1611F00C9440263C
:1038F000B1E33B1611F00C944026E1E74E1611F0AF
:103900000C944026552011F00C944026662011F0AE
:103910000C944026772011F00C944026882011F05A
:103920000C944026992011F00C94402699C4F0E79D
:103930002F1691F48DE6381679F495E7491661F45F
:10394000A8E65A1649F4662039F4772029F488202D
:1039500019F4992009F480C59101A201B301C401B1
:1039600010E7A12E0DE6B02EE5E7CE2EF8E6DF2E0D
:10397000EE24FF2400E010E00E94095A823008F093
:103980004DC02A1489F4BCE63B1671F4E5E64E16E8
:1039900059F45D1449F4662039F4772029F488201D
:1039A00019F4992009F44EC3F1E62F1691F48DE62F
:1039B000381679F495E7491661F4A8E65A1649F4E1
:1039C000662039F4772029F4882019F4992009F425
:1039D00032C5B9E62B1611F00C944026ECE63E16E3
:1039E00011F00C944026F1E64F1611F00C9440268D
:1039F00083E6581611F00C944026662011F00C94C2
:103A00004026772011F00C944026882011F00C9469
:103A10004026992011F00C944026B0C094E7291656
:103A200091F4A3E73A1679F4B5E64B1661F4E2E7B0
:103A30005E1649F4662039F4772029F4882019F4B9
:103A4000992009F4A3C59101A201B301C401E4E7DF
:103A5000AE2EF3E7BF2EA5E6CA2EB2E7DB2EEE248C
:103A6000FF2400E010E00E94095A823020F5F1E3C3
:103A70002F1611F00C9440263D1411F00C944026A2
:103A800087E7481611F00C94402690E7591611F07C
:103A90000C944026662011F00C944026772011F0FB
:103AA0000C944026882011F00C944026992011F0A7
:103AB0000C9440263BC0A2E72A1691F4B7E63B16C9
:103AC00079F4E0E74E1661F4F5E75F1649F46620F5
:103AD00039F4772029F4882019F4992009F432C3A5
:103AE0008CE6281611F00C94402691E6391611F058
:103AF0000C944026A4E74A1611F00C944026B8E72F
:103B00005B1611F00C944026662011F00C944026B0
:103B1000772011F00C944026882011F00C94402658
:103B2000992011F00C9440260C94062660917404A0
:103B30007091750480E090E00E9486638C0162E7DA
:103B400073E00E949B63009719F477980C944226C7
:103B5000C80165E773E00E949B63009719F4779AA8
:103B60000C944226779903C082E793E002C085E770
:103B700093E000D000D02FE935E09DC4609174043B
:103B80007091750480E090E00E9486638C016CE780
:103B900073E00E949B63009709F043C06091740436
:103BA0007091750480E090E00E9486638C0100971C
:103BB00011F40C9442266FE773E00E949B63009718
:103BC00029F482E29FEFACECBBE318C0C8010E946D
:103BD00079626B017C0120E030E040E050E00E941F
:103BE000B35E8823D1F081E00E948C099B01AC0177
:103BF000C701B6010E94B75EDC01CB0180937B0454
:103C000090937C04A0937D04B0937E048BE794E0B2
:103C100063E170E044E050E074C200D088E399E0D2
:103C20009CC0C80165E873E00E949B63009709F09F
:103C300045C0609174047091750480E090E00E942A
:103C400086638C01009711F40C9442266FE773E0B1
:103C50000E949B63009729F482E29FEFACECBBE3E8
:103C600018C0C8010E9479626B017C0120E030E03D
:103C700040E050E00E94B35E8823C1F082E00E94E1
:103C80008C099B01AC01C701B6010E94B75EDC0143
:103C9000CB018093770490937804A0937904B09338
:103CA0007A0487E794E06FE070E0B4CF00D085E459
:103CB00099E0EDB7FEB79283818355C0C80168E8EB
:103CC00073E00E949B63009709F052C060917404F6
:103CD0007091750480E090E00E9486638C010097EB
:103CE00009F4D0C76FE773E00E949B63009729F443
:103CF0008DEE97E4AAE8BCE320C0C8010E94796277
:103D00006B017C0120E030E040E050E00E94B35EB7
:103D1000882301F180E00E948C094B015C01C701FE
:103D2000B60121EE3AE744E95EE30E944E5EA5014A
:103D300094010E94B75EDC01CB0180937F049093D5
:103D40008004A0938104B09382048FE794E067E13C
:103D500070E060CF00D082E599E0ADB7BEB71296B3
:103D60009C938E9311970E941C640F900F908AC7AA
:103D70000E94E009AB01BC0100D000D000D08FE56B
:103D800099E0EDB7FEB792838183438354836583C3
:103D900076830E941C64EDB7FEB736960FB6F89492
:103DA000FEBF0FBEEDBF81E00E948C0920917B0415
:103DB00030917C0440917D0450917E040E94D15F3B
:103DC0006B01182F092F82E00E948C09AB01BC0106
:103DD0008DB79EB70A970FB6F8949EBF0FBE8DBFE2
:103DE000EDB6FEB60894E11CF11C86E699E0ADB78D
:103DF000BEB712969C938E93119798018C2D9D2D92
:103E0000A32FB22FF70182839383A483B583CB01C1
:103E1000BA0120917704309178044091790450914F
:103E20007A040E94D15FDC01CB01F701868397837E
:103E3000A087B1870E941C648DB79EB70A960FB603
:103E4000F8949EBF0FBE8DBF18C760917404709127
:103E5000750480E090E00E948663009771F160E055
:103E600070E040E150E00E943861AB01BC018091FC
:103E7000F0059091F1058417950799F15093F1059C
:103E80004093F00580EF95E06BE170E042E050E098
:103E90000E9462658091F0059091F10500D000D0FC
:103EA00023EA35E0ADB7BEB712963C932E93119737
:103EB00014969C938E9313970EC08091F005909169
:103EC000F10500D000D023EB35E0EDB7FEB732832B
:103ED0002183948383830E941C640F900F900F9022
:103EE0000F900E94E70A00D000D087EC95E0ADB7B4
:103EF000BEB712969C938E93119781E090E0149632
:103F00009C938E9313970E941C6484ED95E0EDB70B
:103F1000FEB79283818382E090E0948383830E9442
:103F20001C648FED95E0ADB7BEB712969C938E934F
:103F3000119784E090E014969C938E9313970E94BF
:103F40001C648AEE95E0EDB7FEB79283818388E02A
:103F500090E0948383830E941C6486EF95E0ADB764
:103F6000BEB712969C938E93119780E190E01496C1
:103F70009C938E9313970E941C6481E096E0EDB7AA
:103F8000FEB79283818380E290E0948383830E94D2
:103F90001C648DE096E0ADB7BEB712969C938E93ED
:103FA000119780E490E014969C938E9313970E944F
:103FB0001C648BE196E0EDB7FEB79283818380E8C5
:103FC00090E0948383830E941C6489E296E0ADB7FD
:103FD000BEB712969C938E93119780E091E0149651
:103FE0009C938E9313970E941C6488E396E0EDB730
:103FF000FEB79283818380E092E0948383830E9462
:104000001C6487E496E0ADB7BEB712969C938E937E
:10401000119780E094E014969C938E9313970E94DE
:104020001C6483E596E0EDB7FEB79283818380E060
:1040300098E0948383830E941C640F900F900F90EC
:104040000F9020C60E9425151DC6609174047091C2
:10405000750480E090E00E9486636FE773E00E9441
:104060009B63009711F481E001C080E00E942C174F
:1040700020917604222309F405C600D000D0EDB7C4
:10408000FEB7319681E696E0B8C50E94DE15209114
:104090007604222309F4F6C500D000D0EDB7FEB7B0
:1040A000319684E696E0A9C50E94D9152091760440
:1040B000222309F4E7C500D000D0EDB7FEB7319652
:1040C00087E696E09AC5609174047091750480E06B
:1040D00090E00E9486638C0162E773E00E949B631C
:1040E000009791F480915A0490915B0484609093BE
:1040F0005B0480935A048AE594E069E070E042E052
:1041000050E00E946265BEC5C80165E773E00E9489
:104110009B639C0180915A0490915B0421153105A9
:1041200011F48B7FE4CF82FF03C082E793E002C0EB
:1041300085E793E000D000D022E739E0BCC10C94C1
:104140000000A0C500D08AE696E0ADB7BEB71296D3
:104150009C938E9311970E941C64209176040F907B
:104160000F902223A9F000D000D0EDB7FEB7319612
:104170008EE696E0ADB7BEB712969C938E931197DC
:10418000228313820E941C640F900F900F900F9057
:1041900088E10FB6F89480936000109260000FBE23
:1041A0000C94007C6FC5609174047091750480E07C
:1041B00090E00E9486637C0162E773E00E949B634B
:1041C000009749F40E94AA3A80915A0490915B04A6
:1041D00081608D7F8CCFC70165E773E00E949B6390
:1041E000009741F40E949B3B80915A0490915B049C
:1041F0008C7F7DCF0DE813E0C701B8010E949B635F
:10420000009749F40E949B3B80915A0490915B0473
:104210008E7F82606CCF80915A0481FF0BC000D0EA
:1042200000D086E799E0EDB7FEB7928381831483CF
:10423000038301CF80FF03C082E793E002C085E7DC
:1042400093E000D000D02AE739E0ADB7BEB71296B0
:104250003C932E93119714969C938E931397EBCEC9
:1042600000D081E796E0EDB7FEB7928381830E948C
:104270001C648DB79EB70C970FB6F8949EBF0FBE07
:104280008DBFEDB7FEB7319680E996E0ADB7BEB70A
:1042900012969C938E9311978091251B9091261BCB
:1042A000A091271BB091281B82839383A483B5839D
:1042B0008091291B90912A1BA0912B1BB0912C1B44
:1042C00086839783A087B18780912D1B90912E1BA9
:1042D000A0912F1BB091301B82879387A487B5874D
:1042E0000E941C6420917604EDB7FEB73E960FB68F
:1042F000F894FEBF0FBEEDBF222309F4C3C400D063
:1043000000D0EDB7FEB7319687EA96E076C4F89410
:1043100009E081E090E0FC0100935700C895F02C83
:1043200020E030E0F90100935700C895E02C789424
:10433000F89423E030E0F90100935700C895102D60
:1043400082E090E0FC0100935700C895002D78941E
:1043500000D000D000D02AEA36E0EDB7FEB73283B5
:1043600021838091F9129091FA12A091FB12B091E1
:10437000FC1283839483A583B6830E941C6400D0BF
:1043800000D0EDB7FEB7319684EB96E0ADB7BEB77F
:1043900012969C938E931197028313821483158235
:1043A000E6821782F08611860E941C64EDB7FEB784
:1043B0003A960FB6F894FEBF0FBEEDBF0E9490165E
:1043C0002091660000D000D0EDB7FEB731968BED9E
:1043D00096E0ADB7BEB712969C938E931197228349
:1043E00013820E941C640F900F900F900F900E94F8
:1043F000E70A20917604222309F444C400D000D0B7
:10440000EDB7FEB7319687EE96E0F7C380E090E017
:104410000E94F30A81E090E00E94F30A2091760462
:10442000222309F42FC400D000D0EDB7FEB7319697
:104430008AEE96E0E2C30E9494140E94E70A20915B
:104440007604222309F41EC400D000D0EDB7FEB7D5
:1044500031968DEE96E0D1C360917404709175042D
:1044600080E090E00E9486638C0162E773E00E9426
:104470009B63009731F480915A0490915B048860AB
:1044800036CEC80165E773E00E949B639C01809172
:104490005A0490915B042115310511F4877F27CED2
:1044A00083FF03C082E793E002C085E793E000D07A
:1044B00000D02EE739E0EDB7FEB732832183B9CDC6
:1044C000609174047091750480E090E00E948663AE
:1044D00062E973E00E949B63009729F41092FB0548
:1044E0001092FA0546C08AEF95E00E946A2B7C0183
:1044F00008E913E03BC08DB79EB70C970FB6F89450
:104500009EBF0FBE8DBFEDB7FEB73196ADB7BEB73C
:1045100012961C930E931197D70112968C911297B5
:104520008283138213968C91139784831582189635
:104530008C9118978683178214968D919C9115976C
:104540009187808716968D919C9117979387828784
:104550000E940A64EDB7FEB73C960FB6F894FEBF12
:104560000FBEEDBFC7010E94102C7C01E114F104C5
:1045700011F620917604222309F484C300D000D0E0
:10458000EDB7FEB7319680EF96E037C30E94701703
:1045900079C3609174047091750480E090E00E948A
:1045A0008663009731F160E070E040E150E00E94E6
:1045B0003861DC01CB0190935F0480935E0400D0EE
:1045C00000D04DB75EB74F5F5F4F23EF36E0EDB7DA
:1045D000FEB732832183FA01938382830E941C6495
:1045E0000F900F900F900F908EE594E06DE070E0CB
:1045F00086CD00D000D084E097E0ADB7BEB712966C
:104600009C938E93119780915E0490915F04149611
:104610009C938E9313970E941C640F900F900F90A1
:104620000F900E94E70A00D000D087E197E0EDB735
:10463000FEB79283818381E090E0948383830E941C
:104640001C6484E297E0ADB7BEB712969C938E933C
:10465000119782E090E014969C938E9313970E949A
:104660001C6480E397E0EDB7FEB79283818384E01A
:1046700090E0948383830E941C648FE397E0ADB73E
:10468000BEB712969C938E93119788E090E0149693
:104690009C938E9313970E941C648EE497E0EDB771
:1046A000FEB79283818380E190E0948383830E94AC
:1046B0001C648BE597E0ADB7BEB712969C938E93C2
:1046C000119780E290E014969C938E9313970E942A
:1046D0001C648AE697E0EDB7FEB79283818380E49D
:1046E00090E0948383830E941C6487E797E0ADB7D2
:1046F000BEB712969C938E93119780E890E0149623
:104700009C938E9313970E941C6487E897E0EDB703
:10471000FEB79283818380E091E0948383830E943B
:104720001C6484E997E0ADB7BEB712969C938E9354
:10473000119780E092E014969C938E9313970E94B9
:104740001C6483EA97E0EDB7FEB79283818380E033
:1047500094E0948383830E941C6480EB97E0ADB760
:10476000BEB712969C938E93119780E098E01496B2
:104770009C938E9313970E941C648DEB97E0EDB78A
:10478000FEB79283818380E090E1948383830E94CB
:104790001C64209176040F900F900F900F902223AD
:1047A00009F470C200D000D0EDB7FEB731968AECA4
:1047B00097E023C2609174047091750480E090E0EA
:1047C0000E948663009751F160E070E04AE050E09B
:1047D0000E943861DC01CB0190935D0480935C04FE
:1047E00000D000D04DB75EB74F5F5F4F2DEC37E084
:1047F000EDB7FEB732832183FA01938382830E944F
:104800001C640F900F900F900F908CE594E06BE07C
:1048100070E042E050E00E94626518C000D000D015
:104820008AEE97E0ADB7BEB712969C938E93119720
:1048300080915C0490915D0414969C938E931397E1
:104840000E941C640F900F900F900F90209176049F
:10485000222309F417C200D000D0EDB7FEB731967D
:104860008BE098E0CAC10E94872D20917604222314
:1048700009F408C200D000D0EDB7FEB731968EE043
:1048800098E0BBC100D081E198E0EDB7FEB792831C
:1048900081830E941C640F900F9080E00E942C176F
:1048A0000E94DE1500D000D084E298E0ADB7BEB71C
:1048B00012969C938E93119780E490E014969C93AB
:1048C0008E9313970E941C6400D0EDB7FEB731960B
:1048D0008CE398E0ADB7BEB712969C938E93119778
:1048E0008091CF1F828313828091D01F8483158291
:1048F0000E941C640F900F908FE498E0EDB7FEB714
:104900009283818380915C0490915D04948383837E
:104910000E941C648AE698E0ADB7BEB712969C93DD
:104920008E93119780915E0490915F0414969C93EE
:104930008E9313970E941C640F900F900F900F900E
:104940000E94E009AB01BC0100D000D000D083E898
:1049500098E0EDB7FEB792838183438354836583E8
:1049600076830E941C64EDB7FEB736960FB6F894B6
:10497000FEBF0FBEEDBF0E94290A0E94FA09AB01DB
:10498000BC0100D000D000D080E998E0ADB7BEB740
:1049900012969C938E931197EDB7FEB74383548381
:1049A000658376830E941C648DB79EB706960FB60A
:1049B000F8949EBF0FBE8DBF1D9B03C089E793E097
:1049C00002C085E793E000D000D02EE938E0ADB713
:1049D000BEB712963C932E93119714969C938E9388
:1049E00013970E941C648091721B9091731BA0917D
:1049F000741BB091751B4091761B5091771B609191
:104A0000781B7091791B00D000D000D00DB71EB775
:104A10000F5F1F4F2AEA38E0EDB7FEB732832183DC
:104A2000F80182839383A483B58346835783608789
:104A300071870E941C64EDB7FEB738960FB6F894E4
:104A4000FEBF0FBEEDBF87EC98E0928381830E948A
:104A50001C6480915A040F900F9081FF0EC000D00B
:104A600084ED98E0ADB7BEB712969C938E931197E4
:104A70000E941C640F900F9017C080FF03C082E754
:104A800093E002C085E793E000D000D02AED38E043
:104A9000EDB7FEB732832183948383830E941C6425
:104AA0000F900F900F900F9080915A0483FF03C0D6
:104AB00082E793E002C085E793E000D000D02EEDBE
:104AC00038E0ADB7BEB712963C932E93119714966B
:104AD0009C938E9313970E941C648091F005909193
:104AE000F10521EF38E0EDB7FEB7328321839483DF
:104AF00083830E941C640F900F900F900F90779902
:104B000003C082E793E002C085E793E000D000D0C5
:104B10002EEF38E0ADB7BEB712963C932E931197A7
:104B200014969C938E9313970E941C642091760494
:104B30000F900F900F900F90222309F4A3C000D084
:104B400000D0EDB7FEB731968AE099E056C00E94DA
:104B5000B51620917604222309F494C000D000D029
:104B6000EDB7FEB731968DE099E047C00E94A80EE0
:104B700000D000D000D080E199E0EDB7FEB792837D
:104B8000818380911D1390911E13A0911F13B091EA
:104B9000201383839483A583B6830E941C648BE1D6
:104BA00099E0ADB7BEB712969C938E931197809102
:104BB000CB1F9091CC1FA091CD1FB091CE1FEDB710
:104BC000FEB783839483A583B6830E941C648DB74C
:104BD0009EB706960FB6F8949EBF0FBE8DBF0E947B
:104BE000E70A20917604222309F44CC000D000D0BB
:104BF000EDB7FEB7319688E299E0ADB7BEB7129631
:104C00009C938E9311972283138215CA609174042A
:104C10007091750480E090E00E9486636FEB73E012
:104C20000E949B630097A1F46091740470917504D5
:104C300080E090E00E948663009721F10E947D62EF
:104C4000803100F590915201982B909352011AC037
:104C50008091520100D000D02BE239E0EDB7FEB7D1
:104C60003283218390E08F709070948383830E94BD
:104C70001C640F900F900F900F900E94E70A02C0E3
:104C80000E94FE14A981BA8111961C921E9283E0A3
:104C90000F900F90DF91CF911F910F91FF90EF90A8
:104CA000DF90CF90BF90AF909F908F907F906F904C
:104CB0005F904F903F902F900895F89491E2E0E03C
:104CC000F0E0909357008491E2E0F0E09093570079
:104CD0004491E4E0F0E090935700E49190E0A0E08C
:104CE000B0E0DC019927882750E060E070E0762F83
:104CF000652F542F4427840F951FA61FB71F8E0FB3
:104D0000911DA11DB11D8093F9129093FA12A093E9
:104D1000FB12B093FC1278940895CF93DF9300D0E8
:104D200000D000D0CDB7DEB7CE0101966DE070E0C7
:104D300042E050E00E94446589819A812FEF8F3FC5
:104D4000920749F48EE594E06DE070E042E050E0B7
:104D50000E94626504C090935F0480935E04CE015C
:104D600001966BE070E042E050E00E94446589816A
:104D70009A812FEF8F3F920779F48CE390E0909324
:104D80005D0480935C048CE594E06BE070E042E0AD
:104D900050E00E94626504C090935D0480935C04BF
:104DA000CE01019669E070E042E050E00E94446567
:104DB00089819A812FEF8F3F920779F482E090E00A
:104DC00090935B0480935A048AE594E069E070E074
:104DD00042E050E00E94626504C090935B048093BF
:104DE0005A04CE0101966BE170E042E050E00E946F
:104DF000446589819A812FEF8F3F920769F4109261
:104E0000F1051092F00580EF95E06BE170E042E073
:104E100050E00E94626504C09093F1058093F00514
:104E20008FEB9FE160E070E049E050E00E94446554
:104E30000E946F0CCE01039663E170E044E050E005
:104E40000E9444658B819C81AD81BE818F3F2FEF95
:104E500092072FEFA2072FEFB20749F48BE794E0F8
:104E600063E170E044E050E00E94626508C08BE7B7
:104E700094E063E170E044E050E00E944465CE01BC
:104E800003966FE070E044E050E00E9444658B813F
:104E90009C81AD81BE818F3F2FEF92072FEFA2073C
:104EA0002FEFB20749F487E794E06FE070E044E049
:104EB00050E00E94626508C087E794E06FE070E010
:104EC00044E050E00E944465CE01039667E170E043
:104ED00044E050E00E9444658B819C81AD81BE819D
:104EE0008F3F2FEF92072FEFA2072FEFB20749F462
:104EF0008FE794E067E170E044E050E00E94626573
:104F000008C08FE794E067E170E044E050E00E9461
:104F1000446526960FB6F894DEBF0FBECDBFDF9175
:104F2000CF9108956C9A6B9A6A9A6F9A729A749A52
:104F3000739A779A809880B3897F80BB87E080934B
:104F40007E00549A0E945D260E948D2681E00E9478
:104F5000F10880E090E00E94830C0E946134089583
:104F6000CF93DF93EC0188819981009731F027E09E
:104F70008533920709F077C06DC00E949227809117
:104F80005A0480FD02C00E949B3B809170008C7F80
:104F9000809370008091B60080628093B60010927A
:104FA000B20082E08093B1008091B60090E08770FB
:104FB00090700097C9F780917000816080937000B5
:104FC0000E9405080E94A70880E090E066E976E06C
:104FD0000E946D390E94D91580E00E942C170E9412
:104FE000043E8093FC050E945D3C8093FD0500D04B
:104FF00000D000D0EDB7FEB7319624EC33E0ADB76A
:10500000BEB712963C932E931197828313828091A0
:10501000FC05848315820E940A641092FF05109299
:10502000FE058DB79EB706960FB6F8949EBF0FBECD
:105030008DBF80E594E09093C91F8093C81F83E2E1
:1050400090E0909301068093000685E397E09983B2
:1050500088830DC0633259F48EEF95E060E070E014
:105060000E94FF17E6CF1982188283E001C081E019
:10507000DF91CF9108950895FC01DB018C9180832D
:1050800011968C91119781830895FC01DB01908129
:105090008C91981741F421E030E0918111968C9128
:1050A0001197981711F020E030E0C9010895BC0174
:1050B0008FEC9FE10E943C280895DC011996ED9148
:1050C000FC911A970280F381E02D309709F0099541
:1050D00008950F931F93CF93DF9300D0CDB7DEB722
:1050E0008C0188E10E94FD30BC01CE0101960E9436
:1050F0003C28D8011996ED91FC911A970190F08106
:10510000E02DC801BE016F5F7F4F09950F900F9092
:10511000DF91CF911F910F910895EF92FF920F931E
:105120001F93CF93DF93EC018B017A0145E954E0A3
:105130000E94B928FA86E986C80169E974E00E94EC
:105140001729DF91CF911F910F91FF90EF90089554
:105150000E94D2280895CF93DF93EC0188E16FEC91
:105160007FE10E94F330CE010E94D528DF91CF91DC
:105170000895EF92FF920F931F93CF93DF93EC016B
:105180008B017A010E94F328F886EF82C8016DE94D
:1051900074E00E941729DF91CF911F910F91FF902A
:1051A000EF9008950E94FC2808950E9413410895ED
:1051B000DC011796ED91FC9118970190F081E02D9C
:1051C00009950895DC011796ED91FC9118970280DE
:1051D000F381E02D309709F0099508958CE999E065
:1051E0000E94662B0895FC01738362838CE999E029
:1051F000BF010E94D92B0895BC018CE999E00E945F
:10520000A42B0895CF93DF93EC018CE999E00E94E1
:105210006A2B08C0FC01228133812C173D0721F045
:105220000E94102C0097B1F7DF91CF9108950F9352
:105230001F93CF93DF938B010E940229EC0100970B
:1052400031F01D830C83C8010E9456438E83DF9189
:10525000CF911F910F9108951F93CF93DF93EC018E
:10526000162F888580FF1DC0EC81FD813097C9F025
:10527000D0939F09C0939E0982E08887CE0106964D
:105280000995992787FD909502978230910510F036
:10529000133829F4CE01BE010E94552902C081E0D5
:1052A0008887DF91CF911F910895CF92DF92EF927F
:1052B000FF920F931F93CF93DF93EC017B01C0907C
:1052C0009E09D0909F090091A0091091A109F801B1
:1052D00003C00190F081E02DEC17FD0719F0309725
:1052E000C1F746C0209709F443C08885882309F197
:1052F00018860BC0C017D10729F0C80167E8AE01B6
:105300000E942C29F801008111810115110591F7E6
:10531000EC81FD81309769F0CE15DF0551F0D09317
:105320009F09C0939E09CE01069663E840E050E0D5
:105330000995E091A009F091A109CE17DF0791F43A
:10534000888199819093A1098093A0090DC08081E3
:1053500091818C179D0729F488819981918380839D
:1053600003C0FC01309799F7D0929F09C0929E0923
:10537000DF91CF911F910F91FF90EF90DF90CF9031
:1053800008951F93CF93DF931092A209C091A009B3
:10539000D091A10911E00EC08985882341F01887BA
:1053A0001986CE0162E840E050E00E942C29099065
:1053B000D881C02D209781F7DF91CF911F9108955B
:1053C0008091A309982F9F5F9093A30908956091FE
:1053D0009E0970919F090E94552908958AE880933B
:1053E000A3091092A4091092A5091092A109109284
:1053F000A00910929F0910929E0908958091A20918
:10540000882311F00E94C1297091A509772309F41E
:1054100055C02091A40930E0F901EE0FFF1FEE0FF7
:10542000FF1FE20FF31FEA55F64F60816093460AB3
:10543000418152815093480A4093470A8381948165
:1054400090934A0A8093490A2F5F3F4F2F71307023
:105450002093A40971507093A509009741F580919C
:10546000A0099091A10918C08091A209882311F088
:105470000E94C1294091470A5091480A80914B0AE5
:1054800090914C0A6091460A0E942C29E0914B0AA7
:10549000F0914C0A8081918190934C0A80934B0A41
:1054A00080914B0A90914C0A0097F1F607C0613841
:1054B00019F421E0FC0120870E942C298091A20987
:1054C0002091A50990E0820F911D08958091A20975
:1054D0002091A50990E0820F911D08959C01709183
:1054E000A5097032D9F08091A409870F8F7180933C
:1054F0004D0A90E0FC01EE0FFF1FEE0FFF1FE80FBB
:10550000F91FEA55F64F6083528341833483238326
:105510007F5F7093A50980E090E0089581E090E0BE
:105520000895CF93DF93C0919E09D0919F090E9467
:105530002C29D0939F09C0939E09DF91CF910895A4
:10554000FC01AB019091A0098091A109A92FB82F6E
:1055500003C00D90BC91A02DAE17BF0791F010971E
:10556000C1F7309771F090838183F093A109E093A4
:10557000A00981E0808717821682CF0161E80E942E
:10558000912A0895FC01009741F080858150823076
:1055900020F481E081878093A209089521E030E022
:1055A000FC018085882311F420E030E0C9010895D2
:1055B000CF93DF93EC014A815B818C819D8160E018
:1055C00070E00E9494632A813B8188819981289FA1
:1055D000A001299F500D389F500D11248E819F816D
:1055E00060E070E00E949463DF91CF910895DC0148
:1055F00012962D913C91139780E090E01DC0149677
:10560000ED91FC911597E80FF91F4081442399F41F
:1056100021E020832D913C911197829FA001839FCF
:10562000500D929F500D112416968D919C911797B5
:10563000840F951F089501968217930701F780E064
:1056400090E00895FC0146815781A281B38120E05A
:1056500030E019C04617570781F4A481B581A20F25
:10566000B31F8C91181614F481508C930480F5812B
:10567000E02DE20FF31F8081089580819181480F12
:10568000591F2F5F3F4F2A173B0721F78FEF0895D0
:10569000FC014681578164177507A8F0A081B1818C
:1056A00082819381A89F9001A99F300DB89F300DF2
:1056B0001124240F351F81E090E06217730728F052
:1056C00080E090E0089580E090E00895FC01118270
:1056D00010820895FC01808191810895FB01208151
:1056E0003181FC01318320830895FC018081918107
:1056F000009711F40895C901FC0120813181211521
:105700003105C9F70895DC01ED91FC9111973097AF
:1057100029F40BC0DF010190F081E02D808191819F
:105720000097C1F711961C921E92CF010895DC01DB
:10573000ED91FC911197309729F08081918111961C
:105740009C938E93CF010895CF93DF93EC01E88172
:10575000F9813097B9F0A0E0B0E002C0DF01FC01B0
:1057600080819181E617F70759F4109719F499830E
:10577000888303C011969C938E931182108202C07D
:10578000009761F7DF91CF9108950F931F93CF9307
:10579000DF938C01EB010E94A42BF80180819181A1
:1057A00099838883D183C083DF91CF911F910F911B
:1057B00008950F931F93CF93DF938C01EB010E9409
:1057C000A42B19821882C8010E94752B009711F42E
:1057D000F80101C0FC01D183C083DF91CF911F91FB
:1057E0000F910895DC01ED91FC91119780E090E01C
:1057F00004C001960190F081E02D3097D1F7089513
:10580000FB01BA01309719F40E94C52B08958081DD
:105810009181DA0111969C938E9351834083089570
:10582000009721F0FC0180819181089580E090E053
:10583000089580914E0A90914F0A009729F4109292
:10584000510A1092500A08950E941B38BC01E09141
:105850004E0AF0914F0A4281538180819181480F15
:10586000591F461B570B0CC08281938120813181C7
:10587000820F931F861B970B8417950708F4AC01C2
:105880000480F581E02D309779F7460F571F50932C
:10589000510A4093500A08958BEA94E00E94C22A6C
:1058A0000895EF92FF920F931F93CF93DF937C01A4
:1058B000FC0180819181009729F08A35910509F0DA
:1058C0006DC00BC010924F0A10924E0A8AE590E00C
:1058D000F7019183808381E065C0673859F5A09115
:1058E0004E0AB0914F0A04C014960D90BC91A02DA1
:1058F000109741F316968D919C91179784179507F1
:1059000099F3A0934E0AB0934F0A0DC086819781F8
:105910008417950739F48481958115969C938E930D
:105920001497FD01DF011496ED91FC9115973097C6
:1059300069F7CCCF623851F6C0914E0AD0914F0A28
:1059400000E010E028C0CE010E943B470097F1F034
:105950008E819F8168E8AE010E946E2A0097A1F4B3
:105960001F821E828C819D810115110521F0F80195
:105970009583848304C090934F0A80934E0A1D82BE
:105980001C820E94192CD8CF0E944C2C9C818D81A6
:105990008E01C92FD82F2097B1F698CFF701118229
:1059A000108283E0DF91CF911F910F91FF90EF90D4
:1059B0000895CF93DF93EC010E944C2C8E819F8140
:1059C00030914E0A20914F0A009759F0E32FF22FA1
:1059D00006C0EC17FD0789F00480F581E02D3097B3
:1059E000C1F780919E0990919F099F838E833C838C
:1059F0002D83D0934F0AC0934E0A0E94192CDF9139
:105A0000CF910895CF93DF93EC010E941B47CE0105
:105A10000E94D92CDF91CF910895CF93DF93EC01B1
:105A20000E942747CE010E94D92CDF91CF91089583
:105A3000CF93DF93EC010E943147CE010E94D92C15
:105A4000DF91CF910895FC0180819181860F971F8E
:105A5000918380830E94192C089521E030E0FC019D
:105A600086819781009711F020E030E0C901089508
:105A7000FC012281338180819181280F391FC90166
:105A80000895FC0180819181089581E090E020914A
:105A90004E0A30914F0A2115310511F480E090E053
:105AA000089580914E0A90914F0A009729F08091B5
:105AB000500A9091510A089580E090E00895CF93A4
:105AC000DF93EC01E0914E0AF0914F0A8E179F0789
:105AD00041F48C819D8190934F0A80934E0A14C0AB
:105AE000FC01309731F0848195818C179D07C1F7B7
:105AF00007C01D821C821F821E82DF91CF910895F4
:105B00008C819D81958384830E94192CF2CFCF9341
:105B1000DF93D091CF1FC091D01F0E944738AB01B7
:105B2000BC018DB79EB7825590400FB6F8949EBFCA
:105B30000FBE8DBFEDB7FEB7319688E899E0ADB7DF
:105B4000BEB712969C938E931197D2831382C4830F
:105B5000158246835783608771878091C221909117
:105B6000C321A091C421B091C52182879387A487C6
:105B7000B5878091C6219091C721A091C821B0918D
:105B8000C92186879787A08BB18B8091CA2190917C
:105B9000CB21A091CC21B091CD21828B938BA48B72
:105BA000B58B8091CE219091CF21A091D021B09141
:105BB000D121868B978BA08FB18F8091D22190912C
:105BC000D321A091D421B091D521828F938FA48F1E
:105BD000B58F8091D6219091D721A091D821B091F5
:105BE000D921868F978FA0A3B1A38091DA219091BC
:105BF000DB21A091DC21B091DD2182A393A3A4A39A
:105C0000B5A38091DE219091DF21A091E021B09198
:105C1000E12186A397A3A0A7B1A78091E22190914B
:105C2000E321A091E421B091E52182A793A7A4A745
:105C3000B5A78091E6219091E721A091E821B0914C
:105C4000E92186A797A7A0ABB1AB8091EA219091FB
:105C5000EB21A091EC21B091ED2182AB93ABA4ABF1
:105C6000B5AB8091EE219091EF21A091F021B09100
:105C7000F12186AB97ABA0AFB1AF8091F2219091AB
:105C8000F321A091F421B091F52182AF93AFA4AF9D
:105C9000B5AFEDB7FEB7FF968091F6219091F72151
:105CA000A091F821B091F92180839183A283B383DD
:105CB000EDB7FEB7ED5BFF4F8091FA219091FB218C
:105CC000A091FC21B091FD2180839183A283B383B5
:105CD000EDB7FEB7E95BFF4F8091FE219091FF2168
:105CE000A0910022B091012280839183A283B3838B
:105CF000EDB7FEB7E55BFF4F809102229091032242
:105D0000A0910422B091052280839183A283B38362
:105D1000EDB7FEB7E15BFF4F80910622909107221D
:105D2000A0910822B091092280839183A283B3833A
:105D30000E941C64D091CF1FC091D01F8DB79EB719
:105D40008E5A9F4F0FB6F8949EBF0FBE8DBF0E9414
:105D50004738AB01BC01ADB7BEB7D2970FB6F894C8
:105D6000BEBF0FBEADBFEDB7FEB7319684E69AE079
:105D700012969C938E931197D2831382C4831582BB
:105D8000468357836087718780910A2290910B2206
:105D9000A0910C22B0910D2282879387A487B587AA
:105DA00080910E2290910F22A0911022B091112289
:105DB00086879787A08BB18B8091122290911322B6
:105DC000A0911422B0911522828B938BA48BB58B5A
:105DD0008091162290911722A0911822B091192239
:105DE000868B978BA08FB18F80911A2290911B2266
:105DF000A0911C22B0911D22828F938FA48FB58F0A
:105E000080911E2290911F22A0912022B0912122E8
:105E1000868F978FA0A3B1A38091222290912322F5
:105E2000A0912422B091252282A393A3A4A3B5A379
:105E30008091262290912722A0912822B091292298
:105E400086A397A3A0A7B1A7809132229091332275
:105E5000A0913422B091352282A793A7A4A7B5A719
:105E60008091362290913722A0913822B091392228
:105E700086A797A7A0ABB1AB0E941C648DB79EB755
:105E8000C2960FB6F8949EBF0FBE8DBFDF91CF9123
:105E9000089580E38093560A0895CF93DF9360912D
:105EA000560A70E0C0E3D0E0C61BD70B675A754FA7
:105EB000AE010E948B63CE01DF91CF910895CF9206
:105EC000DF92EF92FF920F931F93CF93DF937C01AA
:105ED000C090540AD090550A6091560A70E086012D
:105EE000005D1F4F061B170B01381105D8F4C0E3E6
:105EF000D0E0C61BD70B675A754FAE010E948B636B
:105F0000C7018C0F9D1F6091570A7091580A20910C
:105F1000520A3091530A620F731FA6010E948B63CD
:105F2000C80102C080E090E0DF91CF911F910F91F6
:105F3000FF90EF90DF90CF9008959091560A980FC0
:105F40009093560A08954091540A5091550A9C0125
:105F50004817590798F08091520A9091530A820F7E
:105F6000931F9093530A8093520A421B530B5093F2
:105F7000550A4093540A81E090E0089580E090E053
:105F800008959093550A8093540A08958091520A77
:105F90009091530A8757954F08958091560A90E043
:105FA000875A954F089581E090E02091570A3091EB
:105FB000580A4AE02938340711F480E090E0089547
:105FC0000E94D32F009769F089E89AE06091570A00
:105FD0007091580A4091540A5091550A0E948B635F
:105FE00008954091520A5091530A41155105C1F04C
:105FF0008091540A9091550AC096A9E8BAE020E32E
:1060000030E007C0FD01E40FF51F60816D932F5F45
:106010003F4F28173907B4F31092530A1092520ACF
:1060200008958091570A9091580A08958091540AD2
:106030009091550A08959091560A80E3891B08951E
:1060400020E38091560A281B8091540A9091550AAA
:10605000820F911D08951F93CF93DF93EC01109150
:10606000560A812F90E08C179D076CF00E9420301B
:106070008C0F9D1F8138910530F41C1B1093560A1C
:1060800081E090E002C080E090E0DF91CF911F912D
:106090000895CF93DF93E9EDFFE11192119280E231
:1060A000E930F807D1F7C0E0D0E0CE01880F991FA2
:1060B0008F52904E63E974E00E943C282196C430D0
:1060C000D10599F7DF91CF9108951092530A10925C
:1060D000520A1092550A1092540A80E38093560A8D
:1060E00089E89AE09093580A8093570A0E944930B1
:1060F00008950F931F93CF93DF93EC018B010E94C0
:106100006530D093580AC093570A1093550A0093EC
:10611000540ADF91CF911F910F910895EF92FF9252
:106120000F931F93CF93DF9300D0CDB7DEB78C01D1
:1061300069837A830E9465306981E62E7A81F72E21
:1061400081E8E816F10418F030E8E32EF12C809194
:10615000570A9091580AB801A7010E948B63F092E8
:10616000550AE092540AC7010F900F90DF91CF912A
:106170001F910F91FF90EF900895FC01A9EDBFE1F1
:1061800080E30D9001928150E1F7FB01A1EDBFE1A9
:1061900088E00D9001928150E1F70895A9EDBFE1EB
:1061A000FC0180E301900D928150E1F7A1EDBFE188
:1061B000FB0188E001900D928150E1F70895E82FEE
:1061C000F0E0EE0FFF1FE752F04E7183608381E035
:1061D00090E00895E82FF0E0EE0FFF1FE752F04E39
:1061E00080819181089590E0880F991F8F55904E7E
:1061F0000E943C2881E090E0089590E0880F991F6C
:106200008F55904E08958115910511F00197F1F782
:106210000895E0910C20F0910D20908180910B2049
:1062200089230895E0910920F0910A2080819091BE
:106230000B20892B8083E0910E20F0910F2080812C
:1062400090910B20892B80830895E0910920F09193
:106250000A20908180910B20809589238083E09192
:106260000E20F0910F20908180910B208095892342
:10627000808308951F93CF93DF93E0910920F091DD
:106280000A20908180910B20809589238083E09162
:106290000E20F0910F20808190910B20892B80831C
:1062A0008FEB93E00E9403311FB7F894E0910E202A
:1062B000F0910F20908180910B208095892380831D
:1062C00083E890E00E940331E0910C20F0910D20D2
:1062D000D081C0910B201FBF78948BE393E00E9484
:1062E0000331E0910C20F0910D20808190910B20E2
:1062F000892319F08D2F8C2301C081E0DF91CF918C
:106300001F91089550930F2040930E2070930A2000
:106310006093092090930D2080930C2081E090E001
:1063200002C0880F991F2A95E2F780930B200E94E4
:106330003A310895CF93DF93C82FDFB7F894E091F7
:106340000E20F0910F20808190910B20892B80836B
:1063500083E090E00E940331CC2351F0E0910E20C5
:10636000F0910F20908180910B208095892380836C
:1063700087E190E00E940331E0910C20F0910D2024
:10638000808190910B20892309F4C0E089E590E099
:106390000E940331E0910E20F0910F2090818091B6
:1063A0000B20809589238083DFBF8BE390E00E94E0
:1063B00003318C2FDF91CF910895CF93DF93C82FB6
:1063C000D8E08C2F81700E949A31C6958111C068E7
:1063D000D150B9F78C2FDF91CF9108958FEF0E94A4
:1063E000DD310895DF92EF92FF920F931F93CF93C9
:1063F000DF93182FEB010E943A31882381F580EF5B
:106400000E94DD31EE2400E498E0D92E81E00E9464
:106410009A31F82E81E00E949A31882319F0FF20EA
:1064200069F020C0FF2051F4011728F0888180FF17
:1064300005C0101719F0E02EFF24F3948F2D0E9451
:106440009A31888186958883FF2011F0806888833F
:106450000150DA94D9F621960023B1F605C0EE2456
:10646000EA9402C08EEFE82E8E2DDF91CF911F911E
:106470000F91FF90EF90DF9008950F931F93CF93AC
:10648000DF93182FEB010E943A31209751F085E5F8
:106490000E94DD3108E089910E94DD310150D9F779
:1064A00003C08CEC0E94DD31812F0E94DD31DF9131
:1064B000CF911F910F9108950F931F93CF93DF9367
:1064C000E82FDB01EA01B9014C9150E011969C9153
:1064D000119780E0482B592BE03181F4CA018E7F5F
:1064E00033E0880F991F3A95E1F716962C9116978D
:1064F0004CE050E0421B5109480F591F57FF06C09E
:1065000081E08883509541955F4F01C01882E83241
:1065100099F414968C91149790E09C012076307039
:106520002036310549F086FF02C04E7F05C085FF49
:1065300002C04C7F01C0487FCA0124E09695879530
:106540002A95E1F7FB0180834F70F801408380E0DA
:10655000DF91CF911F910F9108950F931F93CF93C8
:10656000DF93EC018B018881B8010E94F2318883AE
:1065700081508D3F30F4F8018081883211F08031F4
:1065800091F7DF91CF911F910F910895CF93DF93F2
:10659000EC010E943A3184EBBE010E943D3281E061
:1065A0000E949A31C82F0E943A3181E0CC2309F42D
:1065B00080E0DF91CF9108951F93CF93DF93182F41
:1065C000EB010E943A310E940931882349F084E4AA
:1065D000BE010E943D32113029F00E94123102C0EA
:1065E00082E001C080E0DF91CF911F9108956F920A
:1065F0007F928F929F92BF92CF92DF92EF92FF9203
:106600000F931F93CF93DF93CDB7DEB729970FB6C4
:10661000F894DEBF0FBECDBF7C014B013A0169018A
:106620000E943A318EEBB7010E943D328E010F5F1E
:106630001F4FE9E0BE2E0E94EE31F80181938F01D9
:10664000BA94C9F7CE01019669E070E00E94094D45
:10665000882361F4F7018081BE016F5F7F4FA40141
:10666000930186010E945C3280E001C083E029969C
:106670000FB6F894DEBF0FBECDBFDF91CF911F9153
:106680000F91FF90EF90DF90CF90BF909F908F90F1
:106690007F906F9008958F929F92AF92BF92CF920A
:1066A000DF92EF92FF920F931F93CF93DF93CDB7BB
:1066B000DEB729970FB6F894DEBF0FBECDBFD82E38
:1066C0005B014A0179018EEB60E070E00E943D328F
:1066D0008E010F5F1F4FF9E0CF2E0E94EE31F801BF
:1066E00081938F01CA94C9F7CE01019669E070E0E9
:1066F0000E94094D882359F48D2DBE016F5F7F4F95
:10670000A501940187010E945C3280E001C083E012
:1067100029960FB6F894DEBF0FBECDBFDF91CF91A3
:106720001F910F91FF90EF90DF90CF90BF90AF90AF
:106730009F908F900895EF92FF921F93CF93DF93D6
:10674000CDB7DEB728970FB6F894DEBF0FBECDBF2A
:10675000182F262FDE011196E5EBF4E088E001907A
:106760000D928150E1F7E42EFF24E7FCF09441E71D
:1067700052E0E49EC001E59E900DF49E900D112420
:1067800064E670E00E946760CB0134E6239F9001CD
:106790001124820F931FFE01319640E0219130E0D9
:1067A000E216F30611F4019603C04F5F4830B1F7CB
:1067B000112319F0909581959F4F28960FB6F89464
:1067C000DEBF0FBECDBFDF91CF911F91FF90EF9045
:1067D00008950F931F93CF93DF93CDB7DEB72B9719
:1067E0000FB6F894DEBF0FBECDBF182F092F885FFC
:1067F000612F792F0E94DC32882309F048C066E4BB
:1068000071E48FE090E00E945434812F902FBE01FC
:106810006D5F7F4FAE014E5F5F4F9E012F5F3F4F19
:106820000E94F732882399F5DE011496E5EBF4E037
:1068300088E001900D928150E1F7E9814E2F50E000
:1068400021E732E0429FC001439F900D529F900D7F
:10685000112464E670E00E946760CB013A8124E66F
:10686000329F90011124820F931FDE01149620E0C5
:106870003D91E31711F4019603C02F5F2830C1F753
:106880002B81222331F0909581959F4F02C084E3A4
:1068900091E22B960FB6F894DEBF0FBECDBFDF910D
:1068A000CF911F910F910895DC01CB0181159105C6
:1068B000A105B10529F081509040A040B040D9F722
:1068C000089581E08093B90080E28093B800089534
:1068D00094EA9093BC009091BC0097FFFCCF9091FC
:1068E000B900987F983011F0903199F48093BB00F3
:1068F00084E88093BC008091BC0087FFFCCF90911E
:10690000B900987F983139F081E0903429F480E023
:10691000089581E0089580E0089544EA34E824E988
:106920004093BC009091BC0097FFFCCF9091B900C0
:10693000987F983011F0903199F78093BB00309395
:10694000BC009091BC0097FFFCCF9091B900987F5C
:10695000903211F0983539F42093BC009091BC002E
:1069600094FDFCCFDDCF08950E946834089584E93A
:106970008093BC008091BC0084FDFCCF089580937F
:10698000BB0084E88093BC008091BC0087FFFCCFF3
:106990009091B900987F81E0983209F480E00895E1
:1069A00084EC8093BC008091BC0087FFFCCF809179
:1069B000BB00089584E88093BC008091BC0087FFF1
:1069C000FCCF8091BB000895FC0180E191919093F0
:1069D0003F018150D9F780913C018F7D80933C012C
:1069E00080913C01877F80933C01FB0180E1919184
:1069F00090933E018150D9F780913C01806880934B
:106A00003C0180913D0180FFFCCF4051504080917E
:106A10003C01806280933C0180913C01877F8093A0
:106A20003C0112C0FB0180E1919190933E018150A5
:106A3000D9F780913C01806880933C0180913D01B1
:106A400080FFFCCF40515040141615065CF3F9014D
:106A500080E190913E0191938150D9F781E090E0DF
:106A60000895E6E4F1E08081208190813081829573
:106A700086958695837022952F70822B832B929515
:106A80009F70892B0895DF92EF92FF920F931F93CF
:106A9000CF93DF9300D0CDB7DEB780E06CE046E067
:106AA0000E94DF3889E18093C4001092C50082E023
:106AB0008093C00080E00E9481390E940B3884B727
:106AC00084B784B784B784B7E0E9F8E222E432E41B
:106AD000318320833A968DB79EB70A97E817F90756
:106AE000B8F300D000D083ED9AE0ADB7BEB71296F0
:106AF0009C938E9311978DEB94E014969C938E93B8
:106B000013970E941C640F900F900F900F900E949B
:106B10003A490E94EE298BEA94E060E070E00E941E
:106B2000A02A0E94CD47E0910805F091090509953A
:106B30000E94313590E00E947749CE0101960E9473
:106B40003D37882359F000D08EEE9AE0EDB7FEB7BE
:106B5000928381830E941C640F900F90CE01019656
:106B60000E9457280E9447378C010E944C37BC0175
:106B7000C801AE014F5F5F4F0E947B3C0E94AA3666
:106B80000E94603C0E9451370E94FC3D00D08EE084
:106B90009BE0ADB7BEB712969C938E9311970E945F
:106BA0001C6400D0EDB7FEB731960BE11BE0ADB72A
:106BB000BEB712961C930E9311978A81828313821B
:106BC0000E941C64EDB7FEB73196ADB7BEB7129602
:106BD0001C930E9311978981828313820E941C64F7
:106BE0000F900F908FE19BE0EDB7FEB7928381830A
:106BF0000E941C640F900F900E947D49E0918B05CC
:106C0000F0918C050995E0917205F0917305099555
:106C1000E0913405F09135050995009170051091CA
:106C20007105E0908905F0908A050E945D3CD82EA0
:106C30000E94043E2DB73EB72A5030400FB6F8945C
:106C40003EBF0FBE2DBFEDB7FEB7319621E23BE050
:106C5000ADB7BEB712963C932E9311971383028360
:106C6000F582E482D6821782808711860E941C6496
:106C7000E0919505F09196052DB73EB7265F3F4F01
:106C80000FB6F8943EBF0FBE2DBF3097D1F00995D7
:106C9000BC0100D000D08CE39BE0ADB7BEB712962C
:106CA0009C938E93119780E890E00E945360EDB71B
:106CB000FEB7748363830E941C640F900F900F9043
:106CC0000F9000D08FE49BE0ADB7BEB712969C93B7
:106CD0008E9311970E941C640F900F908DEC95E09D
:106CE00060E070E00E94A02A86ED93E00E94FF46DB
:106CF00000D081E59BE0EDB7FEB7928381830E94CF
:106D00001C640F900F900F900F90DF91CF911F9107
:106D10000F91FF90EF90DF90089500D000D000D049
:106D2000EDB7FEB7319629E53BE0ADB7BEB7129699
:106D30003C932E93119793838283758364830E947F
:106D40001C648DB79EB706960FB6F8949EBF0FBE13
:106D50008DBF08950F931F93CF93DF93CDB7DEB709
:106D6000A0970FB6F894DEBF0FBECDBF82E290E0D1
:106D70000E945C65082F282F2B50203108F0982F97
:106D80009095891709F46DC000D08FE79BE0ADB7EF
:106D9000BEB712969C938E9311970E941C648E012D
:106DA0000F5F1F4F0F900F90D80180E090E0FC0123
:106DB000E958F44FE491ED93019688309105B9F7C5
:106DC000F894CE0101966EE370E048E050E00E9436
:106DD0006265D80180E090E0FC01E759F44FE4914E
:106DE000ED9301968E309105B9F7CE01019660E3DF
:106DF00070E04EE050E00E94626580E090E0FC01AF
:106E0000E15AF44FE491D801ED938D0101968A3057
:106E10009105A9F7CE01019666E270E04AE050E0E4
:106E20000E94626580E290E06DEC7BEA0E947A65E8
:106E30008EE190E060E070E00E947A658DE190E084
:106E400060E00E946C6584E290E060E070E00E9487
:106E50007A650AE182E290E06AE175EE0E947A6565
:106E60007894802FA0960FB6F894DEBF0FBECDBFEA
:106E7000DF91CF911F910F910895F8946EE370E028
:106E800042E050E00E944465789480E0089580E2FA
:106E900090E00E945C6508958EE190E00E945C6540
:106EA00008958DE190E00E945465089540911E2060
:106EB00050911F20609120207091212090E0A0E04F
:106EC000B0E0480F591F6A1F7B1F40931E2050934C
:106ED0001F20609320207093212040911A20509110
:106EE0001B2060911C2070911D20480F591F6A1FA4
:106EF0007B1F40931A2050931B2060931C2070939B
:106F00001D202091BE212223A1F0409116205091F6
:106F100017206091182070911920480F591F6A1F7F
:106F20007B1F409316205093172060931820709376
:106F3000192008951F920F920FB60F920BB60F9261
:106F400011242F933F934F935F936F937F938F936E
:106F50009F93AF93BF93EF93FF9380910D0B90910D
:106F60000E0B019690930E0B80930D0B80910C0BE2
:106F70008F5F80930C0B8038A9F410920C0B8091DA
:106F80001E2090911F20A0912020B09121200196D9
:106F9000A11DB11D80931E2090931F20A09320203F
:106FA000B09321208091BE218823E1F080910B0BCA
:106FB0008F5F80930B0B8038A9F410920B0B80919C
:106FC000162090911720A0911820B09119200196B9
:106FD000A11DB11D8093162090931720A093182017
:106FE000B09319200E94452D009711F00E944C2C5F
:106FF000FF91EF91BF91AF919F918F917F916F9191
:107000005F914F913F912F910F900BBE0F900FBE4C
:107010000F901F901895F8941092B60016BC83EF4D
:1070200087BD82E084BD94E095BD95B395BB809308
:107030006E007894089580910D0B90910E0B209125
:107040000D0B30910E0B82179307A9F7089507C017
:1070500022E330E0000021503040E1F70197009733
:10706000B9F708950F931F93CF93DF938C010E947C
:107070001B38EC010E941B388C1B9D0B801791075D
:10708000C8F3DF91CF911F910F91089508950F9349
:107090001F9300911E2010911F20209120203091DD
:1070A000212080911E2090911F20A0912020B0913E
:1070B0002120081719072A073B0759F7B801C9010A
:1070C0001F910F9108951F920F920FB60F921124E6
:1070D0001092D3040F900FBE0F901F9018951F921F
:1070E0000F920FB60F920BB60F9211242F933F936E
:1070F0004F935F936F937F938F939F93AF93BF93C0
:10710000EF93FF93E091C904F091CA048081E0916C
:10711000D404F091D504309709F00995FF91EF91CF
:10712000BF91AF919F918F917F916F915F914F919F
:107130003F912F910F900BBE0F900FBE0F901F909D
:1071400018951F920F920FB60F9211241092E0041F
:107150000F900FBE0F901F9018951F920F920FB6B1
:107160000F920BB60F9211242F933F934F935F937F
:107170006F937F938F939F93AF93BF93EF93FF93FF
:10718000E091D604F091D7048081E091E104F09180
:10719000E204309709F00995FF91EF91BF91AF910B
:1071A0009F918F917F916F915F914F913F912F911F
:1071B0000F900BBE0F900FBE0F901F90189590E090
:1071C0002DE030E0829FF001839FF00D929FF00D43
:1071D0001124E753FB4FA281B3811C92A481B58196
:1071E0006C93A681B78188ED8C93A085B1854C9373
:1071F000128614861386089590E02DE030E0829F79
:10720000F001839FF00D929FF00D1124E753FB4F87
:1072100081E08287A081B1816C933A968081882336
:10722000E9F70895CF93C82F8A3031F480914F0B3E
:107230006DE00E94FC3802C08D3029F080914F0B28
:107240006C2F0E94FC3880E090E0CF9108951F934E
:10725000CF93DF93182FEB010CC08A3021F4812FDC
:107260006DE00E94FC3869916D3019F0812F0E9409
:10727000FC388881882389F7DF91CF911F91089589
:107280000F931F93CF93DF93CDB7DEB79E01265F99
:107290003F4F0FE01BE0C80160E470E0488559856E
:1072A0000E94AE648F81B8010E942739DF91CF918F
:1072B0001F910F9108951F93CF93DF93182FEB0128
:1072C00004C0812F0E94FC382196FE016491662340
:1072D000C1F7DF91CF911F91089590E02DE030E04C
:1072E000829FF001839FF00D929FF00D1124E753D0
:1072F000FB4F748763870895682F80E00E94FC38F5
:10730000089580934F0B83EE94E090938B288093A5
:107310008A28089584B7877F84BF88E10FB6F894E0
:1073200080936000109260000FBE08952FE088E106
:1073300090E00FB6F894A895809360000FBE20935C
:1073400060000895A895089588E10FB6F894809399
:107350006000109260000FBE0895F89428E088E164
:1073600090E00FB6F894A895809360000FBE20932C
:107370006000FFCF809129208091292090E008951E
:107380008091390181FD10C081E491E06FE140E01E
:107390000E949B3F813059F021E030E0813111F0B3
:1073A00020E030E0C901089580E090E0089581E098
:1073B00090E0089581E491E06FE140E00E949B3FFE
:1073C0000895E9E3F1E0808180818D7F80838DE005
:1073D00090E00197F1F782E491E06FE140E023E073
:1073E0000E94A53F83E090E00197F1F70895909106
:1073F000390191FD0AC0282F803108F02FE085E483
:1074000091E06FE040E00E94A53F0895809139012E
:1074100081FD13C081E491E06FE140E00E949B3F59
:10742000982F8151823038F09F3129F0913019F036
:1074300081E0923019F480E0089581E008950E947F
:10744000063A8823E1F30895CF93DF93C82F88305D
:1074500049F0863039F0893029F0863119F08931C8
:1074600009F045C08091390181FD44C00E941F3A56
:107470000E94DA39D82FC817B9F1C83019F40E9420
:10748000E1392BC0C93141F48631A9F482E491E09D
:107490006FE140E029E009C0C63169F4893159F44F
:1074A00082E491E06FE140E026E00E94A53FE3E046
:1074B000F0E03197F1F782E491E06FE140E02C2FAA
:1074C0000E94A53FD83029F489E691E00197F1F7B1
:1074D00004C0E3E0F0E03197F1F70E94DA398C174D
:1074E00019F083E490E008C080E490E005C082E4F5
:1074F00090E002C084E490E0DF91CF910895809104
:10750000940090919500909357228093562221E009
:10751000209343228091390181FF15C02093BD2122
:1075200080919400909195009093532280935222E1
:1075300020934122809139018D7F80933901809180
:10754000BD218823E1F786E10E94243A81E08093FF
:10755000BE2108958091BE21882351F48091510B62
:10756000882321F081E08093D30B02C00E947F3AF0
:1075700081E090E008950E941F3A1092BE210E947F
:10758000E1398091390182608093390180914122F3
:107590008823E9F1809194009091950020915222E6
:1075A0003091532282179307A0F480911E2290916C
:1075B0001F22A0912022B09121228C57914EAF4FD3
:1075C000BF4F80931E2290931F22A0932022B0933E
:1075D00021228091940090919500821B930BA0E052
:1075E000B0E040911E2250911F22609120227091A4
:1075F0002122840F951FA61FB71F80931E229093F0
:107600001F22A0932022B093212210924122809128
:1076100043228823E9F18091940090919500209174
:1076200056223091572282179307A0F48091262288
:1076300090912722A0912822B09129228C57914E17
:10764000AF4FBF4F8093262290932722A0932822EA
:10765000B09329228091940090919500821B930B06
:10766000A0E0B0E04091262250912722609128228C
:1076700070912922840F951FA61FB71F8093262281
:1076800090932722A0932822B0932922109243227C
:1076900008958091D30B882321F00E947F3A1092A5
:1076A000D30B8091D40B882321F00E94BB3A109217
:1076B000D40B1092510B08950F931F93CF93DF9328
:1076C000F82FE92FAB0181E08093510B009102224A
:1076D0001091032220910422309105220F5F1F4F49
:1076E0002F4F3F4F00930222109303222093042236
:1076F00030930522862F8E5F87FF0CC08091BB21BF
:107700009091BC2101969093BC218093BB21CFEF37
:10771000DFEF09C022E53BE0C9016F2F7E2F0E94F9
:107720008B63C0E0D0E00E94493BCE01DF91CF9156
:107730001F910F9108958091BE21882399F0809127
:10774000510B882321F40E94063A882331F481E00A
:107750008093D40B81E090E008950E94BB3A80E0D2
:1077600090E0089580E090E008951F93CF93DF9319
:107770000F92CDB7DEB78FB789838091510B8823E5
:1077800031F5F8948091BE21882351F08091390120
:1077900081FD1BC00E94063A8823B9F080E003C037
:1077A0000E94AA3A81E0909147019E3010F010E0CB
:1077B00001C01FEF882311F00E949B3B16FF05C0FC
:1077C00089818FBF81E090E004C089818FBF80E014
:1077D00090E00F90DF91CF911F9108958093500B0F
:1077E00008950E94DA398250813130F4E82FF0E0B8
:1077F000E45EFA4F8081089581E0089508958FEF47
:1078000080934E018CE691E060EF44E022E00E941C
:10781000A53F8CE290E06EE041E025E00E94A53FAC
:1078200080E880936F018091460180936D0184E42C
:1078300091E060E245E021E00E94A53F0895CF93EA
:10784000DF93CDEFD3E0CE010197F1F70E94913F96
:10785000109232201092B4201092362110923120D2
:1078600010923020E9E3F1E080818E7F8083808177
:107870008D7F80838DE090E00197F1F780818160BA
:10788000808382E491E06FE140E023E00E94A53F25
:107890002197F1F780915D0180915E010E94FF3B8D
:1078A0008EEF94E060E070E00E94A02A0E947F3A90
:1078B00081E090E0DF91CF9108958091D50B0895FC
:1078C000CF93DF930F92CDB7DEB789830E941F3A23
:1078D00029812093D50B88E491E06FE140E00E947C
:1078E000A53F0F90DF91CF9108950E94603C86E004
:1078F0000E94243A0895FA018093620190936301F3
:1079000060936001709361013097C1F08081809332
:107910006B01818180936A018281809369018381F7
:1079200080936801848180936701858180936601DB
:1079300086818093650187818093640108958EEF2D
:1079400094E00E94C22A81E08093292080912A201D
:1079500090912B20019690932B2080932A2081E0F8
:1079600090E00895CF93DF9350913120252F30E0A0
:10797000F901EE0FFF1F3695322F222737952795F5
:10798000E20FF31FEE5CFF4D4081442309F4F4C085
:107990002091390121FDF0C02091BE21222309F45C
:1079A000EBC047FF23C0852F90E0FC01EE0FFF1FC7
:1079B0009695982F882797958795E80FF91FEE5C85
:1079C000FF4D10828091F2219091F321A091F4213A
:1079D000B091F5210196A11DB11D8093F2219093E4
:1079E000F321A093F421B093F521C6C0433018F5DC
:1079F000852F90E0FC01EE0FFF1F9695982F8827AA
:107A000097958795E80FF91FEE5CFF4D10828091E6
:107A1000EE219091EF21A091F021B091F1210196FA
:107A2000A11DB11D8093EE219093EF21A093F02131
:107A3000B093F121A1C0C42FD0E022976C177D072D
:107A400018F5852F90E0FC01EE0FFF1F9695982FFB
:107A5000882797958795E80FF91FEE5CFF4D1082F8
:107A60008091EA219091EB21A091EC21B091ED2140
:107A70000196A11DB11D8093EA219093EB21A09363
:107A8000EC21B093ED2178C0252F30E0B901660FCD
:107A9000771F3695322F222737952795620F731F50
:107AA0006D5C7F4D50E00E948B6320913120822FCE
:107AB00090E0FC01EE0FFF1F9695982F8827979571
:107AC0008795E80FF91FEE54FF4D808180932220A7
:107AD000822F90E0FC01EE0FFF1F9695982F8827CC
:107AE00097958795E80FF91FEE5CFF4D10822F5F89
:107AF00020933120233010F01092312080913120DA
:107B000090E0FC01EE0FFF1F9695982F8827979520
:107B10008795E80FF91FEE5CFF4D8081882311F0F7
:107B20000E949F3C60914701609323208091282010
:107B3000882311F0681710F46093282084E070E027
:107B40000E94DF306091222083E070E00E94DF30ED
:107B50008091062290910722A0910822B0910922DB
:107B60000196A11DB11D8093062290930722A09338
:107B70000822B093092202C0C0E0D0E0CE01DF911C
:107B8000CF910895CF93DF93EC018881998100977D
:107B900029F024E08B3F920739F505C08BEF94E084
:107BA0009983888325C0623819F5109229200E9494
:107BB00065300E94C62F60E870E00E94B23C181643
:107BC000190644F40E94C12FE0918F05F0919005B1
:107BD0000995E4CF809126209091272001969093DB
:107BE000272080932620DACF1982188283E001C0F3
:107BF00081E0DF91CF91089591E09093510B0E9425
:107C0000F7390E94493B08958091390181FD07C0F1
:107C100085E491E06FE040E00E949B3F089580E1A1
:107C200008950F931F93CF93DF93C82F21E02093E4
:107C3000510BD091BE218091390181FF16C08091F6
:107C40009400909195009093532280935222209318
:107C500041222093BD21809139018D7F809339018C
:107C60008091BD218823E1F7D0E00E941F3A8091E6
:107C7000BE21882309F441C0809143228823E9F181
:107C80008091940090919500209156223091572236
:107C900082179307A0F48091262290912722A09129
:107CA0002822B09129228C57914EAF4FBF4F80931D
:107CB000262290932722A0932822B09329228091F4
:107CC000940090919500821B930BA0E0B0E040914E
:107CD0002622509127226091282270912922840F18
:107CE000951FA61FB71F8093262290932722A0934B
:107CF0002822B09329221092432289E10E94243A3B
:107D000086E00E94EA30009751F00E94043E082F5E
:107D100086E00E94EA3081500E94F73902C000E0FC
:107D200010E080919400909195009093552280935B
:107D3000542281E080934222F8948091390182603C
:107D400080933901809139018D7F809339016C2FA7
:107D50006E5F82E59BE00E94D63F78948091B821C7
:107D60009091B92101969093B9218093B8210E94F6
:107D70001F3A82E491E060EE45E00E949B3FC82FED
:107D800086E00E94EA30009719F0802F0E94F739B0
:107D9000DD2319F00E947F3A02C00E94BB3A809115
:107DA00042228823E9F180919400909195002091DE
:107DB00054223091552282179307A0F480912222F9
:107DC00090912322A0912422B09125228C57914E8C
:107DD000AF4FBF4F8093222290932322A09324225F
:107DE000B09325228091940090919500821B930B73
:107DF000A0E0B0E040912222509123226091242201
:107E000070912522840F951FA61FB71F80932222F1
:107E100090932322A0932422B093252210924222F1
:107E20008091BE21882361F080919400909195000B
:107E3000909357228093562281E08093432207C07B
:107E400082E491E06FE140E023E00E94A53F0E94C0
:107E5000493BC130E1F0C330A9F48091FA219091FF
:107E6000FB21A091FC21B091FD210196A11DB11D26
:107E70008093FA219093FB21A093FC21B093FD21E4
:107E8000C2E00AC0C53029F0C73031F404C0C0E0F8
:107E900003C0C3E001C0C1E08C2F90E0DF91CF911F
:107EA0001F910F910895CF93DF93EB010E945C3BEC
:107EB000009729F4CE010E94113E009751F02091C5
:107EC000BB213091BC212F5F3F4F3093BC212093C9
:107ED000BB21DF91CF910895CF93DF938091BE2195
:107EE000882321F40E94AA3AC1E001C0C0E00E94A8
:107EF000DA39863111F0813119F4D091470109C086
:107F000086E491E06FE140E00E949B3FD82FDD0FB7
:107F1000D80FCC2311F00E949B3B8D2FDF91CF9186
:107F200008951092D70B1092D60BEFE6F0E0808107
:107F3000806280830895FC018081862390E002C0E6
:107F4000959587954A95E2F70895F894FC019081FC
:107F5000862F8095892330E002C0220F331F4A9577
:107F6000E2F72623282B208378940895CF93DF937C
:107F7000EC012196E0917B01DC01EC932E2FA0E82F
:107F8000B1E03D9139932150E1F7E150F0E0E05844
:107F9000FE4F2181FC01E058FF4F20838F579F4FF8
:107FA00021E0FC012083DF91CF910895FC016093D3
:107FB0008001A1E8B1E0615881918D936A17E1F7E2
:107FC00008951F920F920FB60F920BB60F921124C5
:107FD0002F933F934F935F936F937F938F939F93D1
:107FE000AF93BF93EF93FF9380914701809323203A
:107FF0002091302030E0C901880F991F3695322F2B
:10800000222737952795820F931F8E5C9F4D0E94E4
:10801000B63F809130208F5F80933020833010F006
:10802000109230200E949F3CFF91EF91BF91AF9141
:108030009F918F917F916F915F914F913F912F9180
:108040000F900BBE0F900FBE0F901F9018951F92B0
:108050000F920FB60F9211240F900FBE0F901F902A
:1080600018951F920F920FB60F9211240F900FBE0A
:108070000F901F9018951F920F920FB60F92112418
:108080000F900FBE0F901F9018951F920F920FB672
:108090000F9211241092BD210F900FBE0F901F90D0
:1080A00018951F920F920FB60F9211241092BD21B6
:1080B0000F900FBE0F901F9018951F920F920FB642
:1080C0000F9211248F9381E0809329208F910F903C
:1080D0000FBE0F901F9018951F920F920FB60F9220
:1080E00011241092BD210F900FBE0F901F90189574
:1080F0001F920F920FB60F9211248F939F9380912E
:10810000D60B9091D70B01969093D70B8093D60BFB
:108110009F918F910F900FBE0F901F9018950F9306
:108120001F93CF93DF938091C6219091C721A09197
:10813000C821B091C9210196A11DB11D8093C6210E
:108140009093C721A093C821B093C9210E942743CF
:108150008C0188ED9BE00E946A2B08C0EA81FB81BC
:10816000309709F00995CE010E94102CEC01009780
:10817000A9F70115110519F0C8010E94D828DF914F
:10818000CF911F910F9108950E947D490E94653003
:108190000E94404180E795E09093C1218093C021E7
:1081A0000E94244382E090E060E074E040E05EE101
:1081B0002FEF31E00E94E5420895CF92DF92EF92D7
:1081C000FF920F931F93CF93DF936C018B017A0182
:1081D00088ED9BE00E946A2B09C0EC81FD813097FD
:1081E00011F0C8010995CE010E94102CEC010097F6
:1081F000A1F7C601B801A7010E94E228DF91CF9143
:108200001F910F91FF90EF90DF90CF900895BC01E8
:1082100088ED9BE00E94D92B0895BC0188ED9BE07E
:108220000E94A42B0895CF93DF93EC018091C2218B
:108230009091C321A091C421B091C5210196A11DA7
:10824000B11D8093C2219093C321A093C421B09308
:10825000C521CE010E943A43009769F00E94E02FA9
:10826000E0917405F09175058DED90E4BE010995DE
:1082700081E090E002C080E090E0DF91CF9108952E
:108280008AED9BE00E94662B08950F93CF93DF93B6
:10829000EC017B836A8318865F834E838AED9BE0C3
:1082A000BE010E94D92BE091DC0BF091DD0B3097E1
:1082B00049F04C815D818A819B81688520E030E0B6
:1082C00001E00995DF91CF910F910895BC018AEDEE
:1082D0009BE00E94A42B08950F93DC0118961C923A
:1082E0001897E091DC0BF091DD0B309759F0129666
:1082F0008D919C91139760E040E050E020E030E0E9
:1083000000E009950F9108950F93DC01AB011496DD
:108310002D913C91159781E018968C93189715969E
:108320007C936E931497E091DC0BF091DD0B30970A
:1083300039F012968D919C91139761E000E00995B8
:108340000F9108950F93DC01E091DC0BF091DD0BB0
:10835000309769F014962D913C91159712968D9156
:108360009C91139718966C91A90101E009950F91C2
:108370000895E091DE0BF091DF0B309709F009953D
:1083800008959093DF0B8093DE0B08959093DD0B9F
:108390008093DC0B08958AED9BE00E946A2B089580
:1083A000EF92FF920F931F93CF93DF938C01EB011A
:1083B0007A018AED9BE00E946A2B15C0DC011296BF
:1083C0002D913C9113972C173D0759F41696ED917A
:1083D000FC911797309749F0B801AE0197010995C4
:1083E00004C00E94102C009749F7DF91CF911F9194
:1083F0000F91FF90EF9008950895AF92BF92CF92A2
:10840000DF92EF92FF920F931F93CF93DF9300D0F1
:10841000CDB7DEB75B010E94C62FFC01E080F18082
:10842000FA82E982FCE0EF16F10418F400E010E0B3
:108430002DC000D000D088E395E0EDB7FEB7928361
:108440008183F482E3820E940A640F900F900F9060
:108450000F901FC00E94C62FF801EE0FFF1FEE0FF6
:10846000FF1FE80FF91FC280D3800E94C62F0F5F45
:108470001F4FF801EE0FFF1FEE0FFF1FE80FF91F50
:1084800040815181C501B6010E94D0410E151F05E2
:1084900009F70F900F90DF91CF911F910F91FF90EF
:1084A000EF90DF90CF90BF90AF900895CF93DF9380
:1084B000CBEFDBE06091110C7091120CCE0149E71B
:1084C00052E420E030E00E94DA470E947A4960914D
:1084D000110C7091120C0E945360BC01CE014097A8
:1084E0004DE952E420E030E00E94DA47DF91CF917D
:1084F00008958091110C9091120C20910F0C3091E5
:10850000100C880F991F2817390708F4C901909398
:10851000120C8093110C0E94564208950F93013063
:1085200051F480910B0C90910C0C9093120C809351
:10853000110C0E9456420F910895CF93DF930E9431
:1085400065300E94C62FEC01198218820E94CB412F
:1085500020C012962D913C911397FC01EE0FFF1F46
:10856000EE0FFF1FEC0FFD1F3383228314962D9116
:108570003C9115970196FC01EE0FFF1FEE0FFF1FB8
:10858000EC0FFD1F3183208399838883CD010E94E6
:10859000102CDC0188819981109729F018962C9174
:1085A00018972223B1F6880F991F880F991F0296FA
:1085B0000E94C12F88819981009721F080EE9BE075
:1085C0000E94AB28DF91CF910895EF92FF920F9315
:1085D0001F93CF93DF93FC018B017A01E90180EEB9
:1085E0009BE0BF0145E555E00E948D2810930C0CDF
:1085F00000930B0CF0920E0CE0920D0CD093100C2B
:10860000C0930F0C8EE892E40E94C641DF91CF9197
:108610001F910F91FF90EF900895CF93DF93CBEFD1
:10862000DBE0CE010E946148CE0140970E94614884
:10863000CE014B970E94A828DF91CF910895809199
:10864000110C9091120C08950E94EE280895CF937A
:10865000DF93E0915905F0915A050995EC010097D7
:1086600029F06A817B8181E00E94DF30CE01DF91B9
:10867000CF9108950F931F93CF93DF93EC01E09177
:108680005B05F0915C0509958C016A817B8181E035
:108690000E94DF3081E090E00115110511F480E0C7
:1086A00090E0DF91CF911F910F910895E0915D05CA
:1086B000F0915E05099508959C0180E090E005C069
:1086C000F90131974081840F911D2E5F3F4FF901D1
:1086D000329740814423A1F70895FC01308120E0C6
:1086E000818190E0822B932B02C0880F991F6A959D
:1086F000E2F7892F9927FA01E15AFA4F208130E0F9
:108700008223932328E030E0241B350B02C096958A
:1087100087952A95E2F708956F927F928F929F92A4
:10872000AF92BF92CF92DF92EF92FF920F931F937F
:10873000CF93DF935C013B018A0169012830310549
:1087400044F4CB01BA01A9010E946D43F501808375
:108750004EC0790173E0F594E7947A95E1F74115FD
:10876000510521F04501C0E0D0E005C0F301D5017D
:1087700080E090E021C0C3018C0F9D1FB80148E04C
:1087800050E00E946D43F40181934F012196CE1574
:10879000DF058CF3C701F7FE02C080E090E0A60180
:1087A000477050704115510511F1E501C80FD91FEF
:1087B000860D971DB80118C021912D9301968E1535
:1087C0009F05D4F3C701F7FE02C080E090E0A60148
:1087D000477050704115510551F0E501C80FD91F80
:1087E000860D971D60E070E00E946D438883DF91E5
:1087F000CF911F910F91FF90EF90DF90CF90BF909E
:10880000AF909F908F907F906F9008958F929F92DE
:10881000AF92BF92CF92DF92EF92FF920F931F938E
:10882000CF93DF9300D000D0CDB7DEB70E94C62F24
:108830008C0182E090E00E94A32F009709F45FC0B2
:10884000F801918180E02081820F911D0E94022910
:108850007C01009709F455C00E94C62F4C01F70116
:108860008681482F46954695469550E090E0877062
:10887000907021E030E0009711F420E030E0CA0170
:10888000820F931F0E94A32F0097C9F1F701048163
:108890001581CC24DD242EC0F801A180BB24B601B3
:1088A000A3E075956795AA95E1F7680D791DA60176
:1088B00047705070883168F0CE01039695010E9490
:1088C0008C43F8018081BE016D5F7F4F0E94F330C1
:1088D0000DC01A821982CE01019695010E948C4327
:1088E00069817A81F80180810E94DF30CA0CDB1C2B
:1088F0000E5F1F4FF8018081882371F602C0EE24BD
:10890000FF24C7010F900F900F900F90DF91CF9130
:108910001F910F91FF90EF90DF90CF90BF90AF909D
:108920009F908F900895FC0150E080E190E0861BBD
:10893000970B821B930B02C0440F551F8A95E2F7D9
:108940008081852B80838181842B818308956F9220
:108950007F928F929F92AF92BF92CF92DF92EF92CF
:10896000FF920F931F93CF93DF933C016B015A014A
:1089700079012830310524F4C301FA01408159C03E
:108980008901B3E015950795BA95E1F76115710571
:1089900021F04A01C0E0D0E005C0FA01D30180E037
:1089A00090E023C0F40141914F01C3018C0F9D1F42
:1089B000B60128E030E00E9493442196C017D10709
:1089C0008CF3980117FF02C020E030E0D701A770B8
:1089D000B070109781F1F501E20FF31F408150E074
:1089E000C6018A1B9B0B089619C021912D930196F5
:1089F00080179107D4F3980117FF02C020E030E000
:108A0000D701A770B0701097B1F0F501E20FF31F16
:108A1000408150E088E090E08A1B9B0B02C0559596
:108A200047958A95E2F7C301820F931F60E070E0DB
:108A30009D010E949344DF91CF911F910F91FF9070
:108A4000EF90DF90CF90BF90AF909F908F907F90EE
:108A50006F9008956F927F928F929F92AF92BF9284
:108A6000CF92DF92EF92FF920F931F93CF93DF93FA
:108A700000D0CDB7DEB77C01DC0116968C9116973D
:108A8000282F26952695269530E090E087709070E7
:108A900001E010E0009711F400E010E0020F131F56
:108AA000C80102960E942B30009709F451C00E9421
:108AB000CD2FFC01D70112968C91129780831396CB
:108AC0008C9181830E94CD2F32E0632E712C680E31
:108AD000791EC30160E070E0A8010E949463F70171
:108AE000E480F580CC24DD242CC0D7011196AC9015
:108AF0001197BB24860193E0159507959A95E1F7A8
:108B0000060D171D27E0822E912C8C209D20883188
:108B100030F00E94FD30AC01C801B40109C00E94D0
:108B2000EA309A838983C801B401AE014F5F5F4F79
:108B300095010E94A744CA0CDB1CE2E0F0E0EE0EB7
:108B4000FF1ED7018C91882381F681E090E002C05E
:108B500080E090E00F900F90DF91CF911F910F91E7
:108B6000FF90EF90DF90CF90BF90AF909F908F904D
:108B70007F906F900895E0918D05F0918E05099595
:108B80000895E0913605F091370509950895E09133
:108B90009105F091920509950895E0919305F09162
:108BA00094050995089580E090E008950895E09176
:108BB0001805F09119050995089580E090E0089551
:108BC0000F931F93CF93DF93CDB7DEB7E0970FB628
:108BD000F894DEBF0FBECDBF0E9416308C010E94FC
:108BE000C62F602FAE014F5F5F4F0E940A4F882350
:108BF00009F446C088A99801281B3109C9010E94BF
:108C0000A32F0097E9F12E81222379F18A859B8594
:108C10003BEA8D3C930721F03FEF8F3F930781F5AF
:108C2000223069F088E090E00197E1E0F0E0EC0F9D
:108C3000FD1FE80FF91F23852F3F21F007C082E0B9
:108C400090E0F2CF181619067CF30FC089E1BE013F
:108C5000645F7F4F0E94F33089E10E94FD306FEC2A
:108C60007FE10E944528009759F088E1BE016A5EC5
:108C70007F4F0E94F330E0917605F09177050995DA
:108C8000E0960FB6F894DEBF0FBECDBFDF91CF9157
:108C90001F910F910895AF92BF92CF92DF92EF9202
:108CA000FF920F931F93CF93DF93CDB7DEB7E0977B
:108CB0000FB6F894DEBF0FBECDBF5C016B01FE01A5
:108CC000319680E3DF011D928A95E9F781E089837F
:108CD0008CE00E94EA308C831D821F828091150CEB
:108CE00089878F5F8093150C03E008878DEC9BEAE2
:108CF0009B878A8789E10E94FD3063E974E00E94C6
:108D00004528009731F082E08E838FEF8C878D8726
:108D100009C089E10E94FD30BC01CE010C960E9481
:108D20003C280E838DEC9BEA9D8B8C8BCE01469666
:108D30006FEC7FE10E943C280E94C62F9FA78EA760
:108D40000E94163088ABCE0101960E941B4E082F60
:108D500090E00E942B30009749F10E94CD2FBC017A
:108D6000CE010196402F0E94394E00910E051091C0
:108D70000F050E94CD2F7C010E942030BC01C7014D
:108D8000F8010995A114B10489F0009721F0813010
:108D9000910561F404C0C60160E070E003C0C60143
:108DA00064E070E041E050E0F5010995E0960FB60F
:108DB000F894DEBF0FBECDBFDF91CF911F910F9111
:108DC000FF90EF90DF90CF90BF90AF9008950E94FA
:108DD0007A498093150CE0911805F09119050995D1
:108DE0000895009731F0E0911805F0911905099563
:108DF0000895E0911A05F0911B0509950895CF9308
:108E0000DF93EC0104C060E070E00E94A02A899129
:108E100099910097C1F7DF91CF910895CF93DF9398
:108E2000EC0102C00E94E729899199910097D1F73E
:108E3000DF91CF910895CF93DF93EC017B836A8319
:108E40000E941B3899838883DF91CF910895FC019C
:108E50008081918122813381820F931F918380834E
:108E60000895CF93DF93EC010E941B389983888388
:108E7000DF91CF910895CF93DF93EC010E941B38CF
:108E800028813981AC01421B530B9A012F5F3F4F60
:108E900081E090E04A815B814217530710F080E047
:108EA00090E0DF91CF910895CF93DF93FC01C281D1
:108EB000D38180819181C80FD91F0E941B389E01E8
:108EC000281B390BC901DF91CF910895EF92FF92D2
:108ED0000F931F93CF93DF937C018A01FC01808164
:108EE0009181009729F08B34910509F049C01AC08F
:108EF00087E19CE00E946A2BEC0109C06C817D81B6
:108F0000CE0102960E94022D0990D881C02D209793
:108F1000A9F781E08093160C8BE490E0F701918330
:108F2000808333C0683889F587E19CE00E946A2B12
:108F3000EC0123C0CE01029608171907D9F487E186
:108F40009CE0BE010E94A42B00919E0910919F09F4
:108F50008A859B8590939F0980939E09EC85FD856A
:108F6000309719F08E859F85099510939F0900937E
:108F70009E09D2CF0990D881C02D2097D9F6CCCFA9
:108F8000F7011182108283E001C081E0DF91CF916F
:108F90001F910F91FF90EF9008951092160C87E1AA
:108FA0009CE00E94662B86EA95E060E070E00E94FB
:108FB000A02A08950F931F93CF93DF93EC010091A4
:108FC0009E0910919F091B870A875D874C873F8701
:108FD0002E878091160C882379F086EA95E090938D
:108FE0009F0980939E09CE0102960E94022D109344
:108FF0009F0900939E0902C07D836C8387E19CE0FA
:10900000BE010E94A42B87E19CE0BE010E94D92BE7
:10901000DF91CF911F910F9108950F931F93CF93DD
:10902000DF93EC018091160C882391F000919E094A
:1090300010919F0986EA95E090939F0980939E097D
:10904000CE0102960E940D2D10939F0900939E0958
:1090500087E19CE0BE010E94A42B87E19CE0BE0159
:109060000E94D92BDF91CF911F910F9108950F93FB
:109070001F93CF93DF93EC018091160C882391F01E
:1090800000919E0910919F0986EA95E090939F09AF
:1090900080939E09CE0102960E94182D10939F097D
:1090A00000939E0987E19CE0BE010E94A42B87E10A
:1090B0009CE0BE010E94D92BDF91CF911F910F91AF
:1090C0000895CF93DF93EC018091160C882329F04B
:1090D000CE0102960E945F2D04C01F821E82198657
:1090E000188687E19CE0BE010E94A42BDF91CF91FE
:1090F0000895CF93DF93EC018091160C882329F01B
:10910000CE0102960E942D2D12C087E19CE00E94A4
:109110006A2B06C08C179D0741F0FC01808191816C
:109120000097C1F781E090E002C080E090E0DF911D
:10913000CF910895CF93DF93E8E4F2E2CAE0D2E260
:10914000ACE3B2E21192119219921992199219920A
:109150001D9282E2E036F807A9F7DF91CF910895DA
:109160000F931F93CF93DF93FC01E45CFD4D2081AF
:109170008C01000F111F000F111F222311F12091EC
:10918000940030919500E801C65FDD4DFC01EE0FC3
:10919000FF1FE85BFD4D80819181A901481B590BA0
:1091A000CA01A0E0B0E0488159816A817B81840FC7
:1091B000951FA61FB71F88839983AA83BB8331831A
:1091C0002083F801E65FFD4D60817181828193818A
:1091D000DF91CF911F910F91089560E070E080E0E2
:1091E00090E00895FC01EE0FFF1FEE0FFF1FE65FFA
:1091F000FD4D40835183628373830895EF92FF9204
:109200000F931F93CF93DF93BCE3EB2EB2E2FB2EC1
:10921000EAE0F2E2C8E4D2E220E030E0D7018D914A
:109220007D018823C9F000919400109195008881F8
:109230009981A801481B590B60E070E08081918101
:10924000A281B381840F951FA61FB71F80839183CE
:10925000A283B383198308832F5F3F4F34962296EE
:109260002C303105D9F6DF91CF911F910F91FF90EE
:10927000EF9008950E949D4D08950F931F93FC0158
:109280008091190C90911A0C3383228315830483E7
:1092900071836083F0931A0CE093190C009719F412
:1092A000CB010E94B74D80E090E01F910F9108958F
:1092B0008091190C90911A0C0097C1F010921A0C21
:1092C0001092190CDC0114966D917C9115971296F1
:1092D000ED91FC9113970995E091190CF0911A0CFE
:1092E000309721F0808191810E94B74D08950E94AE
:1092F0002D6108950E942861089580EB95E00E94F9
:10930000D82A88EB95E00E94D82A0895CF93DF935E
:109310000E94D32F0097A9F088EB95E00E94F72ACE
:10932000EC01009729F10E941630998388830E94EE
:1093300011309B838A83CE0104960E944D2F8CAB03
:1093400017C080EB95E00E94F72AEC01009771F0BE
:1093500002960E945F2F99838883BE016E547F4FCF
:10936000CE018E579F4F0E94BD3002C0C0E0D0E0BA
:10937000CE01DF91CF910895BC016E547F4F8E577F
:109380009F4F0E94BD300895CF93DF93EC0180EB97
:1093900095E0BE010E94482B009719F080EB95E004
:1093A00009C088EB95E0BE010E94482B009729F088
:1093B00088EB95E0BE010E94222BDF91CF910895AA
:1093C000CF93DF93EC0180EB95E0BE010E94482B28
:1093D000009779F068817981CE0102960E948E30E3
:1093E000BE016E547F4FCE018E579F4F0E94CE30EC
:1093F0001CC088EB95E0BE010E94482B0097A9F0A5
:109400000E946530688179818A819B810E948E30BB
:109410008CA990E00E942B300E94CD2F4CA9BE0158
:109420006C5F7F4F50E00E948B63DF91CF91089576
:10943000CF93DF93EC0180EB95E0BE010E94482BB7
:10944000009719F0CE0102960CC088EB95E0BE01A2
:109450000E94482B009719F08A819B8102C080E00E
:1094600090E0DF91CF910895FC0180819181089572
:1094700070E06F5B7F4F660F771F680F791FCB011E
:109480000895E62FF0E0EF5BFF4FEE0FFF1FE80FB0
:10949000F91F808191810895089584E792E10E94E7
:1094A0002D2D009721F084E792E10E94182D089558
:1094B000E0915F12F0916012309711F009950895D4
:1094C00080E00895EF92FF920F931F93CF93DF9365
:1094D0007C018A01FC0180819181009731F0F3E0E9
:1094E0008C309F0709F0FFC02BC080E0E82FF0E030
:1094F000EE0FFF1FEE0FFF1FEE59FD4E118210827F
:109500008F5F843098F38093611280919E099091CF
:109510009F09E2E6F2E1918B808B0E94E029809323
:10952000602284E792E160E470E00E94022D0E94D4
:109530007F508CE093E0F7019183808381E0D7C076
:10954000623009F4B2C0633030F4662309F482C09B
:10955000613079F795C0673819F0683851F73AC02B
:1095600010927C12C2E6D2E113C08A819B818017DF
:10957000910741F4888199810E94B551198218821E
:109580001B821A82249680917C128F5F80937C12BA
:1095900080917C12843048F3E0E7F7E2848D958D6A
:1095A0008017910719F4158E148E118EB09627E24C
:1095B000E03FF20798F3E6E0F8E2818592858017B4
:1095C000910711F4158214823D9688E2E838F80775
:1095D000A0F3AFCFE2E144375E0709F0AACFCA019A
:1095E0000E942D2D009709F4A4CF10927C122DC05B
:1095F000F0E035E0EE0FFF1F3A95E1F7E059F84D46
:10960000818D8823E9F084E792E10E94182D8091F2
:109610007C1290E025E0880F991F2A95E1F7805988
:10962000984D90936F2780936E2782E00E94E951B6
:109630008091612290916222009711F00E94584A15
:1096400080917C128F5F80937C12E0917C12E430D9
:1096500078F26FCF4115510509F46BCF50936F2706
:1096600040936E2783E00E94E9518091612290919E
:109670006222009711F00E94584A0E944D4A59CF29
:109680004115510509F455CF50936B2740936A2734
:1096900085E00E94E95180916122909162220097B9
:1096A00009F447CF0E94584A44CF8091612290919B
:1096B0006222009709F43DCF80917222863031F406
:1096C00080918A2281FF02C00E944D4A81E00E945F
:1096D000E9518091612290916222009709F429CF8B
:1096E0000E94854C26CFF7011182108283E0DF9122
:1096F000CF911F910F91FF90EF900895909360127A
:1097000080935F1208959C0140919E0950919F099A
:1097100060E0E2E6F2E114C0808191818217930754
:1097200069F4828193818417950741F460937D12D7
:1097300011821082C9010E94B551089534966F5F5D
:10974000643050F360937D12089540E0E2E6F2E168
:1097500016C0542F5F5F208131812115310569F4D6
:1097600040937E129183808320919E0930919F09BE
:10977000338322830E94CF5108953496452F44307D
:1097800040F340937E120895FC0180919E099091D0
:109790009F09958F848F778F668F0895FC01809144
:1097A0009E0990919F0992878187748763870895A6
:1097B000CF93DF93EA010E944151009749F0209135
:1097C0009E0930919F09FC0132872187D487C38786
:1097D000DF91CF9108950F931F93CF93DF9300D024
:1097E00000D0CDB7DEB78C01AB018FEF89838A83C0
:1097F0008B838C83CE010196B8010E94D84B0097D1
:1098000019F0FC01158304830F900F900F900F90B7
:10981000DF91CF911F910F9108958DEC95E062E05B
:1098200040E050E00E94912A109262221092612240
:109830000895AC018DEC95E061E00E946E2A0895D8
:10984000AC018DEC95E060E00E946E2A08950F93C4
:109850001F93CF93DF938A010E94B550EC010097CC
:1098600059F080919E0990919F099D8F8C8F1F8F39
:109870000E8FCE010E94204CCE01DF91CF911F911F
:109880000F910895CF93DF93A0916E27B0916F272A
:10989000109719F0ED016C9605C0C0916A27D09120
:1098A0006B2729968091692786FF22C010927F122C
:1098B00040E0E2E6F2E116C08081918114962D919C
:1098C0003C9115978217930759F4828193810097F1
:1098D00039F040937F12998388831B821A8206C0D5
:1098E00034964F5F443040F340937F120E944D4ABC
:1098F00088819981009731F04A815B816091602273
:109900000E94912ADF91CF9108950F931F93CF93D7
:10991000DF9380917222863009F074C080916122B9
:109920009091622225E08030920709F06BC0C4E973
:10993000D2E0D0936222C093612202E000936B22B6
:1099400014E910936C2210928E2210928D220E94A4
:1099500077508095909590938E2280938D221092CF
:109960007422109273220E94665080959095909375
:109970007422809373220E94584AD0936222C0932B
:10998000612200936B2210936C2290916C2780913E
:109990006D27E92FF82FDF01A459BD4F8CE692E027
:1099A0000D9001920197E1F781E892E26CE672E096
:1099B0000E942350809165228093812280916622AB
:1099C00080938222809167228093832280916822F3
:1099D0008093842210928E2210928D220E947750C2
:1099E0008095909590938E2280938D221092742270
:1099F000109273220E9466508095909590937422E5
:109A0000809373220E94584ADF91CF911F910F914A
:109A10000895FC0120E030E080E0A8E111C0419110
:109A200098E0542F5827B52FB17050FD8A2786959E
:109A3000B13009F480684695915099F72F5F3F4FF8
:109A40002617370761F708951F920F920FB60F92EE
:109A50000BB60F9211242F933F934F935F936F9305
:109A60007F938F939F93AF93BF93EF93FF938091D7
:109A700094009091950090934D2280934C2281E028
:109A800080933E2280917100807D809371000E94BE
:109A9000584980913E228823E9F180919400909169
:109AA000950020914C2230914D2282179307A0F40B
:109AB0008091122290911322A0911422B09115222C
:109AC0008C57914EAF4FBF4F809312229093132229
:109AD000A0931422B0931522809194009091950048
:109AE000821B930BA0E0B0E0409112225091132210
:109AF0006091142270911522840F951FA61FB71F25
:109B00008093122290931322A0931422B0931522D3
:109B100010923E22FF91EF91BF91AF919F918F9153
:109B20007F916F915F914F913F912F910F900BBE5D
:109B30000F900FBE0F901F9018959FB7F894E1E714
:109B4000F0E08081807D808388B38F6288BB109233
:109B50009000E1E9F0E010821092920010929500DE
:109B6000109294008081856080839FBF08952FB7F5
:109B7000F894909399008093980088B38F6288BB83
:109B8000E1E7F0E08081826080832FBF0895CF936A
:109B9000DF93FC01DB0185E0EB0119928A95E9F77F
:109BA000858190E083709070009711F082E08C9333
:109BB000878190E083709070009721F082E0129688
:109BC0008C931297858190E083709070009799F044
:109BD000878190E083709070009769F023893489C1
:109BE000818592852817390731F481E084831296A4
:109BF0001C92129701C01482C581C370C250C2303A
:109C000028F4D0E0C952DA4F888101C080E0119673
:109C10008C931197E781E370E250E23028F4F0E092
:109C2000E952FA4F808101C080E013968C9313971C
:109C3000DF91CF910895CF93DF9300D000D00F92A2
:109C4000CDB7DEB7BE016F5F7F4F0E94C74D8981E0
:109C50009A81890F8D5F9B81890F9C81890F9D81DE
:109C6000890F0F900F900F900F900F90DF91CF9171
:109C70000895DF92EF92FF920F931F93CF93DF939C
:109C800000D000D000D0CDB7DEB78C017B01BE0183
:109C90006F5F7F4F4E830E94C74D79816A81AB8190
:109CA000BC81872F90E00396860F911D8A0F911D2E
:109CB0008B0F911D2D81820F911D4E8150E0481711
:109CC00059070CF498C0F801218130E02170307000
:109CD00083E0220F331F8A95E1F7828190E0817043
:109CE000907034E0880F991F3A95E1F7822B9081AC
:109CF0009770892B438150E04170507095E0440F7C
:109D0000551F9A95E1F7842B448150E041705070C3
:109D100026E0440F551F2A95E1F7842BF701808335
:109D2000F801258130E023703070220F331F220F9D
:109D3000331F868190E08370907054E0880F991FE4
:109D40005A95E1F7822B97819295990F990F907C04
:109D5000982BF7019183F8018085F7018283723097
:109D600051F4F8018185F7018383F8018285F701B9
:109D7000848355E001C053E040E080E090E098012A
:109D8000260F311D09C0F901E80FF91FD384F7012F
:109D9000E70FF11DD0824F5F742F750F01974617A3
:109DA00091F7972FA23089F49701270F311DF80101
:109DB0008389F9018083872F8F5F9701280F311DD9
:109DC000F8018489F90180839E5F40E020E030E063
:109DD0000B0F111D09C0F801E20FF31F5589F701A0
:109DE000E80FF11D50834F5F842F890F21503040C1
:109DF0004B1789F701C080E026960FB6F894DEBFB6
:109E00000FBECDBFDF91CF911F910F91FF90EF90CB
:109E1000DF900895BF92CF92DF92EF92FF920F935F
:109E20001F93CF93DF937C01B62EEA0182E0861761
:109E300008F0AEC0F7018081D82ED294D694D69483
:109E400063E0D622F1E0DF22F7019181292F2695E8
:109E500026952370C92EC294C694C69473E0C72277
:109E6000382F37703883382F3695369536953170C0
:109E70003983382F329531703A8382958695817077
:109E80008B83DC822D83892F829583708E83CF8292
:109E900082818887222369F13381948180E0830F56
:109EA000911D9A878987223079F4CA010B9663E95C
:109EB00074E00E943C28F70186818B8785818C871E
:109EC0008701095F1F4F20C087010B5F1F4F2330A1
:109ED000D9F4F7013D96DA0180E092911B969C93AC
:109EE0001B978F5F11968830C1F78701035F1F4F63
:109EF0000BC087010D5F1F4FCA010B9663E974E029
:109F00000E943C281A861986CC2089F1DD2059F45C
:109F1000F8012081918180E0820F911D9C8B8B8BB9
:109F20000E5F1F4F04C089859A859C8B8B8BF2E056
:109F3000CF1671F4CE01459663E974E00E943C2887
:109F4000F80181818D8B80818E8B0E5F1F4F17C032
:109F5000F3E0CF16A1F4085F1F4FD801FE0180E0A7
:109F60009E91958B8F5F31968830D1F708C0CE01D6
:109F7000459663E974E00E943C281C8A1B8A802F66
:109F80008E199B2D981B9FA71EA70DA7B81608F426
:109F900080E0DF91CF911F910F91FF90EF90DF90C4
:109FA000CF90BF9008959C0141505040460F571FDD
:109FB000FB010EC0B081A0E08181BD01680F711D61
:109FC000260F371F2617370710F42F5F3F4F3296A3
:109FD000E417F50778F3E417F50749F4908180E07A
:109FE000280F391F2817390710F42F5F3F4FC90179
:109FF0000895CF93DF93C0916C22D0E064973091A5
:10A000006B2220E0C20FD31F9E01280F311DC90112
:10A0100065E772E248E050E00E94D34F6DE772E2DC
:10A02000AE010E94D34F009721F0982789279827E7
:10A0300002C08FEF9FEFDF91CF9108959093871229
:10A04000809386120895FC014381460F4093682255
:10A05000872F99272281280F20936722A181A0931F
:10A06000662250815093652230E02817390748F462
:10A070008A2F8F5F80936622882319F45F5F509345
:10A080006522842F90E070708617970798F480916E
:10A0900067228F5F80936722882361F48091662214
:10A0A0008F5F80936622882329F4809165228F5FD9
:10A0B0008093652208959C01AB0180E090E0B90196
:10A0C0000E94D34F982789279827089580E090E031
:10A0D00069E672E244E150E00E94D34F009721F01C
:10A0E00098278927982708958FEF9FEF089586E096
:10A0F0000E94F94F089581E10E94F94F089580E090
:10A10000E82FF0E0EE0FFF1FE051F84D11821082B2
:10A110008F5F8430A8F380E0E82FF0E035E0EE0FA9
:10A12000FF1F3A95E1F7E059F84D118E8F5F8430AB
:10A1300098F380E094E090938A128093891240E033
:10A140008DE090E0242F30E0289FF001299FF00D52
:10A15000389FF00D1124EA5FF74D158214824F5F8E
:10A160004A3080F3409388120895CF93DF93EC0137
:10A170002091891230918A122F5F3F4F8DE7203056
:10A18000380710F020E030E1522F432FA0E012C03A
:10A19000EA2FF0E0B5E0EE0FFF1FBA95E1F7E059C6
:10A1A000F84D818D882329F0848195818417950746
:10A1B00019F3AF5FA43061F730938A1220938912AC
:10A1C0001092881280E0E0E0F0E01EC0A82FB0E01E
:10A1D00055E0AA0FBB1F5A95E1F7A059B84D599603
:10A1E0009C915997992321F480938812FD0110C006
:10A1F000973049F4309731F05A962C915A97928DB6
:10A20000921708F4FD018F5F843000F38093881269
:10A21000309799F182E0818F80918B1284878091B1
:10A220008C12858780918D12868780918E12878708
:10A2300088ED94E0938B828B958B848B81E090E00A
:10A24000918B808B138E81E0828F83E0808F168AC2
:10A2500080E1878B8091891290918A1298278927B3
:10A260009827958384837783668388819981AA81DF
:10A27000BB8180839183A283B383CF01DF91CF9190
:10A2800008950F931F93CF93DF93EC018B012091DF
:10A29000891230918A126DE070E02F5F3F4F8DE799
:10A2A0002030380710F020E030E1522F432FA0E09B
:10A2B00011C08A2F90E0869FF001879FF00D969F36
:10A2C000F00D1124EA5FF74D84819581AF5F84170B
:10A2D000950719F3AA3069F730938A1220938912EF
:10A2E00040E02DE030E018C0542F5F5F842F90E0F5
:10A2F000829FF001839FF00D929FF00D1124EA5F81
:10A30000F74D84819581009731F4409388129F0125
:10A31000309749F424C0452F4A3030F340938812D7
:10A3200020E030E01CC08091891290918A12982719
:10A33000892798279583848317830683209729F498
:10A34000108211821282138208C088819981AA81A9
:10A35000BB8180839183A283B38380E48087C9011A
:10A36000DF91CF911F910F91089540E013C0E42F2A
:10A37000F0E0542F5F5FEE0FFF1FE051F84D20819A
:10A3800031812817390729F44093881211821082ED
:10A390000895452F443058F340938812089540E0C3
:10A3A00013C0E42FF0E0542F5F5FEE0FFF1FE0516A
:10A3B000F84D208131812115310529F4409388120F
:10A3C000918380830895452F443058F34093881239
:10A3D0000895AF92BF92CF92DF92EF92FF920F93C8
:10A3E0001F93CF93DF93C0916E27D0916F27843056
:10A3F00009F4F1C121E932E230936D2720936C27F3
:10A400003093642220936322833071F4898D90E02D
:10A410008F7090708330910509F074C08889998994
:10A42000009709F031C78DC0823009F08EC080914D
:10A430008E128F5F80938E12882399F480918D12F3
:10A440008F5F80938D12882361F480918C128F5FCF
:10A4500080938C12882329F480918B128F5F8093D4
:10A460008B12109262221092612210920528109293
:10A470000428898D873011F0853041F48A8D8F5FF3
:10A480008A8F843109F000C7198EFEC6882309F42B
:10A49000FBC6288939892115310509F44EC09A8DEA
:10A4A000292F21502A8F992309F0EEC69B8D9830D1
:10A4B00031F0282F2150223048F4953039F4198E8C
:10A4C00080E8809369270E94424C94C5953048F4F7
:10A4D00023E030E0092E02C0220F331F0A94E2F776
:10A4E00001C020E32A8F9F5F9B8F90E08F70907058
:10A4F00083309105E1F0843091054CF48130910571
:10A5000009F469C38230910509F0BEC60DC08630DA
:10A51000910509F47EC58830910509F47AC5843027
:10A52000910509F0B1C675C510928A2257C384E01F
:10A53000809369270E94424C92C58F70833009F046
:10A54000A3C688E0809369274AC5853019F5E09154
:10A550006A27F0916B2784819581009709F494C64E
:10A5600010926F2710926E272C50304030936D2739
:10A5700020936C2730936422209363221092052845
:10A5800010920428109262221092612288E0809337
:10A5900069271FC180916922853409F075C6109121
:10A5A0006B2200E080916C22080F111D80916122C6
:10A5B000909162228017910708F466C61093622278
:10A5C0000093612280916F2290E08F7390700097CA
:10A5D00009F05AC680917022882309F055C640912F
:10A5E000002850910128A090D905B090DA054A15AD
:10A5F0005B0559F480910228909103282091DB0596
:10A600003091DC0582179307A1F080917922909117
:10A610007A228417950709F037C620917B22309162
:10A620007C2280910228909103282817390709F08D
:10A630002BC60E9466502FEF8F3F920709F024C669
:10A6400080917222863009F42EC18131D1F181309E
:10A6500009F01AC680917D22883009F015C6109243
:10A660007D2280917F22909180222FEF873F920759
:10A6700010F0099601C008969093802280937F2263
:10A68000E9E6F2E28091752290917622A0917722FC
:10A69000B09178228093792290937A22A0937B22A2
:10A6A000B0937C228091002890910128A0910228EB
:10A6B000B091032884879587A687B78780E4808731
:10A6C000C0C50C511040109362220093612285E8AE
:10A6D00092E290936D2780936C27809183229091D2
:10A6E0008422009739F00E947B502FEF8F3F920712
:10A6F00009F0CAC540917F22509180224115510531
:10A7000009F4C2C586E098E290936B2780936A278C
:10A7100060917D2270917E22A091DB05B091DC05D5
:10A72000C091DD05D091DE050091DF051091E005B7
:10A73000E0907522F0907622C0907722D090782217
:10A740002EC084819581009721F14817590709F59A
:10A7500086819781009719F068177907D1F42081D5
:10A7600031812A153B0529F4828193818A179B0741
:10A77000F9F02C173D0729F4828193818017910706
:10A78000B9F0E216F30629F482819381C816D9063E
:10A7900079F0CF010D9690936B2780936A27E09113
:10A7A0006A27F0916B2788E2E838F80750F26CC509
:10A7B00010926F2710926E2782E08093692785E8B8
:10A7C00092E2909364228093632210920528109263
:10A7D00004280E94424C80910428909105280097FB
:10A7E00009F452C59C01245E3F4F309362222093AE
:10A7F000612230936B2220936C22E0916A27F091C2
:10A800006B2720852093712221E1209372220896E4
:10A8100098278927982790938222809381221092EB
:10A820008422109283228481958190937E2280934A
:10A830007D22868197819093802280937F228091D0
:10A84000002890910128A0910228B09103288093BC
:10A85000752290937622A0937722B09378228081FC
:10A860009181A281B3818093792290937A22A093DF
:10A870007B22B0937C2281E992E290936D278093B2
:10A880006C270E947B5080959095909384228093B2
:10A890008322009709F0D5C48FEF9FEF9093842215
:10A8A00080938322CEC40E9477502FEF8F3F920770
:10A8B00009F0EAC420917F223091802221153105D0
:10A8C00009F4E2C440917D2250917E224115510548
:10A8D00009F4DAC4E0917522F0917622A0917722F2
:10A8E000B0917822C0E7D7E2698D6623A9F08C8108
:10A8F0009D812817390781F48E819F814817590758
:10A9000059F488819981E817F90731F48A819B818C
:10A91000A817B90709F47AC1A09687E2C03DD80705
:10A9200019F310F380918A228F738230B9F4309337
:10A93000901220938F1240E00DC0E42FF0E0EE0F54
:10A94000FF1FE051F84D808191814F5F2817390733
:10A9500009F47DC0443088F34093881280918A22A4
:10A9600082FD92C484E180938A2288E290E09093F1
:10A9700062228093612280E58093892280918422E3
:10A980009091882290938422309183229091872203
:10A990009093832230938722209182229091862265
:10A9A0009093822220938622909181229093881204
:10A9B0004091852240938122909385228F5F8093DE
:10A9C0008822882379F4832F8F5F809387228823BE
:10A9D00049F4822F8F5F80938622882319F49F5F2A
:10A9E0009093852280917D2290917E229093901267
:10A9F00080938F1220917F223091802230937E228B
:10AA000020937D229093802280937F2280917522D3
:10AA100090917622A0917722B0917822809379222A
:10AA200090937A22A0937B22B0937C22809100287D
:10AA300090910128A0910228B0910328809375225B
:10AA400090937622A0937722B0937822DFC310925E
:10AA5000881280E0C0E0D0E022C0E82FF0E075E08E
:10AA6000EE0FFF1F7A95E1F7E059F84D918D99238C
:10AA700021F480938812EF0116C0973079F4209763
:10AA800021F0228D9A8D921748F4C82FD0E065E00E
:10AA9000CC0FDD1F6A95E1F7C059D84D8F5F843028
:10AAA000E0F280938812209709F4EEC3D0936F27C9
:10AAB000C0936E2783E08A8F888F1E8A84E08F8BF5
:10AAC0001B8E80917F22909180229D838C83809128
:10AAD0007D2290917E229F838E838091752290911A
:10AAE0007622A0917722B091782288839983AA83D5
:10AAF000BB8381E0898F80918B128C8780918C122F
:10AB00008D8780918D128E8780918E128F8781E044
:10AB100090E0998B888B809184228B87809183220F
:10AB20008A8780918222898780918122888781E02B
:10AB300090E00E94805A80918922282F30E0207F67
:10AB40003070213531050CF446C082958F7090E04D
:10AB50000597880F991F880F991F3091911220E057
:10AB600031C0E759FD4D30A5332329F420938812D5
:10AB70001092911230C0313011F42F5F23C0323067
:10AB8000E9F441A54430D1F4209388123093911216
:10AB900092A580E023A530E0282B392B309390122A
:10ABA00020938F12C90124E0893D920710F088EDAF
:10ABB00094E09B8B8A8B9D8B8C8B0DC041A544238D
:10ABC00031F0240FE22FF0E0E817F90754F2209358
:10ABD00088123093911280E180938A2280918A2298
:10ABE000826080938A2282E08093912284E0809325
:10ABF00092228093932288ED809394228CE290E0BD
:10AC0000909362228093612280E6ADC2D0936F2739
:10AC1000C0936E271092692740918A2250E042FF2C
:10AC200003C0198E80E248C28091892282958F707C
:10AC3000880F880F809388129801281B31092451AE
:10AC400030403093622220936122862F90E08F70F3
:10AC500090708230910539F4CA018F7390708231FF
:10AC6000910551F429C08130910531F4CA018F73E7
:10AC700090708230910501F12115310529F4CA0146
:10AC8000837090700097C1F0909181228885981709
:10AC900009F05FC2909182228985981709F059C204
:10ACA000909183228A85981709F053C2909184224B
:10ACB0008B85981709F04DC244FF4AC0688979898D
:10ACC0006115710509F444C0CE010C960E94235011
:10ACD00030918522809165223817D1F52091862206
:10ACE000809166222817A1F5909187228091672292
:10ACF000981771F58091882240916822841741F558
:10AD00003C872D879E878F878B8D8823D1F42E8952
:10AD1000888D9A8D891B922F969596959695891B6D
:10AD2000280F2E8B87FD81959F89392F3695369573
:10AD3000931B980F9F8B822F869586958695890FFA
:10AD4000888F81E080936927888D8A8F198A188A75
:10AD5000498D50E0CA018F7090708430910509F4DC
:10AD6000B0C18530910564F482309105C9F183301A
:10AD700091050CF0B6C08130910509F085C211C073
:10AD80008630910509F4DDC1863091050CF4B9C116
:10AD90008730910509F4DDC18830910509F074C24E
:10ADA00085C18091692780FF14C083E0898F80E48A
:10ADB00080936927198A188A809161229091622272
:10ADC000009709F408C122E4209369270E94805A61
:10ADD00002C180918A228F73823009F055C2FBCE66
:10ADE0008091692780FF72C080918A228F7382319F
:10ADF00009F06CC080918922282F30E0207F3070CC
:10AE0000213531050CF446C082958F7090E005978E
:10AE1000880F991F880F991F3091911220E031C03F
:10AE2000E759FD4D30A5332329F420938812109261
:10AE3000911230C0313011F42F5F23C03230E9F469
:10AE400041A54430D1F4209388123093911292A5F9
:10AE500080E023A530E0282B392B309390122093EB
:10AE60008F12C90124E0893D920710F088ED94E02B
:10AE70009B8B8A8B9D8B8C8B0DC041A5442331F01D
:10AE8000240FE22FF0E0E817F90754F2209388121C
:10AE90003093911283E0898F8091812288878091FD
:10AEA00082228987809183228A87809184228B875E
:10AEB00081E090E00E94805A82E480936927198A99
:10AEC000188A109262221092612285C080E28093DB
:10AED00069270E94424CE0916E27F0916F27118EF6
:10AEE0003DCD80918A2280FF25C044FD23C0888902
:10AEF0009989009709F0C8C18091612290916222DE
:10AF000001960E94805A20916927822F8061809348
:10AF100069278091612290916222009719F0226145
:10AF2000209369270E94424C81E090E0998B888BA6
:10AF300088E06DC085FF1CC090918F2280E0209139
:10AF4000902230E0282B392B80916C2790916D272F
:10AF5000820F931F90936D2780936C2780916122BD
:10AF600090916222821B930B9093622280936122C4
:10AF70008091612290916222009749F044FD07C0C0
:10AF8000209169272260209369270E94805A90911E
:10AF90008B2280E020918C22820F911D9093901241
:10AFA00080938F122C893D892817390710F000975C
:10AFB00021F43093901220938F1280918F129091F0
:10AFC00090129B8B8A8B8091692790E083709070A0
:10AFD000009709F459C110920528109204280E9484
:10AFE000424C2091692725FF07C010920528109236
:10AFF0000428198E84E1AEC024FF0DC010920528EC
:10B000001092042881E090E0998B888B84E0898FEE
:10B010001B8E81E19FC080910428909105280097A4
:10B02000E9F020FF02C0198A188A28893989211578
:10B03000310581F42A893B892817390720F4309398
:10B040000528209304288091042890910528998B45
:10B05000888B04C030930528209304281B8E809190
:10B0600063229091642290936D2780936C27809146
:10B07000042890910528009759F0888999890097AC
:10B0800039F08896909362228093612288E10BC008
:10B090008091692781FFF8C088E290E09093622256
:10B0A0008093612280E180938A225CC0809169272D
:10B0B00080FFEAC0198E80E1809369270E94424C8C
:10B0C000E3C08091612290916222009711F00E946A
:10B0D000805A90918A228091692790FF0BC080FF4F
:10B0E00006C087E0898F1A8E198A188A19C086E0EF
:10B0F000898F16C080FF1EC085E0898F198A188A43
:10B10000C3C08091612290916222009711F00E9449
:10B11000805A80918A2280FF0DC087E0898F1A8E25
:10B1200081E090E00E94805A80E1809369270E942C
:10B13000424C0FC08091612290916222009749F4A5
:10B14000A3C08091692780FF9FC087E0898F1A8EF6
:10B150009BC080E180938A2288E290E090936222F3
:10B160008093612280E5809389228885809385225F
:10B170008985809386228A85809387228B85809318
:10B1800088228C85809381228D85809382228E8572
:10B19000809383228F858093842286E0809372221D
:10B1A0008C819D8190937E2280937D228E819F81D0
:10B1B0009093802280937F22809100289091012893
:10B1C000A0910228B0910328809375229093762253
:10B1D000A0937722B093782288819981AA81BB813C
:10B1E0008093792290937A22A0937B22B0937C2241
:10B1F000898D84FF05C010928C2210928B2206C08C
:10B2000084E080938B2288ED80938C2280E480936D
:10B210007122809161229091622290936B2280939F
:10B220006C221092902210928F2210928E221092F5
:10B230008D220E9477508095909590938E228093D6
:10B240008D2285E48093692210926A2210927022E6
:10B2500010926F228091861290918712019690939E
:10B2600087128093861290936D2280936E221092A3
:10B270007422109273220E9466508095909590934C
:10B2800074228093732204C0109262221092612271
:10B2900010926927DF91CF911F910F91FF90EF904E
:10B2A000DF90CF90BF90AF90089598278927982777
:10B2B00008950F931F93DC01CB011A2F0B2F20E071
:10B2C00030E0982789279827A0E0B0E0DC01992793
:10B2D0008827082B192B2A2B3B2BB801C9011F915A
:10B2E0000F910895FC01209163223091642289E638
:10B2F00097E2821B930BAB01861797070CF4AC0106
:10B30000141615065CF44093042850930528E217A0
:10B31000F30721F0C901BF010E948B630895CF920A
:10B32000DF92EF92FF920F93CF93DF93CDB7DEB70B
:10B3300060970FB6F894DEBF0FBECDBF002309F4AF
:10B340005AC029873A874B875C876D877E878F87AE
:10B35000988B80E2801B49855A856B857C85181601
:10B36000B4F019821A821B821C82992787FD90955E
:10B37000909581959F4F04C0440F551F661F771FFE
:10B380008A95D2F74D835E836F8378872CC06A01DC
:10B390007B01002E04C0CC0CDD1CEE1CFF1C0A94AB
:10B3A000D2F7C982DA82EB82FC826A017B0104C097
:10B3B000F694E794D794C7948A95D2F7D701C6013B
:10B3C0004D855E856F85788904C0440F551F661FC3
:10B3D000771F0A95D2F7842B952BA62BB72B8D833D
:10B3E0009E83AF83B88729813A814B815C816D81CF
:10B3F0007E818F81988560960FB6F894DEBF0FBE70
:10B40000CDBFDF91CF910F91FF90EF90DF90CF9064
:10B410000895A0E1B0E0EFE0FAE50C94A46029877C
:10B420003A874B875C876D877E878F87988BA98249
:10B43000BA82CB82DC82ED82FE820F8318874D8533
:10B440005E856F8578898D819E81AF81B88548172B
:10B4500059076A077B07C8F084179507A607B7073F
:10B4600090F049855A856B857C8589819A81AB816D
:10B47000BC81481759076A077B0738F0841795077E
:10B48000A607B70720F482E003C080E001C081E096
:10B490006096EAE00C94C06080E8809361001092AE
:10B4A00061000E9443350E94FE290E94A2398091CA
:10B4B000102090911120009729F00197909311206E
:10B4C00080931020C0901220D0901320E090142080
:10B4D000F09015200E944738DC01CB01C816D90630
:10B4E000EA06FB0601F30E944738DC01CB0180939A
:10B4F000122090931320A0931420B0931520D3CF43
:10B50000BC0180916E2790916F2708960E9423506E
:10B51000E0916E27F0916F2780916522808780915E
:10B520006622818780916722828780916822838743
:10B5300008952F923F924F925F926F927F928F92D7
:10B540009F92AF92BF92CF92DF92EF92FF920F93B2
:10B550001F93CF93DF93CDB7DEB765970FB6F894FF
:10B56000DEBF0FBECDBF4C017F876E87FC01178207
:10B570001682838181FD04C076C34C855D8504C03D
:10B580001E010894211C311CF4019381EE85FF8576
:10B5900093FD859193FF8191FF87EE87882309F4BE
:10B5A0005EC3853241F493FD859193FF8191FF87BE
:10B5B000EE87853259F490E0B4014C8B5D8B0E948C
:10B5C000DE634C895D895D874C87D7CFFF24DD24FE
:10B5D00010E01032B0F48B3269F08C3228F48032F3
:10B5E00051F0833271F40BC08D3239F0803349F45D
:10B5F00011602CC01260146029C0186027C010614F
:10B6000025C017FD2EC0282F20532A3098F416FF8E
:10B6100008C08F2D880FF82EFF0CFF0CF80EF20ECD
:10B6200015C08D2D880FD82EDD0CDD0CD80ED20E56
:10B6300010620CC08E3221F416FD11C3106406C0D6
:10B640008C3611F4106802C0883659F4EE85FF85F7
:10B6500093FD859193FF8191FF87EE87882309F001
:10B66000B8CF982F9554933018F41061805E06C0BF
:10B67000982F9556933008F0A2C11F7E16FD02C088
:10B68000E6E0FE2E1F73853611F4106406C0863680
:10B6900011F4106802C0F110FA9417FF07C0FBE321
:10B6A000FF1548F0EF2CE39427E00DC027E02F159D
:10B6B00030F02F2D07C027E07CE3E72E04C027E001
:10B6C00067E0F62EEE24CA0104969D878C87FA0166
:10B6D0006081718182819381A1010E2D0E949B6204
:10B6E0005C01C9802C2D30E0398B288BC0FE03C053
:10B6F000388933FF06C011FD06C012FF06C000E204
:10B7000005C00DE203C00BE201C000E08889998901
:10B710008C709070009709F43CC0002311F084E015
:10B7200001C083E08D1558F4D81A13FD09C080E2DA
:10B7300090E0B4010E94DE63DA94C9F701C0DD2411
:10B74000002329F0802F90E0B4010E94DE638889F5
:10B7500083FD05C030EBE32E3BE0F32E11C02CEA55
:10B76000E22E2BE0F22E0CC00115110509F08052DB
:10B7700090E0B4010E94DE630894E11CF11C04C057
:10B78000012F10E000711070F7018491882361F798
:10B7900063C217FF0EC0EA0CF889F4FF04C08A8167
:10B7A000813309F4EA941E144CF528E02E1548F173
:10B7B0002CC016FD2AC08F2D90E08A159B0544F001
:10B7C0003CEFA3163FEFB3061CF0106801C0FA94DB
:10B7D000FF2049F0E2E0F0E0EC0FFD1FEF0DF11D5E
:10B7E00080818033A1F317FF10C0EF2CE3948F2DDD
:10B7F00090E0A816B90644F4FA1807C0EE24E394C2
:10B8000004C098E0E92E01C0FF2417FF07C01A14F6
:10B810001B043CF495012F5F3F4F05C025E030E04D
:10B8200002C021E030E0002311F02F5F3F4FFF20E6
:10B8300029F08F2D90E00196280F391F8D2D90E073
:10B840002817390714F4D21A01C0DD24612E772499
:10B85000C30189709070009749F406C080E290E0BF
:10B86000B4010E94DE63DA94DD20C1F7002329F0E1
:10B87000802F90E0B4010E94DE6363FC09C006C023
:10B8800080E390E0B4010E94DE63DA94DD20C1F72A
:10B8900017FF48C08501B7FE02C000E010E0442455
:10B8A000552495012E1931093B8B2A8B3501601ADD
:10B8B000710A620C731C6F2D70E0EE24FF24E61AEF
:10B8C000F70A3FEF0F3F130729F48EE290E0B4012F
:10B8D0000E94DE63A016B10654F02A893B89201726
:10B8E00031072CF4F301E40DF51D818101C080E3E3
:10B8F000015010400894411C511C0E151F052CF0DE
:10B9000090E0B4010E94DE63DCCF0A151B0541F410
:10B910009A81963320F4953319F4388934FF81E302
:10B9200090E049C08A81813311F09FEEC92290E0F6
:10B93000B4010E94DE63FF2089F08EE290E0B40142
:10B940000E94DE6312E0F101E10FF11D1F5F8081B3
:10B9500090E0B4010E94DE63FA94A9F764FE03C08C
:10B9600085E490E002C085E690E0B4010E94DE63C9
:10B97000B7FC05C0A114B10441F4C4FE06C0B094E4
:10B98000A194B108B3948DE201C08BE290E0B401C0
:10B990000E94DE6380E305C08F5FE6EFFFEFAE0E2F
:10B9A000BF1EFAE0AF16B104BCF790E0B4010E94EC
:10B9B000DE63C501C096B4010E94DE634DC18336CB
:10B9C00031F0833789F0833509F059C022C09A01DC
:10B9D0002E5F3F4F3D872C87FA018081898381E06C
:10B9E000E82EF12C510113C09A012E5F3F4F3D8785
:10B9F0002C87FA01A080B18016FF03C06F2D70E084
:10BA000002C06FEF7FEFC5010E94A4637C011F7726
:10BA100014C09A012E5F3F4F3D872C87FA01A0800A
:10BA2000B18016FF03C06F2D70E002C06FEF7FEF93
:10BA3000C5010E947B637C01106813FD1CC006C019
:10BA400080E290E0B4010E94DE63DA948D2D90E0F4
:10BA5000E816F906A8F30FC0F50117FD859117FF49
:10BA600081915F0190E0B4010E94DE63D110DA940D
:10BA70000894E108F108E114F10471F7EDC084368F
:10BA800011F0893671F59A0117FF0AC02C5F3F4FFC
:10BA90003D872C87FA0180819181A281B3810BC0FF
:10BAA0002E5F3F4F3D872C87FA0180819181AA2725
:10BAB00097FDA095BA2F012F0F76B7FF08C0B0955C
:10BAC000A095909581959F4FAF4FBF4F0068BC01E7
:10BAD000CD01A1012AE030E00E94E664E82EE218E0
:10BAE00041C0853721F41F7E2AE030E020C0197F55
:10BAF0008F36A9F0803720F4883509F0B0C00BC02C
:10BB0000803721F0883709F0AAC001C0106114FF06
:10BB100009C0146007C014FF08C0166006C028E002
:10BB200030E005C020E130E002C020E132E0CA018F
:10BB300017FF09C004969D878C87FA016081718187
:10BB40008281938108C002969D878C87FA0160816B
:10BB5000718180E090E0A1010E94E664E82EE21885
:10BB6000012F0F7706FF09C00E7FEF1430F404FF9A
:10BB700006C002FD04C00F7E02C01E2D01C01F2D95
:10BB8000802F90E004FF0CC0FE01EE0DF11D20811E
:10BB9000203311F4097E09C002FF06C01E5F05C0F4
:10BBA00086789070009709F01F5FA02EBB2403FDDC
:10BBB00012C000FF0DC0FE2C1D1550F4FD0CF11A33
:10BBC0001D2D06C080E290E0B4010E94DE631F5F7D
:10BBD0001D15C0F304C01D1510F4D11A01C0DD24D9
:10BBE000A4FE0FC080E390E0B4010E94DE63A2FED9
:10BBF0001FC0A1FE03C088E590E010C088E790E078
:10BC00000DC0C50186789070009791F0A1FC02C02C
:10BC100080E201C08BE207FD8DE290E0B4010E945A
:10BC2000DE6306C080E390E0B4010E94DE63FA9414
:10BC3000EF14C0F3EA94F101EE0DF11D808190E064
:10BC4000B4010E94DE63EE20A9F706C080E290E016
:10BC5000B4010E94DE63DA94DD20C1F78ECCF401DA
:10BC60008681978102C08FEF9FEF65960FB6F8949B
:10BC7000DEBF0FBECDBFDF91CF911F910F91FF901F
:10BC8000EF90DF90CF90BF90AF909F908F907F907C
:10BC90006F905F904F903F902F9008955058BB2722
:10BCA000AA270ED044C135D130F03AD120F031F47A
:10BCB0009F3F11F41EF42AC10EF4E095E7FB20C16A
:10BCC000E92F46D180F3BA176207730784079507F7
:10BCD00018F071F49EF55EC10EF4E0950B2EBA2FAC
:10BCE000A02D0B01B90190010C01CA01A001112482
:10BCF000FF27591B99F0593F50F4503E68F11A162E
:10BD0000F040A22F232F342F4427585FF3CF4695BE
:10BD100037952795A795F0405395C9F77EF41F16E0
:10BD2000BA0B620B730B840BBAF09150A1F0FF0FAA
:10BD3000BB1F661F771F881FC2F70EC0BA0F621F96
:10BD4000731F841F48F4879577956795B795F79586
:10BD50009E3F08F0B3CF9395880F08F09927EE0F18
:10BD6000979587950895A8D008F481E008950CD0A0
:10BD7000DEC0D6D040F0CDD030F021F45F3F19F0D6
:10BD8000BFC0511108C1C2C0E3D098F39923C9F3D1
:10BD90005523B1F3951B550BBB27AA2762177307D1
:10BDA000840738F09F5F5F4F220F331F441FAA1F85
:10BDB000A9F333D00E2E3AF0E0E830D09150504045
:10BDC000E695001CCAF729D0FE2F27D0660F771FF3
:10BDD000881FBB1F261737074807AB07B0E809F0D5
:10BDE000BB0B802DBF01FF2793585F4F2AF09E3F6A
:10BDF000510568F085C0CFC05F3FECF3983EDCF39F
:10BE0000869577956795B795F7959F5FC9F7880FE2
:10BE1000911D9695879597F90895E1E0660F771F34
:10BE2000881FBB1F621773078407BA0720F0621BC5
:10BE3000730B840BBA0BEE1F88F7E0950895E89416
:10BE400009C097FB3EF490958095709561957F4F62
:10BE50008F4F9F4F9923A9F0F92F96E9BB27939510
:10BE6000F695879577956795B795F111F8CFFAF420
:10BE7000BB0F11F460FF1BC06F5F7F4F8F4F9F4F51
:10BE800016C0882311F096E911C0772321F09EE8AF
:10BE9000872F762F05C0662371F096E8862F70E015
:10BEA00060E02AF09A95660F771F881FDAF7880FEF
:10BEB0009695879597F90895990F0008550FAA0B45
:10BEC000E0E8FEEF16161706E807F907C0F01216AD
:10BED0001306E407F50798F0621B730B840B950BB0
:10BEE00039F40A2661F0232B242B252B21F4089505
:10BEF0000A2609F4A140A6958FEF811D811D0895A2
:10BF000097F99F6780E870E060E008959FEF80EC0C
:10BF1000089500240A9416161706180609060895AF
:10BF200000240A9412161306140605060895092E15
:10BF30000394000C11F4882352F0BB0F40F4BF2B84
:10BF400011F460FF04C06F5F7F4F8F4F9F4F0895C4
:10BF500057FD9058440F551F59F05F3F71F04795BA
:10BF6000880F97FB991F61F09F3F79F0879508959F
:10BF7000121613061406551FF2CF4695F1DF08C0BE
:10BF8000161617061806991FF1CF869571056105DB
:10BF900008940895E894BB2766277727CB0197F983
:10BFA00008950BD0C4CFB5DF28F0BADF18F0952381
:10BFB00009F0A6CFABCF1124EECFCADFA0F3959F37
:10BFC000D1F3950F50E0551F629FF001729FBB2780
:10BFD000F00DB11D639FAA27F00DB11DAA1F649F2C
:10BFE0006627B00DA11D661F829F2227B00DA11DDF
:10BFF000621F739FB00DA11D621F839FA00D611D65
:10C00000221F749F3327A00D611D231F849F600D85
:10C01000211D822F762F6A2F11249F5750408AF0BE
:10C02000E1F088234AF0EE0FFF1FBB1F661F771F4A
:10C03000881F91505040A9F79E3F510570F060CF86
:10C04000AACF5F3FECF3983EDCF386957795679532
:10C05000B795F795E7959F5FC1F7FE2B880F911D68
:10C060009695879597F90895629FD001739FF00187
:10C07000829FE00DF11D649FE00DF11D929FF00D78
:10C08000839FF00D749FF00D659FF00D9927729FAF
:10C09000B00DE11DF91F639FB00DE11DF91FBD013A
:10C0A000CF0111240895AA1BBB1B51E107C0AA1F91
:10C0B000BB1FA617B70710F0A61BB70B881F991F49
:10C0C0005A95A9F780959095BC01CD01089597FBED
:10C0D000092E07260AD077FD04D0E5DF06D0002020
:10C0E0001AF4709561957F4F0895F6F790958195B4
:10C0F0009F4F0895A1E21A2EAA1BBB1BFD010DC084
:10C10000AA1FBB1FEE1FFF1FA217B307E407F50707
:10C1100020F0A21BB30BE40BF50B661F771F881FE3
:10C12000991F1A9469F760957095809590959B0179
:10C13000AC01BD01CF0108952F923F924F925F92C3
:10C140006F927F928F929F92AF92BF92CF92DF9227
:10C15000EF92FF920F931F93CF93DF93CDB7DEB78C
:10C16000CA1BDB0B0FB6F894DEBF0FBECDBF099420
:10C170002A88398848885F846E847D848C849B8477
:10C18000AA84B984C884DF80EE80FD800C811B8185
:10C19000AA81B981CE0FD11D0FB6F894DEBF0FBEB4
:10C1A000CDBFED0108958F929F92AF92BF92CF9233
:10C1B000DF92EF92FF92CF93DF93EC018881998118
:10C1C000AA81BB810097A105B10521F484E299ED14
:10C1D000ABE5B7E0BC01CD012DE133EF41E050E02C
:10C1E0000E94196749015A0127EA31E440E050E012
:10C1F0000E9434606B017C01C501B4012CEE34EF68
:10C200004FEF5FEF0E943460DC01CB01C80ED91EF6
:10C21000EA1EFB1EF7FE08C08FEF9FEFAFEFBFE7F0
:10C22000C80ED91EEA1EFB1EC882D982EA82FB8292
:10C23000C6019F77DF91CF91FF90EF90DF90CF9075
:10C24000BF90AF909F908F9008950E94D360089503
:10C2500081EE95E00E94D3600895A0E0B0E0809365
:10C26000E1059093E205A093E305B093E4050895FA
:10C270003F924F925F926F927F928F929F92AF9276
:10C28000BF92CF92DF92EF92FF920F931F93CF93C3
:10C29000DF9300D000D0CDB7DEB72B017A01611556
:10C2A000710529F0DB018C9311969C931197E11491
:10C2B000F10439F09701225030402332310508F063
:10C2C000FCC06C0186010894C11CD11CF8013080AF
:10C2D0003601832D90E00E947363009799F7FDE289
:10C2E0003F1661F4D80111963C90119792E0692EA7
:10C2F000712C600E711ECC24C3940BC0BBE23B16A4
:10C3000039F4F801318082E0682E712C600E711EC4
:10C31000CC24E114F10421F0F0E1EF16F104F9F47A
:10C3200080E3381691F4D3018C91883711F0883569
:10C3300061F4F301318082E090E0680E791E92E0B2
:10C34000C92AB0E1EB2EF12C0AC0E114F10439F452
:10C35000A0E33A16D1F0AAE0EA2EF12C30C0BAE000
:10C36000EB16F10461F1E0E1EE16F10429F0F8E0DA
:10C37000EF16F104B1F409C0FFEF8F2EFFEF9F2EEF
:10C38000FFEFAF2EFFE0BF2E22C078E0E72EF12CAA
:10C39000EFEF8E2EEFEF9E2EEFEFAE2EEFE1BE2EE3
:10C3A00016C09701442737FD4095542F6FEF7FEF5C
:10C3B0008FEF9FEF0E947A6049015A0108C069E936
:10C3C000862E69E9962E69E9A62E69E1B62E40E02F
:10C3D00000E010E020E030E0C701AA2797FDA0951B
:10C3E000BA2F89839A83AB83BC8350EDD52ED30CAF
:10C3F00099E09D1570F4832D81548A3118F499ECDD
:10C40000D92E06C0832D81568A3168F589EAD82E47
:10C41000D30C8D2D90E08E159F052CF54F3FF9F034
:10C4200080169106A206B306B8F0C901B8012981A9
:10C430003A814B815C810E9434608B019C018D2D7F
:10C4400090E0A0E0B0E0080F191F2A1F3B1F08175B
:10C4500019072A073B0710F44FEF01C041E0D30151
:10C460003D903D01C2CF4114510489F0442339F07D
:10C47000089461087108F2017182608208C0C1FEEF
:10C4800006C0C3010297D20111969C938E93C0FE01
:10C4900007C030952095109501951F4F2F4F3F4FA6
:10C4A00047FF0FC082E290E090938F2880938E2800
:10C4B0000FEF1FEF2FEF3FEF04C000E010E020E090
:10C4C00030E0B801C9010F900F900F900F90DF91ED
:10C4D000CF911F910F91FF90EF90DF90CF90BF9081
:10C4E000AF909F908F907F906F905F904F903F9014
:10C4F0000895662777270C947F65FC018827992784
:10C50000E89421912032E9F3293010F02E30C8F35D
:10C510002B3241F02D3239F4689404C00E94D66366
:10C52000820F911D219120532A30C0F31EF4909563
:10C5300081959F4F0895283008F027E03327DA01CE
:10C54000990F311D87FD916000966105710539F4E1
:10C5500032602E5F3D9330E32A95E1F708959F3FC7
:10C5600030F080387105610509F03C5F3C5F3D9318
:10C57000913008F08068911DDF93CF931F930F9344
:10C58000FF92EF92192F987F9695E92F96959695A1
:10C59000E90FFF27E25FF34F99273327EE24FF24AB
:10C5A000A701E70105900894079428F4360FE71EC9
:10C5B000F81E491F511D660F771F881F991F06948B
:10C5C000A1F70590079428F4E70EF81E491F561F9F
:10C5D000C11D770F881F991F661F0694A1F705904C
:10C5E000079428F4F80E491F561FC71FD11D880F46
:10C5F000991F661F771F0694A1F70590079420F4F2
:10C60000490F561FC71FD81F990F661F771F881F16
:10C610000694A9F784911095177041F0D695C795A7
:10C6200057954795F794E7941A95C1F7E4EBFBE02B
:10C6300068941590159135916591959105907FE2DB
:10C640007395E118F10A430B560BC90BD009C0F7DB
:10C65000E10CF11E431F561FC91FD01D7EF470331D
:10C6600011F48A95E6CFE894015030F0080F0AF4EF
:10C670000027021708F4202F2395022F7A3328F081
:10C6800079E37D932A95E9F710C07D932A9589F681
:10C69000069497956795379517951794E118F10AC1
:10C6A000430B560BC90BD00998F023957E917395D7
:10C6B0007A3308F070E37C932013B8F77E917061B1
:10C6C0007D9330F0839571E37D9370E32A95E1F7D4
:10C6D0001124EF90FF900F911F91CF91DF91992737
:10C6E00087FD90950895911189C3803219F0895082
:10C6F0008550D0F70895FC010590615070400110FD
:10C70000D8F7809590958E0F9F1F089542E952E1CA
:10C710000E94AF630895FB01DC0102C001900D92FD
:10C7200041505040D8F70895DC0101C06D9341504D
:10C730005040E0F70895FB01DC018D9101908019D4
:10C740000110D9F3990B0895FC01615070400190DC
:10C750000110D8F7809590958E0F9F1F0895FA01CC
:10C76000A191B081009719F41097E1F0CD01DC019F
:10C77000CD010D90002011F4C00113C0FB012191E7
:10C78000222319F02015D9F7F3CFFB0121912015B1
:10C7900019F41E92119606C02223C1F70D900020B5
:10C7A000A1F7D001FA01A193B08308957AE0979F91
:10C7B000902D879F802D910D112408950F931F9325
:10C7C000CF93DF938C01EB018B8181FF1BC082FF34
:10C7D0000DC02E813F818C819D812817390764F41B
:10C7E000E881F9810193F983E88306C0E885F9853A
:10C7F000802F0995009731F48E819F8101969F8348
:10C800008E8302C00FEF1FEFC801DF91CF911F9100
:10C810000F910895CF93DF93CDB7DEB7FE01359624
:10C820006191719180918A2890918B28AF010E942B
:10C83000995ADF91CF910895CF93DF93CDB7DEB7AB
:10C84000FE0135966191719180918A2890918B2893
:10C85000DC0113962C911397286013962C93AF014B
:10C860000E94995AE0918A28F0918B282381277F92
:10C870002383DF91CF91089560918A2870918B284E
:10C880000E94DE6308950F931F93CF93DF938C0173
:10C89000E0918A28F0918B28838181FF1AC0C0E043
:10C8A000D0E005C00995009711F0CFEFDFEFF80158
:10C8B00081918F0160918A2870918B28DB011896F5
:10C8C000ED91FC911997882369F78AE00995009703
:10C8D00011F0CFEFDFEFCE01DF91CF911F910F91DC
:10C8E00008950F931F93CF93DF93CDB7DEB72E97A5
:10C8F0000FB6F894DEBF0FBECDBF0D891E898F899C
:10C90000988D26E02C831A83098397FF02C080E06C
:10C9100090E801979E838D83AE01455E5F4FCE0107
:10C920000196698D7A8D0E94995A4D815E8157FDDD
:10C930000AC02F813885421753070CF49A01020F61
:10C94000131FF80110822E960FB6F894DEBF0FBEAB
:10C95000CDBFDF91CF911F910F9108950F931F933A
:10C96000CF93DF93CDB7DEB72E970FB6F894DEBF27
:10C970000FBECDBF8C0186E08C831A83098377FFBD
:10C9800002C060E070E8615070407E836D83CE012C
:10C990000196BA01A9010E94995A4D815E8157FD05
:10C9A0000AC02F813885421753070CF49A01020FF1
:10C9B000131FF80110822E960FB6F894DEBF0FBE3B
:10C9C000CDBFDF91CF911F910F910895FA01AA2752
:10C9D000283051F1203181F1E8946F936E7F6E5FC2
:10C9E0007F4F8F4F9F4FAF4FB1E03ED0B4E03CD070
:10C9F000670F781F891F9A1FA11D680F791F8A1F53
:10CA0000911DA11D6A0F711D811D911DA11D20D0B9
:10CA100009F468943F912AE0269F11243019305D73
:10CA20003193DEF6CF010895462F4770405D419364
:10CA3000B3E00FD0C9F7F6CF462F4F70405D4A33B1
:10CA400018F0495D31FD4052419302D0A9F7EACF79
:10CA5000B4E0A6959795879577956795BA95C9F7A8
:10CA600000976105710508959B01AC010A2E06949B
:10CA70005795479537952795BA95C9F7620F731F54
:10CA8000841F951FA01D0895DC01CB01FC01F999BD
:10CA9000FECF06C0F2BDE1BDF89A319600B40D920A
:10CAA00041505040B8F70895F999FECF92BD81BD2D
:10CAB000F89A992780B50895A8E1B0E042E050E0E7
:10CAC0000C944665DC01CB0103C02D910E946D657D
:10CAD00041505040D0F70895262FF999FECF1FBA44
:10CAE00092BD81BD20BD0FB6F894FA9AF99A0FBE97
:10CAF000019608950E946C65272F0C946D656F92C6
:10CB00007F928F929F92AF92BF92CF92DF92EF92DD
:10CB1000FF920F931F93CF93DF935B016115710514
:10CB200021F0DB018C9311969C937C01E701089422
:10CB3000E11CF11C08816701802F90E00E94736363
:10CB40000097A1F70D3241F4098142E0C42ED12CA7
:10CB5000CC0EDD1E11E009C00B3231F4098132E048
:10CB6000C32ED12CCC0EDD1E10E0E6012197CE01A4
:10CB70006EEA7CE043E050E00E9401670097D1F448
:10CB8000E6012296CE0161EB7CE045E050E00E9498
:10CB90000167009711F4E6012796A114B10419F07A
:10CBA000F501D183C08330E020E090E8112309F43F
:10CBB0000DC107C1CE0166EB7CE043E050E00E946E
:10CBC0000167009759F4A114B10409F4FCC0C6012F
:10CBD0000296D50111969C938E93F5C040E050E0EB
:10CBE00060E070E08824992400530A3090F51260C8
:10CBF000212F30E0C9018870907012FF06C00097A5
:10CC000069F50894811C911C29C0009719F00894BB
:10CC100081089108DB01CA01D2E0880F991FAA1F81
:10CC2000BB1FDA95D1F7480F591F6A1F7B1F440FAE
:10CC3000551F661F771F400F511D611D711D48391B
:10CC4000B9E95B07B9E96B07B9E17B0738F0146014
:10CC500005C00E3F39F413FD43C01860F601019181
:10CC60006F01C2CF053311F00531D1F5D601EC913A
:10CC7000ED3211F4106108C0EB3229F0C6010196C3
:10CC800021E030E008C0D6011196EC911197C60161
:10CC9000029622E030E0E053EA3020F06C01C21A44
:10CCA000D30A1EC0DC0120E030E0FCE020383F0762
:10CCB0005CF4C901880F991F880F991F280F391F2D
:10CCC000220F331F2E0F311DED91E0536D01EA301D
:10CCD00060F314FF03C0309521953F4F820E931EE1
:10CCE000C12FD0E011FF08C0A114B10429F0C60182
:10CCF0000197D5018D939C93CB01BA010E941F5FD0
:10CD00006B017C01CE01837090708330910521F41A
:10CD1000F7FAF094F7F8F094C701B60120E030E09C
:10CD200040E050E00E94B35E882309F445C097FEBE
:10CD300007C09094819491089394C5EEDCE002C002
:10CD4000CDECDCE098EE692E9FEF792E6C0E7D1E07
:10CD500020E2A22EB12C0FC0FE0105911591259164
:10CD60003491C701B601A90198010E94D15F6B01FE
:10CD70007C018A189B088A149B0474F72497B59445
:10CD8000A794C615D705B9F7C601D7012A2F220FD8
:10CD90002B2F221F2F3F51F0BC01CD0120E030E0AE
:10CDA00040E050E00E94B35E882331F482E290E0DC
:10CDB00090938F2880938E283C2D2D2D9E2D8F2D86
:10CDC00006C08FEF04C030E020E090EC8FE7B9019F
:10CDD000AC01872F922FA52FB42FBC01CD01DF917D
:10CDE000CF911F910F91FF90EF90DF90CF90BF9068
:10CDF000AF909F908F907F906F900895992788278C
:10CE00000895FB01DC014150504088F08D91813440
:10CE10001CF08B350CF4805E659161341CF06B3531
:10CE20000CF4605E861B611171F3990B0895881BE9
:10CE3000FCCF97FB092E05260ED057FD04D05AD9FA
:10CE40000AD0001C38F450954095309521953F4FFD
:10CE50004F4F5F4F0895F6F79095809570956195C7
:0CCE60007F4F8F4F9F4F0895F894FFCF35
:10CE6C00263A202573205B414444523D252D642EE7
:10CE7C00252D64205345513D252D64205253534993
:10CE8C003D252D75204C51493D252D752044525082
:10CE9C003D252D642E253032645D0A005363686590
:10CEAC0064756C6564206576656E74206174203DD4
:10CEBC00256C642066756E633D25780D0A005363FE
:10CECC00686564756C6564206576656E74206E6F3C
:10CEDC00773D256C64206E6578743D256C640D0A75
:10CEEC00002845787450777229000049443D00258C
:10CEFC00303278002050533D25640020543D252DC0
:10CF0C00362E3266002054313D252D362E326600E9
:10CF1C0020545F4D43553D252D352E31660020564E
:10CF2C005F4D43553D252D342E3266002050303D4B
:10CF3C00252D6C58002050305F543D252D372E3355
:10CF4C0066002050313D252D6C58002055503D2554
:10CF5C002D6C58002052483D252D342E3166002072
:10CF6C00565F494E3D252D352E32660020565F41C9
:10CF7C00313D252D352E32660020565F41323D2540
:10CF8C002D352E326600263A2025730A00253032C4
:10CF9C0058006C656E3D25640A007374617475737A
:10CFAC003D3078253032780A2000312E3020466909
:10CFBC00726D77617265205665722E20322E362086
:10CFCC00323031322D30372D303500656570726F4F
:10CFDC006D006F6E006F6666004F6E0061310072FF
:10CFEC006573657400613200765F696E00617574FB
:10CFFC006F00666C75736800414444523D252D6486
:10D00C002E252D64205345513D252D64205253531C
:10D01C00493D252D75204C51493D252D750A00742F
:10D02C0072696D0043683D252D64205478507772E9
:10D03C003D252D640A0050043A0424040C04F0032A
:10D04C000000536C6565702070726F6365737300BC
:10D05C000000E203860E0000000062726F616463E0
:10D06C006173742070726F63657373000000FA0350
:10D07C00810F00000000737464696E2070726F631E
:10D08C0065737300000016049E0D00000000666FAF
:10D09C006F2070726F636573730000002E045B0861
:10D0AC0000000000636D642070726F636573730021
:10D0BC0000004404B0270000000002003C008F0276
:10D0CC006162636465666768696A6B6C6D6E6F70CC
:10D0DC0020090D0070041A22FFCC3B22FFCC3BED43
:10D0EC00478A3C01001000B10600000D0040001CF6
:10D0FC00065C06000069285D281810000000004539
:10D10C0076656E742074696D65720000009F045121
:10D11C002C00000000020306070A0B0E0F436F6E73
:10D12C0074696B6920322E3500C600C500C400C17D
:10D13C0000C200000000CE00CD00CC00C900CA0027
:10D14C000000000000000200000000123900000086
:10D15C0000524632333020647269766572000000EA
:10D16C00F104C23D000000001F3C5C3B113E533FEC
:10D17C00B23CB53BC039BA39AA3A9B3B000101011C
:10D18C000101010101010101010101010052696D5F
:10D19C0065002D05C4408F4061646174612E6E750D
:10D1AC006D20776179206F75742074686572653AAB
:10D1BC002025640A00FD41FC4106442A455C4300DD
:10D1CC0080C0E0F0F8FCFEFF6E756C6C6D61630066
:10D1DC006805D645BB45C145C745CD45D3457369A3
:10D1EC0063736C6F776D6163007E05E7464B46E0B9
:10D1FC0045D745F146DD454374696D657220707203
:10D20C006F636573730000009705664700000000AC
:10D21C00BA0008001B0C230C35000200F311F511A9
:10D22C005443502F495020737461636B000000C04D
:10D23C0005624A00000000020800000000FFFFFF2A
:06D24C00FF0100000000DC
:00000001FF
